:020000040800F2
:1000000000060020E1010008E3010008E301000808
:10001000E3010008E3010008E3010008E301000830
:10002000E3010008E3010008E3010008B92F00081C
:10003000E3010008E3010008E3010008E301000810
:10004000E3010008E3010008E3010008E301000800
:10005000E3010008E301000861320008893200086A
:10006000B1320008D932000801330008E30100086A
:10007000E3010008E3010008E3010008E3010008D0
:10008000E3010008E3010008E3010008E3010008C0
:10009000E3010008E3010008E30100082933000838
:1000A000E3010008E3010008E3010008E3010008A0
:1000B000FD330008E3010008E3010008E301000844
:1000C000E3010008E3010008E3010008E301000880
:1000D000E3010008E3010008E3010008E301000870
:1000E0008D330008E3010008E3010008E301000884
:1000F000E3010008E3010008E3010008E301000850
:10010000E3010008E3010008E3010008E30100083F
:10011000E3010008E3010008E3010008E30100082F
:10012000E3010008E3010008E3010008E30100081F
:10013000E3010008E3010008E3010008E30100080F
:10014000E3010008E3010008E30100086D2700084F
:10015000E3010008E3010008E3010008E3010008EF
:10016000E3010008E3010008E3010008E3010008DF
:10017000E3010008E3010008E3010008E3010008CF
:10018000E3010008E3010008E3010008E3010008BF
:10019000E3010008E3010008E3010008E3010008AF
:1001A000E3010008E3010008E3010008E30100089F
:1001B000E3010008E3010008E3010008E30100088F
:1001C000E3010008E3010008E3010008E30100087F
:1001D000E3010008E3010008E3010008E30100086F
:1001E00002E000F000F8FEE772B6374880F30888B6
:1001F000364880F3098836483649086040F20000E6
:10020000CCF200004EF63471CEF200010860BFF36C
:100210004F8FBFF36F8F40F20000C0F2F0004EF638
:100220008851CEF200010860BFF34F8FBFF36F8F8C
:100230004FF00000E1EE100A4EF63C71CEF20001E4
:100240000860062080F31488BFF36F8F01F056FF1B
:1002500002F050FE4FF055301F491B4A91423CBFFF
:1002600041F8040BFAE71D49184A91423CBF41F896
:10027000040BFAE71A491B4A1B4B9A423EBF51F83E
:10028000040B42F8040BF8E700201849184A914281
:100290003CBF41F8040BFAE701F034FF02F07EFEA8
:1002A000144C154DAC4203DA54F8041B8847F9E7A7
:1002B00000F042F8114C124DAC4203DA54F8041B22
:1002C0008847F9E701F01CBF00060020002200204B
:1002D0000000000808ED00E00000002000060020FB
:1002E000C0370008002200204022002040220020C9
:1002F000602E0020E0010008E0010008E001000895
:10030000E00100082DE9F04F2DED108AC1F80CD066
:10031000C3689D46BDEC108ABDE8F08F002383F3CF
:1003200011882846A047002001F084FAFEE701F07A
:10033000EDF900DFFEE7000038B500F061FB01F0E9
:10034000ADFE054601F0D0FE0446D8B90F4B9D42E4
:100350001AD001339D4218BF044641F2883504BFCC
:1003600001240025002001F0A3FE0CB100F076F876
:1003700000F0ECFC00F09AFB284600F0B7F800F023
:100380006DF8F9E70025EDE70546EBE7010007B05A
:1003900008B500F05DFBA0F120035842584108BDAC
:1003A00007B541F21203022101A8ADF8043000F0B4
:1003B0006DFB03B05DF804FB38B5302383F311887F
:1003C000174803680BB101F001FB164A14480023DB
:1003D0004FF47A7101F0F0FA002383F31188124C84
:1003E000236813B12368013B2360636813B163681A
:1003F000013B63600D4D2B7833B963687BB90220F4
:1004000000F01EFC322363602B78032B07D1636856
:100410002BB9022000F014FC4FF47A73636038BDEE
:1004200040220020B9030008602300205822002049
:10043000084B187003280CD8DFE800F00805020804
:10044000022000F0F3BB022000F0E6BB024B0022CA
:100450005A60704758220020602300201F4B204A1A
:1004600010B51C461968013136D004339342F9D1D6
:100470006268A24230D31B4B9B6803F1006303F513
:1004800040439A4228D2002000F02AFB0220FFF7C6
:10049000CFFF154B1A6C00221A64196E1A66196E7A
:1004A000596C5A64596E5A665A6E1A6942F0005273
:1004B0001A611A6922F000521A611B6972B64FF074
:1004C000E0233021C3F8084DD4E9003281F31188CC
:1004D0009D4683F30888104710BD00BF00C0000888
:1004E00020C0000800220020003802402DE9F04F13
:1004F00093B0AA4B00902022FF210AA89D6800F02B
:10050000CFFBA74A1378A3B9A64801210360117055
:10051000302383F3118803680BB101F057FAA24A24
:10052000A04800234FF47A7101F046FA002383F3C8
:100530001188009B13B19D4B009A1A609C4A009C45
:100540001378032B1EBF00231370984A4FF0000A44
:1005500018BF5360D3465646D146012000F066FBD3
:1005600024B1924B1B68002B00F01182002000F098
:100570006FFA0390039B002BF2DB012000F04CFB91
:10058000039B213B162BE8D801A252F823F000BFB1
:10059000ED05000815060008A90600085B0500081F
:1005A0005B0500085B050008330700080309000825
:1005B0001D0800087F080008A7080008CD080008EB
:1005C0005B050008DF0800085B050008510900080A
:1005D0008D0600085B05000895090008F90500086C
:1005E0008D0600085B0500087F0800080220FFF761
:1005F000CFFE002840F0F581009B0221BAF1000FE8
:1006000008BF1C4605A841F21233ADF8143000F0C3
:100610003DFAA2E74FF47A7000F01AFA071EEBDBFE
:100620000220FFF7B5FE0028E6D0013F052F00F2BB
:10063000DA81DFE807F0030A0D101336052305936E
:10064000042105A800F022FA17E054480421F9E734
:1006500058480421F6E758480421F3E74FF01C08F6
:10066000404600F03FFA08F104080590042105A86F
:1006700000F00CFAB8F12C0FF2D1012000FA07F7C4
:1006800047EA0B0B5FFA8BFB4FF0000900F054FBBD
:1006900026B10BF00B030B2B08BF0024FFF780FEE5
:1006A0005BE746480421CDE7002EA5D00BF00B03F5
:1006B0000B2BA1D10220FFF76BFE074600289BD031
:1006C000012000F00DFA0220FFF7B2FE00261FFA0B
:1006D00086F8404600F014FA044690B100214046E6
:1006E00000F01EFA01360028F1D1BA46044641F264
:1006F0001213022105A8ADF814303E4600F0C6F9E9
:100700002BE70120FFF794FE2546244B9B68AB4264
:1007100007D9284600F0E6F9013040F0678104353A
:10072000F3E7234B00251D70204BBA465D603E4623
:10073000ACE7002E3FF460AF0BF00B030B2B7FF404
:100740005BAF0220FFF774FE322000F081F9B0F1B8
:100750000008FFF651AF18F003077FF44DAF0F4AC2
:10076000926808EB050393423FF646AFB8F5807FE9
:100770003FF742AF124B0193B84523DD4FF47A7037
:1007800000F066F90390039A002AFFF635AF019B4B
:10079000039A03F8012B0137EDE700BF0022002088
:1007A0005C23002040220020B903000860230020C1
:1007B0005822002004220020082200200C220020C1
:1007C0005C220020C820FFF7E3FD074600283FF425
:1007D00013AF1F2D11D8C5F1200242450AAB25F0F9
:1007E000030028BF424683490192184400F032FAC0
:1007F000019A8048FF2100F053FA4FEAA8037D498F
:100800000193C8F38702284600F052FA06460028F2
:100810003FF46DAF019B05EB830537E70220FFF73F
:10082000B7FD00283FF4E8AE00F0A6F900283FF439
:10083000E3AE0027B846704B9B68BB4218D91F2F08
:1008400011D80A9B01330ED027F0030312AA1344D8
:1008500053F8203C05934046042205A900F0A0FA75
:1008600004378046E7E7384600F03CF90590F2E7A8
:10087000CDF81480042105A800F008F906E700234C
:10088000642104A8049300F0F7F800287FF4B4AEC4
:100890000220FFF77DFD00283FF4AEAE049800F083
:1008A00053F90590E6E70023642104A8049300F0BF
:1008B000E3F800287FF4A0AE0220FFF769FD0028CE
:1008C0003FF49AAE049800F04FF9EAE70220FFF7F0
:1008D0005FFD00283FF490AE00F05EF9E1E70220F2
:1008E000FFF756FD00283FF487AE05A9142000F05D
:1008F00059F904210746049004A800F0C7F83946C6
:10090000B9E7322000F0A4F8071EFFF675AEBB076A
:100910007FF472AE384A926807EB090393423FF6C0
:100920006BAE0220FFF734FD00283FF465AE27F0E0
:1009300003074F44B9453FF4A9AE484600F0D2F84A
:100940000421059005A800F0A1F809F10409F1E7D8
:100950004FF47A70FFF71CFD00283FF44DAE00F015
:100960000BF9002844D00A9B01330BD008220AA9B6
:10097000002000F09DF900283AD02022FF210AA88B
:1009800000F08EF9FFF70CFD1C4800F059FF13B082
:10099000BDE8F08F002E3FF42FAE0BF00B030B2BB6
:1009A0007FF42AAE0023642105A8059300F064F8C3
:1009B000074600287FF420AE0220FFF7E9FC8046BE
:1009C00000283FF419AEFFF7EBFC41F2883000F04D
:1009D00037FF059800F0E2F9464600F0ADF93C46D5
:1009E000BBE5064652E64FF0000905E6BA467EE64C
:1009F00037467CE65C22002000220020A086010011
:100A00007047000070B50F4B1B780133DBB2012B30
:100A10000C4611D80C4D29684FF47A730E6AA2FB6C
:100A20000332014622462846B047844204D1074B90
:100A300000221A70012070BD4FF4FA7000F000FF20
:100A40000020F8E710220020082600209423002030
:100A500007B50023024601210DF107008DF807308C
:100A6000FFF7D0FF20B19DF8070003B05DF804FB4D
:100A70004FF0FF30F9E700000A4608B50421FFF700
:100A8000C1FF80F00100C0B2404208BD30B4054C47
:100A90002368DD69044B0A46AC460146204630BC5B
:100AA000604700BF08260020A086010070B501F055
:100AB000E7F9094E094D30800024286833888342C5
:100AC00008D901F0D7F92B6804440133B4F5404F3D
:100AD0002B60F2D370BD00BF962300206823002056
:100AE00001F090BA00F1006000F5404000687047E6
:100AF00000F10060920000F5404001F00FBA0000E4
:100B0000054B1A68054B1B889B1A834202D9104477
:100B100001F0B0B900207047682300209623002020
:100B200038B5084D044629B128682044BDE838404E
:100B300001F0C0B92868204401F0A4F90028F3D0DE
:100B400038BD00BF6823002010F003030AD1B0F5C0
:100B5000047F05D200F10050A0F51040D0F8003815
:100B6000184670470023FBE700F10050A0F5104045
:100B7000D0F8100A70470000064991F8243033B1CC
:100B80000023086A81F824300822FFF7B1BF012052
:100B9000704700BF6C230020014B1868704700BFEE
:100BA000002004E070B5194B1D68194B0138C5F3DE
:100BB0000B0408442D0C04221E88A6420BD15C684D
:100BC0000A46013C824213460FD214F9016F4EB11E
:100BD00002F8016BF6E7013A03F10803ECD1814218
:100BE0000B4602D22C2203F8012B0A4A0524168850
:100BF000AE4204D1984284BF967803F8016B013C61
:100C000002F10402F3D1581A70BD00BF002004E0C5
:100C1000E0340008CC340008022802BF024B4FF039
:100C200000729A61704700BF00000240022802BFB4
:100C3000024B4FF400729A61704700BF00000240FF
:100C4000022801BF024A536983F40073536170475D
:100C50000000024010B50023934203D0CC5CC45482
:100C60000133F9E710BD000010B5013810F9013F5C
:100C70003BB191F900409C4203D11AB10131013AD4
:100C8000F4E71AB191F90020981A10BD1046FCE75C
:100C900003460246D01A12F9011B0029FAD1704707
:100CA00002440346934202D003F8011BFAE770475F
:100CB0002DE9F8431F4D144695F824200746884631
:100CC00052BBDFF870909CB395F824302BB92022EA
:100CD000FF2148462F62FFF7E3FF95F82400C0F19B
:100CE0000802A24228BF2246D6B24146920005EB36
:100CF0008000FFF7AFFF95F82430A41B1E44F6B226
:100D0000082E17449044E4B285F82460DBD1FFF745
:100D100033FF0028D7D108E02B6A03EB820383421C
:100D2000CFD0FFF729FF0028CBD10020BDE8F88302
:100D30000120FBE76C230020024B1A78024B1A704B
:100D4000704700BF942300201022002010B50F4CE4
:100D50000F4800F0B5F821460D4800F0DDF8246892
:100D60000C48626DD2F8043843F00203C2F804382C
:100D700000F066FD0849204600F0D4F9626DD2F813
:100D8000043823F00203C2F8043810BDAC35000863
:100D90000826002040420F00B435000870470000CC
:100DA00030B5094D0A4491420DD011F8013B58402D
:100DB000082340F30004013B2C4013F0FF0384EAB6
:100DC0005000F6D1EFE730BD2083B8ED02684368EC
:100DD0001143016003B118477047000013B5446B1D
:100DE000D4F894341A681178042915D1217C022989
:100DF00012D11979128901238B4013420CD101A918
:100E000004F14C0001F032FFD4F89444019B2179A5
:100E10000246206800F0D0F902B010BD143001F095
:100E2000B5BE00004FF0FF33143001F0AFBE00003C
:100E30004C3001F087BF00004FF0FF334C3001F021
:100E400081BF0000143001F083BE00004FF0FF317D
:100E5000143001F07DBE00004C3001F053BF0000A3
:100E60004FF0FF324C3001F04DBF000000207047C2
:100E700010B5D0F894341A6811780429044617D1B3
:100E8000017C022914D15979528901238B401342E4
:100E90000ED1143001F016FE024648B1D4F8944445
:100EA0004FF4807361792068BDE8104000F072B99A
:100EB00010BD0000406BFFF7DBBF00007047000073
:100EC0007FB5124B036000234360C0E90233012564
:100ED00002260F4B057404460290019300F1840230
:100EE000294600964FF48073143001F0C7FD094B7A
:100EF0000294CDE9006304F523724FF48073294610
:100F000004F14C0001F08EFE04B070BD0035000805
:100F1000B50E0008DD0D00080B68302282F3118841
:100F20000A7903EB820290614A79093243F8220080
:100F30008A7912B103EB820398610223C0F89414FA
:100F40000374002080F311887047000038B5037FD8
:100F5000044613B190F85430ABB9201D012502218D
:100F6000FFF734FF04F1140025776FF0010100F062
:100F70008FFC84F8545004F14C006FF00101BDE87F
:100F8000384000F085BC38BD10B50121044604305E
:100F9000FFF71CFF0023237784F8543010BD0000B6
:100FA00038B504460025143001F080FD04F14C00F2
:100FB000257701F04FFE201D84F854500121FFF7E2
:100FC00005FF2046BDE83840FFF752BF90F8443097
:100FD00003F06003202B07D190F84520212A4FF021
:100FE000000303D81F2A06D800207047222AFBD10D
:100FF000C0E90E3303E0034A82630722C26303643D
:10100000012070471122002037B5D0F894341A68B7
:101010001178042904461AD1017C022917D11979C3
:10102000128901238B40134211D100F14C0528464F
:1010300001F0D0FE58B101A9284601F017FED4F8FE
:101040009444019B21790246206800F0B5F803B072
:1010500030BD0000F0B500EB810385B09E69044609
:101060000D46FEB1302383F3118804EB8507301D54
:101070000821FFF7ABFEFB685B691B6806F14C00BB
:101080001BB1019001F000FE019803A901F0EEFDF3
:10109000024648B1039B2946204600F08DF8002304
:1010A00083F3118805B0F0BDFB685A691268002A05
:1010B000F5D01B8A013B1340F1D104F14402EAE769
:1010C000093138B550F82140DCB1302383F3118861
:1010D000D4F894241368527903EB8203DB689B698C
:1010E0005D6845B104216018FFF770FE294604F1E0
:1010F000140001F0F1FC2046FFF7BAFE002383F351
:10110000118838BD7047000001F050B8012303700A
:101110000023C0E90133C36183620362C362436297
:101120000363704738B50446302383F311880025E4
:10113000C0E90355C0E90555416001F047F80223B5
:10114000237085F31188284638BD000070B500EB88
:10115000810305465069DA600E46144618B1102224
:101160000021FFF79DFDA06918B110220021FFF7B3
:1011700097FD31462846BDE8704001F0F1B8000007
:10118000826802F0011282600022C0E904228261BA
:1011900001F072B9F0B400EB81044789E4680125DD
:1011A000A4698D403D43458123600023A2606360B4
:1011B000F0BC01F08DB90000F0B400EB81040789A8
:1011C000E468012564698D403D4305812360002367
:1011D000A2606360F0BC01F007BA000070B50223A2
:1011E000002504460370C0E90255C0E90455C564F2
:1011F000856180F8345001F04FF863681B6823B1B3
:1012000029462046BDE87040184770BD0378052B7D
:1012100010B504460AD080F85030052303704368A7
:101220001B680BB1042198470023A36010BD000088
:101230000178052906D190F85020436802701B6898
:1012400003B118477047000070B590F83430044679
:1012500013B1002380F8343004F14402204601F039
:101260002DF963689B68B3B994F8443013F06005B6
:1012700035D00021204601F0CDFB0021204601F0B1
:10128000BFFB63681B6813B10621204698470623FD
:1012900084F8343070BD204698470028E4D0B4F874
:1012A0004A30E26B9A4288BFE36394F94430E56BBD
:1012B000002B4FF0300380F20381002D00F0F2800C
:1012C000092284F8342083F311880021D4E90E2305
:1012D0002046FFF771FF002383F31188DAE794F8C3
:1012E000452003F07F0343EA022340F20232934297
:1012F00000F0C58021D8B3F5807F48D00DD8012BF0
:101300003FD0022B00F09380002BB2D104F14C02AD
:10131000A2630222E2632364C1E7B3F5817F00F098
:101320009B80B3F5407FA4D194F84630012BA0D127
:10133000B4F84C3043F0020332E0B3F5006F4DD007
:1013400017D8B3F5A06F31D0A3F5C063012B90D8A7
:10135000636894F846205E6894F84710B4F8483003
:101360002046B047002884D04368A3630368E36342
:101370001AE0B3F5106F36D040F6024293427FF484
:1013800078AF5C4BA3630223E3630023C3E794F8C5
:101390004630012B7FF46DAFB4F84C3023F00203DC
:1013A000C4E90E55A4F84C30256478E7B4F844300D
:1013B000B3F5A06F0ED194F8463084F84E30204635
:1013C00000F0C2FF63681B6813B1012120469847F3
:1013D000032323700023C4E90E339CE704F14F0379
:1013E000A3630123C3E72378042B10D1302383F3B5
:1013F00011882046FFF7C4FE85F311880321636836
:1014000084F84F5021701B680BB12046984794F820
:101410004630002BDED084F84F30042323706368FD
:101420001B68002BD6D0022120469847D2E794F8BB
:1014300048301D0603F00F0120460AD501F030F8B0
:10144000012804D002287FF414AF2B4B9AE72B4BD2
:1014500098E701F017F8F3E794F84630002B7FF493
:1014600008AF94F8483013F00F01B3D01A062046A5
:1014700002D501F0E3FAADE701F0D6FAAAE794F855
:101480004630002B7FF4F5AE94F8483013F00F018E
:10149000A0D01B06204602D501F0BCFA9AE701F065
:1014A000AFFA97E7142284F8342083F311882B468F
:1014B0002A4629462046FFF76DFE85F31188E9E6A6
:1014C0005DB1152284F8342083F311880021D4E91A
:1014D0000E232046FFF75EFEFDE60B2284F8342043
:1014E00083F311882B462A4629462046FFF764FEDF
:1014F000E3E700BF30350008283500082C35000828
:1015000038B590F834300446002B3ED0063BDAB2B2
:101510000F2A34D80F2B32D8DFE803F037313108E7
:10152000223231313131313131313737C56BB0F899
:101530004A309D4214D2C3681B8AB5FBF3F203FB09
:1015400012556DB9302383F311882B462A4629465C
:10155000FFF732FE85F311880A2384F834300EE059
:10156000142384F83430302383F3118800231A467F
:1015700019462046FFF70EFE002383F3118838BD7D
:10158000036C03B198470023E7E70021204601F0F0
:1015900041FA0021204601F033FA63681B6813B159
:1015A0000621204698470623D7E7000010B590F89B
:1015B0003430142B044629D017D8062B05D001D877
:1015C0001BB110BD093B022BFBD80021204601F0C6
:1015D00021FA0021204601F013FA63681B6813B159
:1015E000062120469847062319E0152BE9D10B2345
:1015F00080F83430302383F3118800231A461946CB
:10160000FFF7DAFD002383F31188DAE7C3689B69EB
:101610005B68002BD5D1036C03B19847002384F895
:101620003430CEE700230375826803691B6899682C
:101630009142FBD25A680360426010605860704764
:1016400000230375826803691B6899689142FBD87F
:101650005A680360426010605860704708B50846D9
:10166000302383F311880B7D032B05D0042B0DD081
:101670002BB983F3118808BD8B6900221A604FF0E3
:10168000FF338361FFF7CEFF0023F2E7D1E9003299
:1016900013605A60F3E70000FFF7C4BF054BD96839
:1016A0000875186802681A60536001220275D860D4
:1016B000FEF728BE9823002030B50C4BDD684B1C8C
:1016C00087B004460FD02B46094A684600F074F9EB
:1016D0002046FFF7E3FF009B13B1684600F076F960
:1016E000A86907B030BDFFF7D9FFF9E798230020BC
:1016F0005D160008044B1A68DB6890689B68984286
:1017000094BF00200120704798230020084B10B59B
:101710001C68D86822681A60536001222275DC6058
:10172000FFF78EFF01462046BDE81040FEF7EABDF8
:1017300098230020044B1A68DB6892689B689A42E1
:1017400001D9FFF7E3BF70479823002038B5074C55
:1017500007490848012300252370656001F072FBEA
:101760000223237085F3118838BD00BF00260020B6
:10177000383500089823002000F05EB9EFF311809F
:1017800020B9EFF30583302282F3118870470000FF
:1017900010B530B9EFF30584C4F3080414B180F335
:1017A000118810BDFFF7C6FF84F31188F9E7000028
:1017B000034A516853685B1A9842FBD8704700BFD0
:1017C000001000E08B60022308618B82084670479E
:1017D0008368A3F1840243F8142C026943F8442C73
:1017E000426943F8402C094A43F8242CC26843F864
:1017F000182C022203F80C2C002203F80B2C044AAC
:1018000043F8102CA3F12000704700BF1D0300080F
:101810009823002008B5FFF7DBFFBDE80840FFF77D
:101820003BBF0000024BDB6898610F20FFF736BF1B
:1018300098230020302383F31188FFF7F3BF0000C3
:1018400008B50146302383F311880820FFF734FFE1
:10185000002383F3118808BD064BDB6839B1426869
:1018600018605A60136043600420FFF725BF4FF0F3
:10187000FF307047982300200368984206D01A680A
:101880000260506099611846FFF706BF704700007C
:1018900038B504460D462068844200D138BD03683F
:1018A00023605C608561FFF7F7FEF4E710B503681D
:1018B0009C68A2420CD85C688A600B604C60216016
:1018C000596099688A1A9A604FF0FF33836010BD9F
:1018D0001B68121BECE700000A2938BF0A2170B50B
:1018E00004460D460A26601901F0A6FA01F092FAA4
:1018F000041BA54203D8751C2E460446F3E70A2EA6
:1019000004D9BDE87040012001F0DCBA70BD0000D0
:10191000F8B5144B0D46D96103F1100141600A2A54
:101920001969826038BF0A22016048601861A818EE
:10193000144601F073FA0A2701F06CFA431BA34224
:10194000064606D37C1C281901F076FA2746354650
:10195000F2E70A2F04D9BDE8F840012001F0B2BA3D
:10196000F8BD00BF98230020F8B506460D4601F0EB
:1019700051FA0F4A134653F8107F9F4206D12A4668
:1019800001463046BDE8F840FFF7C2BFD169BB68E9
:10199000441A2C1928BF2C46A34202D92946FFF726
:1019A0009BFF224631460348BDE8F840FFF77EBF63
:1019B00098230020A823002010B4C0E903230023AB
:1019C0005DF8044B4361FFF7CFBF000010B5194C21
:1019D000236998420DD0D0E90032816813605A60C3
:1019E0009A680A449A60002303604FF0FF33A361B2
:1019F00010BD2346026843F8102F53600022026096
:101A000022699A4203D1BDE8104001F00FBA9368F1
:101A100081680B44936001F0FDF92269E1699268E5
:101A2000441AA242E4D91144BDE81040091AFFF754
:101A300053BF00BF982300202DE9F047DFF8BC809A
:101A400008F110072C4ED8F8105001F0E3F9D8F83F
:101A50001C40AA68031B9A423ED81444D5E90032C0
:101A60004FF00009C8F81C4013605A60C5F8009098
:101A7000D8F81030B34201D101F0D8F989F31188B8
:101A8000D5E9033128469847302383F311886B69E1
:101A9000002BD8D001F0BEF96A69A0EB04094A45D1
:101AA00082460DD2022001F00DFA0022D8F8103043
:101AB000B34208D151462846BDE8F047FFF728BF9A
:101AC000121A2244F2E712EB090938BF4A462946A6
:101AD0003846FFF7EBFEB5E7D8F81030B34208D030
:101AE0001444211AC8F81C00A960BDE8F047FFF7AC
:101AF000F3BEBDE8F08700BFA82300209823002094
:101B000000207047FEE70000704700004FF0FF30F4
:101B10007047000002290CD0032904D0012907488E
:101B200018BF00207047032A05D8054800EBC20003
:101B30007047044870470020704700BF1036000807
:101B400020220020C435000870B59AB0054608462A
:101B500001A9144600F0C2F801A8FFF799F8431C48
:101B60005B00C5E900340022237003236370C6B212
:101B700001AB02341046D1B28E4204F1020401D806
:101B80001AB070BD13F8011B04F8021C04F8010C14
:101B90000132F0E708B5302383F311880348FFF7DB
:101BA00033FA002383F3118808BD00BF0826002004
:101BB00090F8443003F01F02012A07D190F8452025
:101BC0000B2A03D10023C0E90E3315E003F06003B4
:101BD000202B08D1B0F848302BB990F84520212AA5
:101BE00003D81F2A04D8FFF7F1B9222AEBD0FAE76D
:101BF000034A82630722C26303640120704700BF67
:101C00001822002007B5052917D8DFE801F01916BA
:101C100003191920302383F31188104A0190012100
:101C2000FFF794FA01980E4A0221FFF78FFA0D4848
:101C3000FFF7B6F9002383F3118803B05DF804FBC6
:101C4000302383F311880748FFF780F9F2E7302348
:101C500083F311880348FFF797F9EBE76435000831
:101C6000883500080826002038B50C4D0C4C0D496D
:101C70002A4604F10800FFF767FF05F1CA0204F1E4
:101C800010000949FFF760FF05F5CA7204F118005A
:101C90000649BDE83840FFF757BF00BFD02A0020F3
:101CA00020220020443500084E3500085935000830
:101CB00070B5044608460D46FEF7EAFFC6B2204658
:101CC000013403780BB9184670BD32462946FEF739
:101CD000CBFF0028F3D10120F6E700002DE9F04703
:101CE00005460C46FEF7D4FF2B49C6B22846FFF73F
:101CF000DFFF08B10636F6B228492846FFF7D8FFBD
:101D000008B11036F6B2632E0BD8DFF88C80DFF8FE
:101D10008C90234FDFF894A02E7846B92670BDE84A
:101D2000F08729462046BDE8F04701F0B1BB252EDB
:101D30002ED1072241462846FEF796FF70B9194B6F
:101D4000224603F10C0153F8040B42F8040B8B42BA
:101D5000F9D11B78137007350D34DDE708224946A9
:101D60002846FEF781FF98B90F4BA21C1978090984
:101D70000232C95D02F8041C13F8011B01F00F01C7
:101D80005345C95D02F8031CF0D118340835C3E788
:101D900004F8016B0135BFE73036000859350008FB
:101DA0004636000838360008107AFF1F1C7AFF1FDD
:101DB000BFF34F8F024AD368DB03FCD4704700BFE8
:101DC000003C024008B5094B1B7873B9FFF7F0FFE0
:101DD000074B1A69002ABFBF064A5A6002F18832CF
:101DE0005A601A6822F480621A6008BD2E2D002005
:101DF000003C02402301674508B50B4B1B7893B9A3
:101E0000FFF7D6FF094B1A6942F000421A611A68BF
:101E100042F480521A601A6822F480521A601A68DA
:101E200042F480621A6008BD2E2D0020003C024062
:101E30000B28F0B516D80C4C0C4923787BB90C4D07
:101E40000E460C234FF0006255F8047B46F8042B35
:101E5000013B13F0FF033A44F6D10123237051F8FC
:101E60002000F0BD0020FCE7602D0020302D002078
:101E700058360008014B53F82000704758360008C8
:101E80000C2070470B2810B5044601D9002010BD66
:101E9000FFF7CEFF064B53F824301844C21A0BB993
:101EA0000120F4E712680132F0D1043BF6E700BFED
:101EB000583600080B2838B5044628D8FFF75EFCD2
:101EC000FFF776FFFFF77EFF124AF323D360E300AC
:101ED000DBB243F4007343F002031361136943F46C
:101EE0008033136105462046FFF762FFFFF7A0FF2E
:101EF000094B53F8241000F0E9F82846FFF77CFF5F
:101F0000FFF746FC2046BDE83840FFF7BBBF002086
:101F100038BD00BF003C02405836000812F00103F3
:101F20002DE9F04105460E4614464BD18218B2F118
:101F3000016F61D8314B1B6813F001035CD0304F47
:101F4000FFF71CFCFFF73EFFF323FB60FFF730FFBA
:101F5000314640F20128032C18D824F00104284E01
:101F60000C446D1A40F20118A142336905EB0107D8
:101F70002AD123F001033361FFF73EFFFFF708FC8E
:101F80000120BDE8F081043C0435E4E7AB07E4D16F
:101F90003B6923F440733B613B6943EA08033B61BF
:101FA00051F8046B2E60BFF34F8FFFF701FF2B68D2
:101FB0009E42E8D03B6923F001033B61FFF71CFF21
:101FC000FFF7E6FB0020DCE723F44073336133695D
:101FD00043EA080333610B883B80BFF34F8FFFF761
:101FE000E7FE3F8831F8023BBFB2BB42BCD0336949
:101FF00023F001033361E1E71846C2E700380240ED
:10200000003C0240084908B50B7828B11BB9FFF71E
:10201000D9FE01230B7008BD002BFCD0BDE80840A1
:102020000870FFF7E9BE00BF2E2D002010B5024456
:10203000064BD2B2904200D110BD441C00B253F8FE
:10204000200041F8040BE0B2F4E700BF5028004044
:102050000F4B30B51C6F240407D41C6F44F400747C
:102060001C671C6F44F400441C670A4C236843F44B
:10207000807323600244084BD2B2904200D130BD3D
:10208000441C00B251F8045B43F82050E0B2F4E77E
:1020900000380240007000405028004007B501227F
:1020A00001A90020FFF7C2FF019803B05DF804FB0F
:1020B00013B50446FFF7F2FFA04205D0012201A9A3
:1020C00000200194FFF7C4FF02B010BD704700006C
:1020D000034B1A681AB9034AD2F874281A60704779
:1020E000642D00200030024008B5FFF7F1FF024BDD
:1020F0001868C0F3407008BD642D002070470000D0
:10210000FEE700000A4B0B480B4A90420BD30B4BE7
:10211000DA1C121AC11E22F003028B4238BF0022C1
:102120000021FEF7BDBD53F8041B40F8041BECE78B
:1021300000380008602E0020602E0020602E002055
:1021400070B5D0E915439E6800224FF0FF3504EBCF
:1021500042135101D3F800090028BEBFD3F800098B
:1021600040F08040C3F80009D3F8000B0028BEBF40
:10217000D3F8000B40F08040C3F8000B0132631825
:102180009642C3F80859C3F8085BE0D24FF0011338
:10219000C4F81C3870BD0000890141F020010161C4
:1021A00003699B06FCD41220FFF702BB10B5054C57
:1021B0002046FEF7ABFF4FF0A0436365024BA365DB
:1021C00010BD00BF682D0020AC36000870B5037844
:1021D000012B054650D12A4B446D98421BD1294B07
:1021E0005A6B42F080025A635A6D42F080025A657F
:1021F0005A6D5A6942F080025A615A6922F080028F
:102200005A610E2143205B6900F022FC1E4BE36003
:102210001E4BC4F800380023C4F8003EC0232360DE
:102220006E6D4FF40413A3633369002BFCDA0123B2
:1022300033610C20FFF7BCFA3369DB07FCD41220B2
:10224000FFF7B6FA3369002BFCDA0026A6602846B1
:10225000FFF776FF6B68C4F81068DB68C4F8146891
:10226000C4F81C684BB90A4BA3614FF0FF3363619C
:10227000A36843F00103A36070BD064BF4E700BF01
:10228000682D002000380240401400400300200266
:10229000003C30C0083C30C0F8B5446D0546002114
:1022A0002046FFF779FFA96D00234FF001128F68D8
:1022B000C4F834384FF00066C4F81C284FF0FF30E3
:1022C00004EB431201339F42C2F80069C2F8006B6D
:1022D000C2F80809C2F8080BF2D20B686A6DEB6508
:1022E000636210231361166916F01006FBD11220E9
:1022F000FFF75EFAD4F8003823F4FE63C4F8003820
:10230000A36943F4402343F01003A3610923C4F8F5
:102310001038C4F814380A4BEB604FF0C043C4F8CF
:10232000103B084BC4F8003BC4F81069C4F80039EE
:10233000EB6D03F1100243F48013EA65A362F8BD6C
:102340008836000840800010426D90F84E10D2F898
:10235000003823F4FE6343EA0113C2F800387047E3
:102360002DE9F84300EB8103456DDA68166806F045
:102370000306731E022B05EB41130C4680460FFA31
:1023800081F94FEA41104FF00001C3F8101B4FF0E4
:10239000010104F1100398BFB60401FA03F3916937
:1023A0008EBF334E06F1805606F5004600293AD01E
:1023B000578A04F15801490137436F50D5F81C186A
:1023C0000B43C5F81C382B180021C3F810195369AA
:1023D0000127611EA7409BB3138A928B9B08012A99
:1023E00088BF5343D8F85C20981842EA034301F1B0
:1023F000400205EB8202C8F85C0021465360284683
:10240000FFF7CAFE08EB8900C3681B8A43EA8453BE
:10241000483464011E432E51D5F81C381F43C5F8BB
:102420001C78BDE8F88305EB4917D7F8001B21F4A9
:102430000041C7F8001BD5F81C1821EA0303C0E7C8
:1024400004F13F0305EB83030A4A5A6028462146FC
:10245000FFF7A2FE05EB4910D0F8003923F4004342
:10246000C0F80039D5F81C3823EA0707D7E700BFC2
:102470000080001000040002826D1268C265FFF740
:102480005FBE00005831436D49015B5813F40040B2
:1024900004D013F4001F0CBF02200120704700007D
:1024A0004831436D49015B5813F4004004D013F4E4
:1024B000001F0CBF022001207047000000EB8101CB
:1024C000CB68196A0B6813604B6853607047000053
:1024D00000EB810330B5DD68AA691368D36019B9D0
:1024E000402B84BF402313606B8A1468426D1C44E8
:1024F000013CB4FBF3F46343033323F0030302EB27
:10250000411043EAC44343F0C043C0F8103B2B687A
:1025100003F00303012B09B20ED1D2F8083802EB05
:10252000411013F4807FD0F8003B14BF43F0805378
:1025300043F00053C0F8003B02EB4112D2F8003BDD
:1025400043F00443C2F8003B30BD00002DE9F041E8
:10255000244D6E6D06EB40130446D3F8087BC3F898
:10256000087B38070AD5D6F81438190706D505EBC5
:1025700084032146DB6828465B689847FA071FD525
:10258000D6F81438DB071BD505EB8403D968CCB922
:102590008B69488A5A68B2FBF0F600FB16228AB9AA
:1025A0001868DA6890420DD2121AC3E90024302369
:1025B00083F311880B482146FFF78AFF84F31188C3
:1025C000BDE8F081012303FA04F26B8923EA0203D8
:1025D0006B81CB68002BF3D021460248BDE8F04167
:1025E000184700BF682D002000EB810370B5DD683F
:1025F000436D6C692668E6604A0156BB1A444FF485
:102600000020C2F810092A6802F00302012A0AB267
:102610000ED1D3F8080803EB421410F4807FD4F8ED
:10262000000914BF40F0805040F00050C4F8000989
:1026300003EB4212D2F8000940F00440C2F800094E
:10264000D3F83408012202FA01F10143C3F8341827
:1026500070BD19B9402E84BF4020206020682E8AAA
:102660008419013CB4FBF6F440EAC44040F0005049
:102670001A44C6E72DE9F8433B4D6E6D06EB401357
:102680000446D3F80889C3F8088918F0010F4FEA07
:1026900040171AD0D6F81038DB0716D505EB8003A3
:1026A000D9684B691868DA68904230D2121A4FF034
:1026B00000091A60C3F80490302383F3118821467F
:1026C0002846FFF791FF89F3118818F0800F1CD07E
:1026D000D6F834380126A640334216D005EB8403E1
:1026E0006D6DD3F80CC0DCF814200134E4B2D2F8DC
:1026F00000E005EB04342F445168714515D3D5F83B
:10270000343823EA0606C5F83468BDE8F8830123A7
:1027100003FA04F22B8923EA02032B818B68002B36
:10272000D3D0214628469847CFE7BCF81000AEEB3F
:102730000103834228BF0346D7F8180980B2B3EBE0
:10274000800FE2D89068A0F1040959F8048FC4F80A
:102750000080A0EB09089844B8F1040FF5D818449C
:102760000B4490605360C7E7682D00202DE9F74FB8
:10277000A24C656D6E69AB691E4016F480586E619F
:1027800007D02046FEF72AFD03B0BDE8F04F00F069
:1027900047BC002E12DAD5F8003E98489B071EBFB2
:1027A000D5F8003E23F00303C5F8003ED5F8043801
:1027B00023F00103C5F80438FEF73AFD370505D5C7
:1027C0008E48FFF7BDFC8D48FEF720FDB0040CD508
:1027D000D5F8083813F0060FEB6823F470530CBFDC
:1027E00043F4105343F4A053EB6031071BD56368E7
:1027F000DB681BB9AB6923F00803AB612378052BB9
:102800000CD1D5F8003E7D489A071EBFD5F8003E92
:1028100023F00303C5F8003EFEF70AFD6368DB689A
:102820000BB176489847F30274D4B70227D5D4F891
:102830005490DFF8C8B100274FF0010A09EB4712A6
:10284000D2F8003B03F44023B3F5802F11D1D2F826
:10285000003B002B0DDA62890AFA07F322EA030330
:10286000638104EB8703DB68DB6813B139465846A4
:102870009847A36D01379B68FFB29F42DED9F006EF
:1028800017D5676D3A6AC2F30A1002F00F0302F41B
:10289000F012B2F5802F00F08580B2F5402F08D1FC
:1028A00004EB83030022DB681B6A07F58057904224
:1028B0006AD13003D5F8184813D5E10302D50020BA
:1028C000FFF744FEA20302D50120FFF73FFE63039A
:1028D00002D50220FFF73AFE270302D50320FFF7B7
:1028E00035FE75037FF550AFE00702D50020FFF7F6
:1028F000C1FEA10702D50120FFF7BCFE620702D589
:102900000220FFF7B7FE23077FF53EAF0320FFF756
:10291000B1FE39E7636DDFF8E4A0019300274FF0C3
:102920000109A36D9B685FFA87FB9B453FF67DAF6E
:10293000019B03EB4B13D3F8001901F44021B1F5CF
:10294000802F1FD1D3F8001900291BDAD3F8001902
:1029500041F09041C3F80019D3F800190029FBDBBE
:102960005946606DFFF718FC218909FA0BF321EA3B
:102970000303238104EB8B03DB689B6813B1594687
:10298000504698470137CCE7910708BFD7F8008039
:10299000072A98BF03F8018B02F1010298BF4FEAA2
:1029A000182884E7023304EB830207F58057526846
:1029B000D2F818C0DCF80820DCE9001CA1EB0C0CF4
:1029C000002188420AD104EB830463689B699A68FA
:1029D00002449A605A6802445A606AE711F0030F91
:1029E00008BFD7F800808C4588BF02F8018B01F141
:1029F000010188BF4FEA1828E3E700BF682D0020D7
:102A0000436D03EB4111D1F8003B43F40013C1F8CF
:102A1000003B7047436D03EB4111D1F8003943F49B
:102A20000013C1F800397047436D03EB4111D1F831
:102A3000003B23F40013C1F8003B7047436D03EBE8
:102A40004111D1F8003923F40013C1F8003970475F
:102A500000F1604303F561430901C9B283F8001333
:102A6000012200F01F039A4043099B0003F16043D9
:102A700003F56143C3F880211A60704730B5039CA9
:102A80000172043304FB0325C0E90653049B03636E
:102A90000021059BC160C0E90000C0E90422C0E933
:102AA0000842C0E90A11436330BD0000416A0022B8
:102AB000C0E90411C0E90A22C2606FF00101FEF70B
:102AC000E7BE0000D0E90432934201D1C2680AB9DE
:102AD000181D70470020704703691960C2680132F1
:102AE000C260C269134482690361934224BF436A8E
:102AF00003610021FEF7C0BE38B504460D46E36809
:102B00003BB16269131D1268A3621344E3620020A3
:102B100007E0237A33B929462046FEF79DFE0028B8
:102B2000EDDA38BD6FF00100FBE70000C368C26951
:102B3000013BC3604369134482694361934224BFEC
:102B4000436A436100238362036B03B118477047F4
:102B500070B53023044683F31188866A3EB9FFF7C7
:102B6000CBFF054618B186F31188284670BDA36ACD
:102B7000E26A13F8015BA362934202D32046FFF797
:102B8000D5FF002383F31188EFE700002DE9F84F0C
:102B900004460E46174698464FF0300989F31188CF
:102BA0000025AA46D4F828B0BBF1000F09D1414650
:102BB0002046FFF7A1FF20B18BF311882846BDE81E
:102BC000F88FD4E90A12A7EB050B521A934528BFD8
:102BD0009346BBF1400F1BD9334601F1400251F837
:102BE000040B43F8040B9142F9D1A36A40334036F9
:102BF000A3624035D4E90A239A4202D32046FFF764
:102C000095FF8AF31188BD42D8D289F31188C9E7AC
:102C100030465A46FEF71EF8A36A5B445E44A36240
:102C20005D44E7E710B5029C0172043303FB042105
:102C3000C0E906130023C0E90A33039B0363049B26
:102C4000C460C0E90000C0E90422C0E9084243634F
:102C500010BD0000026AC260426AC0E9042200227C
:102C6000C0E90A226FF00101FEF712BED0E9042389
:102C70009A4201D1C26822B9184650F8043B0B6051
:102C8000704700231846FAE7C368C2690133C3607E
:102C90004369134482694361934224BF436A436199
:102CA0000021FEF7E9BD000038B504460D46E36893
:102CB0003BB123691A1DA262E2691344E36200205A
:102CC00007E0237A33B929462046FEF7C5FD0028E0
:102CD000EDDA38BD6FF00100FBE700000369196011
:102CE000C268013AC260C2691344826903619342B7
:102CF00024BF436A036100238362036B03B1184757
:102D00007047000070B530230D460446114683F32A
:102D10001188866A2EB9FFF7C7FF10B186F31188B4
:102D200070BDA36A1D70A36AE26A01339342A36275
:102D300004D3E16920460439FFF7D0FF002080F377
:102D40001188EDE72DE9F84F04460D469046994667
:102D50004FF0300A8AF311880026B346A76A4FB9AC
:102D600049462046FFF7A0FF20B187F3118830467F
:102D7000BDE8F88FD4E90A073A1AA8EB060797428C
:102D800028BF1746402F1BD905F1400355F8042BE7
:102D900040F8042B9D42F9D1A36A4033A362403628
:102DA000D4E90A239A4204D3E16920460439FFF7A3
:102DB00095FF8BF311884645D9D28AF31188CDE768
:102DC00029463A46FDF746FFA36A3B443D44A362C9
:102DD0003E44E5E7D0E904239A4217D1C3689BB18A
:102DE000836A8BB1043B9B1A0ED01360C368013B0E
:102DF000C360C3691A44836902619A4224BF436A6B
:102E00000361002383620123184670470023FBE718
:102E100000F030B94FF08043586A70474FF080435C
:102E2000002258631A610222DA6070474FF0804333
:102E30000022DA60704700004FF08043586370470B
:102E4000FEE7000070B51B4B01630025044686B009
:102E5000586085620E4600F0BFF804F11003C4E923
:102E600004334FF0FF33C4E90635C4E90044A560DC
:102E7000E562FFF7CFFF2B460246C4E9082304F1C1
:102E800034010D4A256580232046FEF79BFC012373
:102E9000E0600A4A0375009272680192B268CDE957
:102EA0000223074B6846CDE90435FEF7B3FC06B0B4
:102EB00070BD00BF00260020B8360008BD360008EF
:102EC000412E0008024AD36A1843D062704700BFFF
:102ED000982300204B6843608B688360CB68C36095
:102EE0000B6943614B6903628B6943620B68036042
:102EF0007047000008B5264B26481A6940F2FF11BA
:102F00000A431A611A6922F4FF7222F001021A615F
:102F10001A691A6B0A431A631A6D0A431A651E4A24
:102F20001B6D1146FFF7D6FF02F11C0100F5806012
:102F3000FFF7D0FF02F1380100F58060FFF7CAFF0C
:102F400002F1540100F58060FFF7C4FF02F1700147
:102F500000F58060FFF7BEFF02F18C0100F5806094
:102F6000FFF7B8FF02F1A80100F58060FFF7B2FF9C
:102F700002F1C40100F58060FFF7ACFF02F1E0014F
:102F800000F58060FFF7A6FFBDE8084000F0EEB84E
:102F90000038024000000240C436000808B500F0C6
:102FA00059FAFEF7D3FBFFF793F8BDE80840FEF7A8
:102FB0005BBE000070470000EFF3098305494A6BD0
:102FC00022F001024A63683383F30988002383F304
:102FD0001188704700EF00E0302080F3118862B65E
:102FE0000C4B0D4AD96821F4E0610904090C0A432D
:102FF000DA60D3F8FC20094942F08072C3F8FC2063
:103000000A6842F001020A602022DA7783F822007F
:10301000704700BF00ED00E00003FA05001000E07B
:1030200010B5302383F311880E4B5B6813F40063F3
:1030300014D0F1EE103AEFF30984683C4FF080733E
:10304000E361094BDB6B236684F30988FEF752FBCF
:1030500010B1064BA36110BD054BFBE783F311884C
:10306000F9E700BF00ED00E000EF00E02F030008EB
:10307000320300080F4B1A6C42F001021A641A6EF8
:1030800042F001021A660C4A1B6E936843F001037A
:1030900093604FF0804353229A624FF0FF32DA621E
:1030A00000229A615A63DA605A6001225A611A60FA
:1030B000704700BF00380240002004E04FF080421B
:1030C00008B51169D3680B40D9B2C9439B07116198
:1030D00007D5302383F31188FEF74EFB002383F3DB
:1030E000118808BD1F4B1A696FEAC2526FEAD252AB
:1030F0001A611A69C2F308021A614FF0FF301A69A7
:103100005A69586100215A6959615A691A6A62F00C
:1031100080521A621A6A02F080521A621A6A5A6A55
:1031200058625A6A59625A6A1A6C42F080521A649A
:103130001A6E42F080521A661A6E0B4A106840F4FA
:1031400080701060186F00F44070B0F5007F1EBFF3
:103150004FF4803018671967536823F40073536085
:1031600000F054B90038024000700040334B4FF07B
:1031700080521A64324A4FF4404111601A6842F09A
:1031800001021A601A689107FCD59A6822F00302BE
:103190009A602A4B9A6812F00C02FBD1196801F070
:1031A000F90119609A601A6842F480321A601A684C
:1031B0009203FCD55A6F42F001025A671F4B5A6FB7
:1031C0009007FCD51F4A5A601A6842F080721A6054
:1031D0001B4A53685904FCD5184B1A689201FCD558
:1031E000194A9A60194B1A68194B9A42194B21D106
:1031F000194A1168194A91421CD140F205121A600D
:10320000144A136803F00F03052BFAD10B4B9A688D
:1032100042F002029A609A6802F00C02082AFAD17F
:103220005A6C42F480425A645A6E42F480425A66A2
:103230005B6E704740F20572E1E700BF0038024064
:10324000007000400854400700948838002004E0D3
:1032500011640020003C024000ED00E041C20F413B
:10326000074A08B5536903F00103536123B1054AC6
:1032700013680BB150689847BDE80840FFF7D0BE0F
:10328000003C0140E02D0020074A08B5536903F0D7
:103290000203536123B1054A93680BB1D068984784
:1032A000BDE80840FFF7BCBE003C0140E02D002017
:1032B000074A08B5536903F00403536123B1054A73
:1032C00013690BB150699847BDE80840FFF7A8BEE5
:1032D000003C0140E02D0020074A08B5536903F087
:1032E0000803536123B1054A93690BB1D06998472C
:1032F000BDE80840FFF794BE003C0140E02D0020EF
:10330000074A08B5536903F01003536123B1054A16
:10331000136A0BB1506A9847BDE80840FFF780BEBA
:10332000003C0140E02D0020164B10B55C6904F410
:1033300078725A61A30604D5134A936A0BB1D06A16
:103340009847600604D5104A136B0BB1506B984731
:10335000210604D50C4A936B0BB1D06B9847E2055C
:1033600004D5094A136C0BB1506C9847A30504D5DA
:10337000054A936C0BB1D06C9847BDE81040FFF73D
:103380004FBE00BF003C0140E02D0020194B10B59E
:103390005C6904F47C425A61620504D5164A136DD7
:1033A0000BB1506D9847230504D5134A936D0BB1AB
:1033B000D06D9847E00404D50F4A136E0BB1506EE0
:1033C0009847A10404D50C4A936E0BB1D06E984770
:1033D000620404D5084A136F0BB1506F9847230459
:1033E00004D5054A936F0BB1D06F9847BDE81040E4
:1033F000FFF716BE003C0140E02D002008B5FFF7A6
:103400005DFEBDE80840FFF70BBE0000062108B5D1
:103410000846FFF71DFB06210720FFF719FB0621D1
:103420000820FFF715FB06210920FFF711FB0621F5
:103430000A20FFF70DFB06211720FFF709FB0621E5
:103440002820FFF705FBBDE8084007211C20FFF7F7
:10345000FFBA000008B5FFF745FE00F00BF8FDF7D6
:1034600053FEFDF72BFDFFF7A5FDBDE80840FFF774
:10347000CFBC00000023054A19460133102BC2E9D6
:10348000001102F10802F8D1704700BFE02D0020C2
:10349000034611F8012B03F8012B002AF9D17047DC
:1034A00053544D3332463F3F3F0053544D33324621
:1034B0003430780053544D3332463432780053540C
:1034C0004D33324634343658580000000120330062
:1034D0000010410001105A0003105900071031007C
:1034E00000000000A034000813040000AA34000803
:1034F00019040000B434000821040000BE340008A0
:1035000000000000390E0008250E0008610E0008BA
:103510004D0E0008590E0008450E0008310E000837
:103520001D0E00086D0E00080000000001000000E4
:10353000000000006330000034350008F023002054
:10354000002600204172647550696C6F740025423A
:103550004F415244252D424C002553455249414C80
:1035600025000000020000000000000055100008C7
:10357000C110000840004000A02A0020B02A00200E
:103580000200000000000000030000000000000036
:10359000051100080000000010000000C02A0020F3
:1035A000000000000100000000000000682D002065
:1035B00001010200051C0008151B0008B11B0008D2
:1035C000951B000843000000CC35000809024300A9
:1035D000020100C0320904000001020201000524BA
:1035E0000010010524010001042402020524060044
:1035F00001070582030800FF09040100020A000018
:10360000000705010240000007058102400000009C
:1036100012000000183600081201100102000040DC
:1036200009124157000201020301000004030904CA
:1036300025424F4152442500466C79776F6F4634DE
:10364000303550726F0030313233343536373839D7
:103650004142434445460000004000000040000055
:1036600000400000004000000000010000000200D7
:103670000000020000000200000002000000020042
:1036800000000200000002000000000049120008D3
:1036900001150008AD15000840004000C82D0020AD
:1036A000C82D002001000000D82D0020800000005F
:1036B00040010000030000006D61696E0069646CE8
:1036C000650000000000842A00000000AAAAAAAA3F
:1036D00000000024FFFD00000000000000A00A0020
:1036E0004000001100000000AAAAAAAA4000001190
:1036F000FFFF0000000000000000000000000000CC
:1037000000000000AAAAAAAA00000000FFFF000013
:1037100000000000000000000000000000000000A9
:10372000AAAAAAAA00000000FFFF000000000000F3
:10373000000000000000000000000000AAAAAAAAE1
:1037400000000000FFFF000000000000000000007B
:103750000000000000000000AAAAAAAA00000000C1
:10376000FFFF00000000000000000000000000005B
:1037700000000000AAAAAAAA00000000FFFF0000A3
:103780000000000000000000000000000000000039
:103790000A0000000000000003000000000000001C
:1037A0000000000000000000000000000000000019
:1037B0000000000000000000000000000000000009
:1037C000710400000000000000400F000000000035
:1037D000FF009600000000080096000000000800AE
:1037E000040000002C36000800000000000000006B
:1037F00000000000000000000000000000000000C9
:10380000FFFFFFFFFFFFFFFFFFFFFFFFFFFFFFFFC8
:10381000FFFFFFFFFFFFFFFFFFFFFFFFFFFFFFFFB8
:10382000FFFFFFFFFFFFFFFFFFFFFFFFFFFFFFFFA8
:10C000000006002089D20008518D0608AD8C060874
:10C01000198D0608AD8C0608E58C06088BD2000841
:10C020008BD200088BD200088BD200084563080829
:10C030008BD200088BD200088BD200088BD200086C
:10C040008BD200088BD200088BD200088BD200085C
:10C050008BD200088BD20008DD6E0808056F080837
:10C060002D6F0808556F08087D6F0808DD1C08084B
:10C07000051D0808311D08085D1D0808891D0808F0
:10C08000B11D0808DD1D0808611C08088BD20008D6
:10C090008BD200088BD200088BD20008A56F08084D
:10C0A000F1700808F5700808097108080D71080892
:10C0B00011710808257108083971080869230808F2
:10C0C000112508088BD200088BD200088BD20008FB
:10C0D0008BD20008797008088D700808A1700808D4
:10C0E000097008088BD200088BD200085D7108081F
:10C0F000617108087571080879710808091E080837
:10C100008BD200088BD20008497108088BD2000836
:10C11000B5700808C97008088BD200088BD20008D7
:10C12000351E08085D1E0808891E0808B51E080887
:10C13000E11E08088BD200088BD200088BD20008C1
:10C140008BD200088BD200088BD20008716A0808D5
:10C15000091F0808351F0808611F0808DD70080856
:10C160008BD200088BD200088BD200088BD200083B
:10C170008BD200088BD200088BD200088BD200082B
:10C180008BD200088BD200088BD200088BD200081B
:10C190008BD200088BD200088BD200088BD200080B
:10C1A0008BD200088BD200088BD200088BD20008FB
:10C1B0008BD200088BD200088BD200088BD20008EB
:10C1C0008BD200088BD200088BD200088BD20008DB
:10C1D0008BD200088BD200088BD200088BD20008CB
:10C1E00079E500083D6D010891C60208794D040803
:10C1F000FD690408DDBA040821C4040869C70408FD
:10C20000C52F0508C5340508854C0508A9C80508CB
:10C2100011860608711207086998070875BF070894
:10C22000BDD50708310508085D0B0808FFFFFFFFB3
:10C2300081F0004102E000BF83F0004330B54FEAD7
:10C2400041044FEA430594EA050F08BF90EA020F44
:10C250001FBF54EA000C55EA020C7FEA645C7FEAD7
:10C26000655C00F0E2804FEA5454D4EB5555B8BFFA
:10C270006D420CDD2C4480EA020281EA030382EA6B
:10C28000000083EA010180EA020281EA0303362DFD
:10C2900088BF30BD11F0004F4FEA01314FF4801CD0
:10C2A0004CEA113102D0404261EB410113F0004FE2
:10C2B0004FEA03334CEA133302D0524263EB430399
:10C2C00094EA050F00F0A780A4F10104D5F1200E37
:10C2D0000DDB02FA0EFC22FA05F2801841F1000192
:10C2E00003FA0EF2801843FA05F359410EE0A5F166
:10C2F00020050EF1200E012A03FA0EFC28BF4CF097
:10C30000020C43FA05F3C01851EBE37101F000454C
:10C3100007D54FF0000EDCF1000C7EEB00006EEB59
:10C320000101B1F5801F1BD3B1F5001F0CD34908E3
:10C330005FEA30004FEA3C0C04F101044FEA44523A
:10C3400012F5800F80F09A80BCF1004F08BF5FEAC1
:10C35000500C50F1000041EB045141EA050130BDA1
:10C360005FEA4C0C404141EB0101013C28BFB1F5B3
:10C37000801FE9D291F0000F04BF01460020B1FAFE
:10C3800081F308BF2033A3F10B03B3F120020CDAD1
:10C390000C3208DD02F1140CC2F10C0201FA0CF0AF
:10C3A00021FA02F10CE002F11402D8BFC2F1200C14
:10C3B00001FA02F120FA0CFCDCBF41EA0C019040CA
:10C3C000E41AA2BF01EB0451294330BD6FEA040413
:10C3D0001F3C1CDA0C340EDC04F11404C4F12002FE
:10C3E00020FA04F001FA02F340EA030021FA04F310
:10C3F00045EA030130BDC4F10C04C4F1200220FA67
:10C4000002F001FA04F340EA0300294630BD21FAA4
:10C4100004F0294630BD94F0000F83F4801306BF6A
:10C4200081F480110134013D4EE77FEA645C18BF5E
:10C430007FEA655C29D094EA050F08BF90EA020FF5
:10C4400005D054EA000C04BF1946104630BD91EAED
:10C45000030F1EBF0021002030BD5FEA545C05D1F0
:10C460004000494128BF41F0004130BD14F580042F
:10C470003CBF01F5801130BD01F0004545F0FE41A3
:10C4800041F470014FF0000030BD7FEA645C1ABFD8
:10C49000194610467FEA655C1CBF0B46024650EA0F
:10C4A000013406BF52EA033591EA030F41F400213B
:10C4B00030BD00BF90F0000F04BF0021704730B5C1
:10C4C0004FF4806404F132044FF000054FF0000196
:10C4D00050E700BF90F0000F04BF0021704730B557
:10C4E0004FF4806404F1320410F0004548BF40422C
:10C4F0004FF000013EE700BF42004FEAE2014FEA81
:10C5000031014FEA02701FBF12F07F4393F07F4F5B
:10C5100081F06051704732F07F4208BF704793F05E
:10C520007F4F04BF41F40021704730B54FF4607471
:10C5300001F0004521F000411CE700BF50EA010274
:10C5400008BF704730B54FF000050AE050EA01021D
:10C5500008BF704730B511F0004502D5404261EB8D
:10C5600041014FF4806404F132045FEA915C3FF4CE
:10C57000D8AE4FF003025FEADC0C18BF03325FEA6B
:10C58000DC0C18BF033202EBDC02C2F1200300FA1C
:10C5900003FC20FA02F001FA03FE40EA0E0021FA41
:10C5A00002F11444BDE600BF70B54FF0FF0C4CF42F
:10C5B000E06C1CEA11541DBF1CEA135594EA0C0FE1
:10C5C00095EA0C0F00F0DEF82C4481EA030621EA1C
:10C5D0004C5123EA4C5350EA013518BF52EA033557
:10C5E00041F4801143F4801338D0A0FB02CE4FF009
:10C5F0000005E1FB02E506F00042E0FB03E54FF039
:10C600000006E1FB03569CF0000F18BF4EF0010E30
:10C61000A4F1FF04B6F5007F64F5407404D25FEA2C
:10C620004E0E6D4146EB060642EAC62141EA5551DF
:10C630004FEAC52040EA5E504FEACE2EB4F1FD0C21
:10C6400088BFBCF5E06F1ED8BEF1004F08BF5FEA9F
:10C65000500E50F1000041EB045170BD06F0004651
:10C6600046EA010140EA020081EA0301B4EB5C04FE
:10C67000C2BFD4EB0C0541EA045170BD41F48011F6
:10C680004FF0000E013C00F3AB8014F1360FDEBF1B
:10C69000002001F0004170BDC4F10004203C35DAF7
:10C6A0000C341BDC04F11404C4F1200500FA05F37A
:10C6B00020FA04F001FA05F240EA020001F000421B
:10C6C00021F0004110EBD37021FA04F642EB060191
:10C6D0005EEA430E08BF20EAD37070BDC4F10C04BB
:10C6E000C4F1200500FA04F320FA05F001FA04F27F
:10C6F00040EA020001F0004110EBD37041F100016B
:10C700005EEA430E08BF20EAD37070BDC4F1200575
:10C7100000FA05F24EEA020E20FA04F301FA05F2DD
:10C7200043EA020321FA04F001F0004121FA04F285
:10C7300020EA020000EBD3705EEA430E08BF20EA55
:10C74000D37070BD94F0000F0FD101F0004640008F
:10C7500041EB010111F4801F08BF013CF7D041EA11
:10C76000060195F0000F18BF704703F00046520015
:10C7700043EB030313F4801F08BF013DF7D043EAE6
:10C780000603704794EA0C0F0CEA135518BF95EA9C
:10C790000C0F0CD050EA410618BF52EA4306D1D123
:10C7A00081EA030101F000414FF0000070BD50EA42
:10C7B000410606BF1046194652EA430619D094EACC
:10C7C0000C0F02D150EA013613D195EA0C0F05D1B6
:10C7D00052EA03361CBF104619460AD181EA03010A
:10C7E00001F0004141F0FE4141F470014FF00000C2
:10C7F00070BD41F0FE4141F4780170BD70B54FF05D
:10C80000FF0C4CF4E06C1CEA11541DBF1CEA1355DC
:10C8100094EA0C0F95EA0C0F00F0A7F8A4EB0504BE
:10C8200081EA030E52EA03354FEA013100F08880B5
:10C830004FEA03334FF0805545EA131343EA12637E
:10C840004FEA022245EA111545EA10654FEA002633
:10C850000EF000419D4208BF964244F1FD0404F5EC
:10C86000407402D25B084FEA3202B61A65EB030548
:10C870005B084FEA32024FF480104FF4002CB6EB05
:10C88000020E75EB030E22BFB61A754640EA0C0085
:10C890005B084FEA3202B6EB020E75EB030E22BFC5
:10C8A000B61A754640EA5C005B084FEA3202B6EB06
:10C8B000020E75EB030E22BFB61A754640EA9C00C5
:10C8C0005B084FEA3202B6EB020E75EB030E22BF95
:10C8D000B61A754640EADC0055EA060E18D04FEA53
:10C8E000051545EA16754FEA06164FEAC30343EAF3
:10C8F00052734FEAC2025FEA1C1CC0D111F4801FC0
:10C900000BD141EA00014FF000004FF0004CB6E7B8
:10C9100011F4801F04BF01430020B4F1FD0C88BF57
:10C92000BCF5E06F3FF6AFAEB5EB030C04BFB6EB62
:10C93000020C5FEA500C50F1000041EB045170BD55
:10C940000EF0004E4EEA113114EB5C04C2BFD4EB82
:10C950000C0541EA045170BD41F480114FF0000E06
:10C96000013C90E645EA060E8DE60CEA135594EA82
:10C970000C0F08BF95EA0C0F3FF43BAF94EA0C0F85
:10C980000AD150EA01347FF434AF95EA0C0F7FF4FA
:10C9900025AF104619462CE795EA0C0F06D152EA4E
:10C9A00003353FF4FDAE1046194622E750EA410632
:10C9B00018BF52EA43067FF4C5AE50EA41047FF443
:10C9C0000DAF52EA43057FF4EBAE12E74FF0FF3CA8
:10C9D00006E000BF4FF0010C02E000BF4FF0010C79
:10C9E0004DF804CD4FEA410C7FEA6C5C4FEA430CF2
:10C9F00018BF7FEA6C5C1BD001B050EA410C0CBF41
:10CA000052EA430C91EA030F02BF90EA020F0020A2
:10CA1000704710F1000F91EA030F58BF994208BF09
:10CA200090422CBFD8176FEAE37040F001007047C6
:10CA30004FEA410C7FEA6C5C02D150EA013C07D11D
:10CA40004FEA430C7FEA6C5CD6D152EA033CD3D068
:10CA50005DF8040B704700BF8446104662468C4662
:10CA60001946634600E000BF01B5FFF7B7FF002895
:10CA700048BF10F1000F01BD4DF808EDFFF7F4FFBE
:10CA80000CBF012000205DF808FB00BF4DF808ED49
:10CA9000FFF7EAFF34BF012000205DF808FB00BF6C
:10CAA0004DF808EDFFF7E0FF94BF012000205DF88E
:10CAB00008FB00BF4DF808EDFFF7CEFF94BF012043
:10CAC00000205DF808FB00BF4DF808EDFFF7C4FF3C
:10CAD00034BF012000205DF808FB00BF4FEA410C85
:10CAE0007FEA6C5C02D150EA013C0AD14FEA430C68
:10CAF0007FEA6C5C02D152EA033C02D14FF00000A5
:10CB000070474FF0010070474FEA410212F50012E2
:10CB100015D211D56FF47873B3EB625212D94FEA84
:10CB2000C12343F0004343EA505311F0004F23FA6E
:10CB300002F018BF404270474FF00000704750EAC3
:10CB4000013005D111F0004008BF6FF00040704780
:10CB50004FF00000704700BF4A0011D212F50012DA
:10CB600011D20DD56FF47873B3EB62520ED44FEA45
:10CB7000C12343F0004343EA505323FA02F07047C5
:10CB80004FF00000704750EA013002D14FF0FF3003
:10CB900070474FF0000070474FEA4102B2F1E043A6
:10CBA00024BFB3F5001CDCF1FE5C0DD901F0004C94
:10CBB0004FEAC0024CEA5070B2F1004F40EB8300E4
:10CBC00008BF20F00100704711F0804F21D113F110
:10CBD0003872BCBF01F00040704741F480114FEA49
:10CBE0005252C2F11802C2F1200C10FA0CF320FAD2
:10CBF00002F018BF40F001004FEAC1234FEAD323EF
:10CC000003FA0CFC40EA0C0023FA02F34FEA430358
:10CC1000CCE77FEA625307D150EA01331EBF4FF0E1
:10CC2000FE4040F44000704701F0004040F0FE40FC
:10CC300040F40000704700BF80F0004002E000BFF9
:10CC400081F0004142001FBF5FEA410392EA030FF7
:10CC50007FEA226C7FEA236C6AD04FEA1262D2EB41
:10CC60001363C1BFD218414048404140B8BF5B4246
:10CC7000192B88BF704710F0004F40F4000020F0DF
:10CC80007F4018BF404211F0004F41F4000121F0F5
:10CC90007F4118BF494292EA030F3FD0A2F101023F
:10CCA00041FA03FC10EB0C00C3F1200301FA03F17D
:10CCB00000F0004302D5494260EB4000B0F5000FA0
:10CCC00013D3B0F1807F06D340084FEA310102F15F
:10CCD0000102FE2A51D2B1F1004F40EBC25008BF11
:10CCE00020F0010040EA03007047490040EB0000DB
:10CCF000013A28BFB0F5000FEDD2B0FA80FCACF1DC
:10CD0000080CB2EB0C0200FA0CF0AABF00EBC25008
:10CD100052421843BCBFD0401843704792F0000FF6
:10CD200081F4000106BF80F400000132013BB5E749
:10CD30004FEA41037FEA226C18BF7FEA236C21D0BF
:10CD400092EA030F04D092F0000F08BF0846704724
:10CD500090EA010F1CBF0020704712F07F4F04D1F2
:10CD6000400028BF40F00040704712F100723CBF05
:10CD700000F50000704700F0004343F0FE4040F42F
:10CD8000000070477FEA226216BF08467FEA2363ED
:10CD90000146420206BF5FEA412390EA010F40F4D8
:10CDA000800070474FF0000304E000BF10F0004324
:10CDB00048BF40425FEA000C08BF704743F096430B
:10CDC00001464FF000001CE050EA010208BF704726
:10CDD0004FF000030AE000BF50EA010208BF7047AD
:10CDE00011F0004302D5404261EB41015FEA010CC2
:10CDF00002BF84460146002043F0B64308BFA3F1BA
:10CE00008053A3F50003BCFA8CF2083AA3EBC2539B
:10CE100010DB01FA02FC634400FA02FCC2F12002BA
:10CE2000BCF1004F20FA02F243EB020008BF20F0F1
:10CE30000100704702F1200201FA02FCC2F1200257
:10CE400050EA4C0021FA02F243EB020008BF20EA4C
:10CE5000DC7070477BB972B90029BEBF00204FF06B
:10CE6000004106E008BF00281CBF6FF000414FF0F2
:10CE7000FF3000F007BAADF1080C6DE904CE0029CF
:10CE800009DB002B1ADB00F095F8DDF804E0DDE9A2
:10CE9000022304B07047404261EB4101002B1BDBD1
:10CEA00000F088F8DDF804E0DDE9022304B0404238
:10CEB00061EB4101524263EB43037047524263EB23
:10CEC000430300F077F8DDF804E0DDE9022304B065
:10CED000404261EB41017047524263EB430300F073
:10CEE00069F8DDF804E0DDE9022304B0524263EBA7
:10CEF0004303704753B94AB9002908BF00281CBF33
:10CF00004FF0FF314FF0FF3000F0BCB9ADF1080C2D
:10CF10006DE904CE00F04EF8DDF804E0DDE902230F
:10CF200004B07047430803F05533C01A830803F078
:10CF3000333300F03330184400EB101000F00F30A2
:10CF400000EB002000EB0040000E704707EE900A57
:10CF5000F5EEC07AF1EE10FA01D400F00BB8F1EE64
:10CF6000677A08B517EE900A00F004F8404261EBCA
:10CF7000410108BDD0B5FFF7BFFA0C4B00220646B1
:10CF80000F46FFF711FBFFF7E7FD0446FFF792FAA4
:10CF9000074B0022FFF708FB02460B463046394696
:10CFA000FFF74AF9FFF7D8FD2146D0BD0000F03D5C
:10CFB0000000F0412DE9F047089D04468E46002B05
:10CFC0004DD18A42944669D9B2FA82F252B101FA3D
:10CFD00002F3C2F1200120FA01F10CFA02FC41EA4D
:10CFE000030E94404FEA1C48210CBEFBF8F61FFAD2
:10CFF0008CF708FB16E341EA034306FB07F199426D
:10D000000AD91CEB030306F1FF3080F01F8199421F
:10D0100040F21C81023E63445B1AA4B2B3FBF8F0F9
:10D0200008FB103344EA034400FB07F7A7420AD980
:10D030001CEB040400F1FF3380F00A81A74240F2A8
:10D0400007816444023840EA0640E41B00261DB113
:10D05000D4400023C5E900433146BDE8F0878B4248
:10D0600009D9002D00F0EF800026C5E90001304607
:10D070003146BDE8F087B3FA83F6002E4AD18B42E1
:10D0800002D3824200F2F980841A61EB030301208B
:10D090009E46002DE0D0C5E9004EDDE702B9FFDE77
:10D0A000B2FA82F2002A40F09280A1EB0C014FEA22
:10D0B0001C471FFA8CFE0126200CB1FBF7F307FB7F
:10D0C000131140EA01410EFB03F0884208D91CEB22
:10D0D000010103F1FF3802D2884200F2CB804346BF
:10D0E000091AA4B2B1FBF7F007FB101144EA01449E
:10D0F0000EFB00FEA64508D91CEB040400F1FF312D
:10D1000002D2A64500F2BB800846A4EB0E0440EA1A
:10D1100003409CE7C6F12007B34022FA07FC4CEA23
:10D12000030C20FA07F401FA06F31C43F9404FEA16
:10D130001C4900FA06F3B1FBF9F8200C1FFA8CFE2B
:10D1400009FB181140EA014108FB0EF0884202FA7F
:10D1500006F20BD91CEB010108F1FF3A80F0888040
:10D16000884240F28580A8F102086144091AA4B2FD
:10D17000B1FBF9F009FB101144EA014100FB0EFE7E
:10D180008E4508D91CEB010100F1FF346CD28E45AD
:10D190006AD90238614440EA0840A0FB0294A1EB3E
:10D1A0000E01A142C846A64656D353D05DB1B3EB9B
:10D1B000080261EB0E0101FA07F722FA06F3F140CB
:10D1C0001F43C5E9007100263146BDE8F087C2F172
:10D1D0002003D8400CFA02FC21FA03F391400143EA
:10D1E0004FEA1C471FFA8CFEB3FBF7F007FB103623
:10D1F0000B0C43EA064300FB0EF69E4204FA02F4CF
:10D2000008D91CEB030300F1FF382FD29E422DD921
:10D21000023863449B1B89B2B3FBF7F607FB163356
:10D2200041EA034106FB0EF38B4208D91CEB0101D6
:10D2300006F1FF3816D28B4214D9023E6144C91A56
:10D2400046EA004638E72E46284605E70646E3E666
:10D250001846F8E64B45A9D2B9EB020864EB0C0E70
:10D260000138A3E74646EAE7204694E74046D1E77F
:10D27000D0467BE7023B614432E7304609E764442D
:10D28000023842E7704700BF02E000F000F8FEE716
:10D2900072B6374880F30888364880F309883648E4
:10D2A0003649086040F20000CCF200004EF63471BE
:10D2B000CEF200010860BFF34F8FBFF36F8F40F2D3
:10D2C0000000C0F2F0004EF68851CEF20001086076
:10D2D000BFF34F8FBFF36F8F4FF00000E1EE100AE6
:10D2E0004EF63C71CEF200010860062080F31488EF
:10D2F000BFF36F8F79F084F87AF04AFA4FF0553027
:10D300001F491B4A91423CBF41F8040BFAE71D49F3
:10D31000184A91423CBF41F8040BFAE71A491B4AEC
:10D320001B4B9A423EBF51F8040B42F8040BF8E73E
:10D3300000201849184A91423CBF41F8040BFAE713
:10D3400079F062F87AF078FA144C154DAC4203DAB1
:10D3500054F8041B8847F9E701F0FEF8114C124D10
:10D36000AC4203DA54F8041B8847F9E779F04AB86D
:10D37000000600200022002000C0000808ED00E0A8
:10D380000000002000060020D8940A080022002097
:10D390009425002098250020301E0120E0C10008BF
:10D3A0002CC200082CC200082CC200082DE9F04F46
:10D3B0002DED108AC1F80CD0C3689D46BDEC108AD3
:10D3C000BDE8F08F002383F311882846A047002092
:10D3D00077F0C0FEFEE777F017FD00DFFEE7000004
:10D3E00001F0FF01102A2BDB10F0070F08D010F816
:10D3F000013B013A8B422DD010F0070F42B3F6D11A
:10D40000F0B441EA012141EA014122F007047FF032
:10D4100000070023F0E80256083C85EA010586EA89
:10D42000010685FA47F5A3FA87F586FA47F6A5FAC5
:10D4300087F68EB9EED1F0BC01F0FF0102F00702D1
:10D4400032B110F8013B013A83EA010313B1F8D17C
:10D450000020704701387047002D06BF354603385D
:10D46000073815F0010F07D1013015F4807F02BF96
:10D47000013015F4C03F0130F0BC0138704700BFE7
:10D4800010F8012B11F8013B012A28BF9A42F7D06E
:10D49000D01A7047034613F8012B002AFBD1181A43
:10D4A0000138704738B50022002304460D46FFF7C7
:10D4B000EDFA28B920462946BDE8384000F00AB800
:10D4C000204605F1004100F005F8404261EB4101C2
:10D4D00038BD00BFD0B50C4B002206460F46FFF703
:10D4E00063F8FFF739FB0446FEF7E4FF074B002221
:10D4F000FFF75AF802460B4630463946FEF79CFEC7
:10D50000FFF72AFB2146D0BD0000F03D0000F041AE
:10D51000036800221B6818470120704737B5019146
:10D520002021044659F06EFAD0B10E4B93F95613F0
:10D53000A1B1B3F95813D3F8F03A019AB3F90C50EA
:10D5400001F10A039D4203DD40F28D33994205DC6F
:10D550002046054B202159F05BFA002003B030BD76
:10D560000120FBE7A045002018E6080808B505F0F3
:10D570008DFDBDE80840012104F0C6BE2DE9F04351
:10D580008FB00E46054605F081FD002780462E220D
:10D59000394602A801977CF0BDFE322301AA394624
:10D5A000404605F05BF8044648B9184A01AB3146DD
:10D5B000284659F01DFC20460FB0BDE8F083DFF887
:10D5C0005890D9F8680703689B6898470028F2D0FC
:10D5D000A9F5405003F0C8FC814630B90C4A3146E9
:10D5E000284659F005FC4C46E5E76946404604F0FC
:10D5F0007DFE0028DFD09DF801305B06DBD5054AB3
:10D600003146284659F0F4FB3C46D4E72CE608089E
:10D6100035E608084CE60808A055002008B5064B7A
:10D6200093F8293D9B0704D5044A59F0E1FB0020FB
:10D6300008BD0120FCE700BFA04500205CE608080B
:10D6400070B50C4C0546D4F868070368DB680E46D5
:10D65000984710B10124204670BDA4F5405003F056
:10D660009FFC04460028F5D1034A3146284659F06C
:10D67000BFFBF0E7A05500206CE608082DE97043D9
:10D68000274BD3F82C3D1D7B814688465DB9254B41
:10D690001B68986A03685B6B984738B9224A414611
:10D6A000484659F0A5FB2846BDE8708345F004FFC5
:10D6B000202146F06DFE38B145F0FEFE1F2146F0F8
:10D6C00067FE08B1194AEAE7484659F093F938B9B4
:10D6D000D9F80030414648465B6BBDE870431847B7
:10D6E00041464846FFF71AFF41460646484659F06C
:10D6F000E1FF20210640484659F084F9414648465A
:10D70000FFF78CFFF5B2054041464846FFF798FF0A
:10D710004146054048465AF09BF90540C3E700BF23
:10D72000A0450020105E002080E6080897E6080863
:10D7300008B5FFF7A3FF054A92F8181D60F34101F1
:10D7400082F8181D024A907108BD00BFA045002054
:10D75000BD5E00202DE9F04106460F4659F088F9DC
:10D76000044668B30221304659F04CF940B305F045
:10D770008DFC4FF48071804604F0C6FD0546F8B973
:10D780004FF40071404604F0BFFDC8B10E485AF096
:10D790007BFB0E4BD3EDA47AF8EEE77A30EE670A06
:10D7A000DFED0B7AB0EEC00AB4EEE70AF1EE10FA44
:10D7B00006DD084B3A460221304659F029F92C463D
:10D7C0002046BDE8F08100BF28590020A055002068
:10D7D0000000C842B4E60808F8B504460F4659F000
:10D7E00095FB10210546204659F00CF958B120460A
:10D7F000FFF7BCFE064630B9044B3A4610212046DE
:10D8000059F006F935462846F8BD00BFC8E60808B5
:10D8100070B505460E4659F06FF8044678B1802180
:10D82000284659F0EFF850B1094B93F88D3243B1C7
:10D83000084B32468021284659F0EAF80024204659
:10D8400070BD31462846BDE8704059F025BD00BF87
:10D85000A0550020DCE608082DE9F04180460E4680
:10D86000FFF78CFE1A4F044610B90024FC710AE041
:10D87000184D05F54053D3F8680703689B6898472F
:10D8800020B90123FB712046BDE8F0810821404604
:10D8900059F0B8F80028F4D095F8E433B02202FB30
:10D8A000035305F50055B3F8EE21B5F954339A4208
:10D8B00006DD094B32460821404659F0A9F8D4E765
:10D8C0003146404659F0C4F90028DAD1CDE700BF0F
:10D8D000BD5E0020A0250020F0E6080859F0DABD62
:10D8E00070B505460E46FFF749FE084B0446D87151
:10D8F00031462846FFF7A4FE31460028284608BFD7
:10D90000002459F061FF204070BD00BFBD5E0020C3
:10D910002DE9F843414F3B788146002B7BD1404CA9
:10D92000D4F82C5D2D7B01263E701DB13B7028463E
:10D93000BDE8F8835AF04AF9054630B9394A3870DB
:10D94000137843F001031370F1E7DFF8F4803AF045
:10D95000E5FE31463AF008F888F804600B2633F00B
:10D96000EDFC013E33F088FC16F0FF06F7D12E499E
:10D9700048465AF041F805F089FBD0F80C22C4F86B
:10D980003C2D90F89432DA0733D404F0D5FE3AF007
:10D99000C5FE3C213AF0FEFD04F6245300221A6035
:10D9A000224B1B68D86A036801211B689847D4F88A
:10D9B0002C2D137B1BB90123137388F804303AF024
:10D9C000ADFE94F81D2D94F81C1D3AF0BDF938F009
:10D9D0007BF937F0A5FC00233B705BF0EBF9144BAF
:10D9E000C3F85C0794F8193D43F0200384F8193D0F
:10D9F0009DE79B07D4D431460E4802F06DF90E48DE
:10DA00005AF042FADFED0D7A20EE270A04F624538D
:10DA100083ED000AC4E7002589E700BF98250020B0
:10DA2000A0450020DC5E002000E70808105E002012
:10DA3000A0550020A0250020285900200AD7233C0B
:10DA4000BD5E00202DE9F043364DD5F82C3D1B7B03
:10DA500087B006460C46002B61D000294BD02146EA
:10DA600030465AF06BF90446002853D02E49304610
:10DA700059F0C2FF05F00AFB074609F023FF804674
:10DA8000384604F0A9F8D8B198F92430022B17D100
:10DA900000264FF00009F1B203AA38460191CDF8F3
:10DAA0000C90CDF81090CDF8149004F073FC01990F
:10DAB00018B103AA404609F011FC0136032EEAD141
:10DAC000D5F82C2D137B1BB100231373174A137148
:10DAD0003AF024FE002139F047FF154B1B68D86A45
:10DAE000036800211B68984795F8193D6FF34513AB
:10DAF00085F8193D0FE005F580530192D3F86807CA
:10DB00000368DB689847019A0028A8D195F8183D6A
:10DB1000DB06A4D40024204607B0BDE8F08301242E
:10DB2000F9E700BFA045002010E70808BD5E00200F
:10DB3000105E002008B500F5005090F8183DC3F3C2
:10DB400080028A420BD061F3820380F8183D31B124
:10DB50003AF0E4FDBDE808400F213AF01BBD08BDD6
:10DB600010B500F500520C4692F8293D03F0010172
:10DB7000A14209D064F3000382F8293DDB0704D4F5
:10DB800002F0EEFA024B9C7210BD02F097FBF9E72F
:10DB9000BD5E002000F5005090F8293D61F341037F
:10DBA00080F8293D014B1973704700BFBD5E00200E
:10DBB0000020704700207047002070470020704709
:10DBC00000207047002070470020704700207047F9
:10DBD00000207047002070470020704700207047E9
:10DBE000704700007047000000F50D50243070476A
:10DBF00000487047F010090800F5005090F81C0D1F
:10DC000070470000034808601C21117008221A6048
:10DC1000704700BFDCE9080837F0A2BF16F054BE19
:10DC20003AF020B845F052B843F00ABA02F0B8BA58
:10DC300002F0ECB902F018B933F01EBB49F060BA3B
:10DC400045F002BB11F00CBD02F034B802F0E4BCA8
:10DC500002F0A6B902F036BC02F0B0BF17F050B91E
:10DC600003F0B2B902F0D0BA02F082BB70B51F4B1C
:10DC7000036000F500530446D3F8AC0C1C4AC3F80B
:10DC8000542B08B109F06CF81A4B236004F580534B
:10DC900093F84C2F42B9D3F8485F2DB1284615F0C0
:10DCA0005DFC284609F058F804F589500C3058F00E
:10DCB000BDF904F58750103047F03EFC04F6C4452A
:10DCC00004F66446B54204D0183D284615F078F8AD
:10DCD000F8E7094BC4F8983804F694103CF0F4FCCB
:10DCE00004F510603CF0F0FC204670BD18EC08080C
:10DCF0004CC009080CA009083C74090838B5474B0A
:10DD0000044640F8043B47F0ADFD04F1100008F074
:10DD10000BFC04F1680037F0B1FC04F5907010F0D2
:10DD20003BF904F5866007F0EBF904F2545009F072
:10DD30004BF804F6980016F071FC04F5446047F0C7
:10DD400019FD04F5516037F0B7F904F5815018302A
:10DD500039F05AFD04F58750103047F0D5FB04F533
:10DD600089500C3058F04EF904F58A50083038F0DC
:10DD700041F804F591501C3048F022FF04F580531F
:10DD800004F593520025104683F86052244B10305E
:10DD90001A6033F0DFF8294604F5965003F00EFCC4
:10DDA00004F5CA50183050F0AFFF04F5EE501C30A7
:10DDB00055F0A4F904F5F750143057F07DFA04F546
:10DDC000FA50183057F0B2FE04F5FD50103007F04D
:10DDD00095F804F50450103051F024FC04F5065079
:10DDE00010304DF0B1FF04F50A50203047F01AF81A
:10DDF00004F5005304F50C5083F80853094D203006
:10DE000058F0D8FC2B6813B107485AF0A5FF2046FC
:10DE1000064936F045FA2C60204638BD0CA00908AA
:10DE200080690020905F002064E70808449F09088B
:10DE300010B502F09BFF45F03FFB0368BDE81040C2
:10DE40005B681847FFF7F4BF38B500F53555044651
:10DE5000284608F043FA09F035FD90F92130D3B196
:10DE600090F84033BBB12846002107F0FDFFDFEDFD
:10DE70000A7A04F2AC7393ED287A20EE270ADFEDDC
:10DE8000077AA7EE270A04F2545083ED280ABDE86A
:10DE9000384009F027BC38BDCDCCCC3D6666663F26
:10DEA000FFF7D2BF10B50121044603F0B1F810B15D
:10DEB000204601F0D9F84FF48051204603F0A8F82D
:10DEC00020B12046BDE8104001F090B810BD000020
:10DED000FFF7E8BF38B50221044603F099F838B1DE
:10DEE0000121204603F094F810B9204601F0BCF857
:10DEF0000221204603F08CF858B3204601F0C2F806
:10DF00004021204603F084F868B104F581551835A6
:10DF1000284638F0FFFF04F5805393F9F03013B131
:10DF2000284639F041F94FF48061204603F070F83B
:10DF300020B104F58150183039F08EF88021204648
:10DF400003F066F860B118F01DF8BDE8384016F02F
:10DF5000B1B90121204603F05BF80028CDD1CFE70D
:10DF60004FF48021204603F053F80028EBD14FF402
:10DF70000021204603F04CF80028E4D138BD000011
:10DF8000FFF7A8BF10B50121044603F041F810B116
:10DF9000204601F077F88021204603F039F828B1B7
:10DFA00017F0F0FFBDE8104016F060B910BD00009A
:10DFB000FFF7E8BF38B54FF6FF71044603F028F8C5
:10DFC00004F5005528B1D5F8182D0721204601F099
:10DFD00061F846F051FE46F075FC95F8183D074A89
:10DFE00083F01003C3F30013537137F06DFE37F065
:10DFF000BFFABDE83840024850F092B9BD5E00203B
:10E00000145C0020FFF7D6BFF0B52DED028B00F5B4
:10E0100096549FB005460121204604F0BDFF05F54A
:10E020004A513031204604F021FE05F54B510831AC
:10E03000204603F0E5FE05F5B05104F54B701031B4
:10E040001BF030FC05F5405405F54B50D4F8B022D8
:10E05000D4F8B43284EDB50A1CA91C301C921D936F
:10E060003CF052F805F54A5105F54C503831203056
:10E07000B0EE608AF0EE408A3BF0DEFE05F54B51D3
:10E0800005F54D501431C4EDAF8A84EDB08A84EDAE
:10E09000B10A14303BF0D0FE84EDB60A3AF03EFBF4
:10E0A00005465AF08FFE2B4B074618680E46FEF7C2
:10E0B00023FACDE91801D4F8D002FEF71DFACDE914
:10E0C0001601D4F8CC02FEF717FACDE91401D4F802
:10E0D000C802FEF711FACDE91201D4F8D802FEF712
:10E0E0000BFACDE91001D4F8D402FEF705FACDE918
:10E0F0000E01D4F8C402FEF7FFF9CDE90C01D4F803
:10E10000B802FEF7F9F9CDE90A01D4F8C002FEF72A
:10E11000F3F9CDE90801D4F8B402FEF7EDF9CDE941
:10E120000601D4F8BC02FEF7E7F9CDE90401D4F802
:10E13000B002FEF7E1F9CDE90076CDE90201064B28
:10E14000064A074928463AF05BF81FB0BDEC028B3F
:10E15000F0BD00BF783A002078E7080886E7080895
:10E16000B3E70808FFF750BF10B5044602F088FE79
:10E170001021204602F04CFF28B117F003FFBDE844
:10E18000104016F065B910BDFFF7EEBF00F58050E6
:10E1900000F5A56300F23450D3ED005AD0ED006ACB
:10E1A000D1ED017A91ED006A26EEE77A67EEA57A65
:10E1B000A6EE257AE6EE267A81ED007AC1ED017AA7
:10E1C0007047000000F5805000F5A56300F2345060
:10E1D000D3ED005AD0ED006AD1ED017A91ED006ADD
:10E1E00027EEA67A67EEA57AA6EE257AE6EE667A9F
:10E1F00081ED007AC1ED017A704700002DE9F04110
:10E200002DED028B054686B0FFF778FDB94B2B60EC
:10E2100005F50E50183005F5005401F01FFC05F50A
:10E220000D531C3305F52C56C4F8F83A062384F830
:10E23000FC3A304658F06CFB04AFAF4BC4F8003BDF
:10E240003946301D4FF0010805F52D568DF8108028
:10E25000143636F0FDFDA94BC4F8543B06F1080016
:10E2600059F0FAFE0723C4F8B03C0023A4F8B43CEC
:10E2700084F8A88C4FF4D27008F06CFDC4F8AC0C94
:10E2800005F53250383059F0E7FE05F533503C3093
:10E2900059F0E2FE9A4B1A6802B91E6099499FED47
:10E2A0009A8A304635F0FCFF984BC4F8543B05F58C
:10E2B00034500123A4F81C3D1E3059F079FD944BD5
:10E2C0000593944B0495009397E80C004FF400716C
:10E2D00005F5355007F0F6FC05F54A5003A9F7EEB1
:10E2E000008A1430CDED038A3BF062FB05F54A50FD
:10E2F000203008F005FA05F540549FED872A84ED9B
:10E30000AC8A05F59653B0EE083A05F54E50C4F8C0
:10E31000A033F0EE432AF0EE420AB0EE430AF0EEEC
:10E32000481AB0EE481A84EDAD8A84EDAE8A84EDC9
:10E33000AF8A84EDB08A84EDB18A84EDB28A84ED2F
:10E34000B38A84EDB48A84EDC08A84EDC18A84EDF9
:10E35000C28A84EDC38A84EDC48A84EDC58A84EDC3
:10E36000C68A84EDC78A84EDE28A84EDE38A84ED6F
:10E37000E48A84EDE58A84EDE68A84EDE78A243038
:10E3800050F074F9B0EE083A05F55150F0EE432A1A
:10E39000B0EE682AF0EE481AB0EE481AF7EE080A16
:10E3A000B1EE0C0A183050F00FFBB0EE083A05F54C
:10E3B0005350F0EE432AB0EE430A9FED572ADFEDAB
:10E3C000570AF0EE481AB0EE481A103050F0FCFA36
:10E3D000B0EE083A05F55550F0EE432A9FED502A6D
:10E3E000DFED500AF0EE481AB0EE481AB0EE680AB7
:10E3F000083050F03BF9B0EE083A05F55750F0EE12
:10E40000432A9FED490AB0EE482AF0EE481AB0EED2
:10E41000481AF0EE480A3C3050F0D6FAF0EE083ACE
:10E4200005F559509FED410AB0EE485AF0EE684AA2
:10E43000B0EE484AB0EE633AF0EE632AB0EE002A3E
:10E44000F0EE481AB0EE481AF6EE000A34304FF0FB
:10E4500017FF374B3748186005F55D52243200230B
:10E4600014279EB207FB06010133097C0029F8D16D
:10E47000314B1E80314B196811B131485AF06CFC98
:10E4800005F55D502C30C4F868071A6002F07EF87C
:10E490002C4BC4F86C3705F55E501C3002F076F852
:10E4A000294BC4F89C3705F55F500C3002F06EF82C
:10E4B000264BC4F8CC3705F55F503C3002F066F8C7
:10E4C000234BC4F8FC3705F5605004F62C0383EDAC
:10E4D000008A83ED018A83ED028A3C3002F056F80F
:10E4E0001C4BC4F83C38284606B0BDEC028BBDE896
:10E4F000F08100BF18EC08082CE708084CC0090898
:10E50000B06200204CBC090800000000D8EC0808EC
:10E5100069DC00080CEC0808CDCC4C3ECDCCCC3EE0
:10E52000CDCCCC3DCDCC4C3D3333333F9A99993F44
:10E53000585F002078220908565F0020145F0020F1
:10E54000B8E70808C02B0908002B0908742C090833
:10E55000602B0908102C090838B5054B1C68236886
:10E560000A461D68034B01462046A847002038BDD7
:10E57000105E0020A025002010B55AF045F8064C8A
:10E58000064B18602046FFF739FE2046044A05492D
:10E59000BDE8104079F0B8B9A0250020105E002039
:10E5A00004C300206DDC000810B504460180024958
:10E5B00035F076FE204610BDA0EC080810B500230B
:10E5C0004FF07C52274C03654FF07E51C0F88030ED
:10E5D000C0F89030C0F8A030C0F8C0304365C0F833
:10E5E0008430C0F89430C0F8A430C0F8C4308366DA
:10E5F0008367C0F89830C0F8A830C0F8B830C36658
:10E60000C367C0F89C30C0F8AC30C0F8BC304FF0E5
:10E610003F430267C0F8B0204267C0F8B420C0F89A
:10E620008820C0F8C820C0F88C2001664466846544
:10E63000C165C0F8CC304FF47A71212046F0CAF899
:10E640004FF47A71222046F0C5F84FF47A712320F6
:10E6500046F0C0F8BDE810404FF47A71242046F02F
:10E66000B9B800BF000080BFF8B52DED068B037B65
:10E67000044643B90023C0F8D430C0F8D830C0F8FD
:10E68000E030C0F8DC30D4ED371A94ED381AD4ED10
:10E69000360A94ED350A8548DFED858A00F03AFCAC
:10E6A0005820B7EE001AFFEE000A94ED350A18F074
:10E6B000EFFF592084ED350AB7EE001AFFEE000A8D
:10E6C00094ED360A18F0E4FF5A2084ED360AB7EECE
:10E6D000001AFFEE000A94ED380A18F0D9FF5B200B
:10E6E00084ED380AB7EE001AFFEE000A94ED370AFF
:10E6F00018F0CEFF84ED370A5AF054FB07EE900A6B
:10E700009FED6C7AF8EE677A04F1100567EE877A70
:10E710002126C4ED027A2F46F7EE009A94ED35AA31
:10E72000D5ED100AB0EE680A6AEE200A79F098FA80
:10E7300094ED368AD5ED140AB0EE409A68EE200AC0
:10E74000B0EE680A79F08CFAD4ED385AD5ED186A33
:10E7500094ED376A95ED1C7A65EEA66A79EE007A3B
:10E76000F0EEE66A26EE077A77EEA67AB0EEC77A82
:10E7700077EE877AB5EEC09AE5EC017A95ED235AEB
:10E78000C5ED079A28EE058A95ED1F5AAAEE058A6F
:10E7900095ED275AA5EE858AD5ED2B5AA6EE258A4A
:10E7A000F1EE10FACCBF01230023B5EEC00A85EDCF
:10E7B000038AF1EE10FA84F8D030C8BF94F8D03054
:10E7C000F5EEC06AC4BF013384F8D030F1EE10FA20
:10E7D000C8BF94F8D030B5EEC07AC4BF013384F816
:10E7E000D030F1EE10FAC2BF94F8D030013384F883
:10E7F000D03094F9D030002BC1BF07EE103AB8EEFC
:10E80000C77AC8EE076AC5ED036A95ED038AB0EED4
:10E81000C87A77EE877AF4EEE97AF1EE10FAC4BF9F
:10E8200079EEC77A45ED017A94F9E83015ED019A51
:10E8300083B1DFED217AB4EEE79AF1EE10FA09D850
:10E84000DFED1E7AB4EEE77AF1EE10FAA4BF4FF0D6
:10E850008043EB6194ED390AD5ED077A20EE270A63
:10E86000D4ED027A20EE270ADFED157A30EE000AA9
:10E8700020EE270A79F06EF9A9EE008A30B201364F
:10E880009FED100A85ED0B8A28EE000AB6B245F01E
:10E890007DFF252E7FF442AFBDEC068B04F12002F4
:10E8A00039460248BDE8F84000F066BBA0250020CC
:10E8B00000000000BD3786359A99193FCDCCCC3E7B
:10E8C000DB0F494000007A440022C0F8D420C0F891
:10E8D000D820C0F8E020C0F8DC20FFF7C5BE00005B
:10E8E00000207047002070470120704790F82C30BE
:10E8F0008B4286BF0C3150F8210000207047000089
:10E9000090F82C308B4286BF0C3150F8210000204B
:10E9100070470000FA207047D0E9083242F4E05214
:10E920004262826A43F4F84342F4E0528262036234
:10E9300070470000014802F085BB00BFA025002001
:10E9400013B54FF45870019108F0FEF9044620B158
:10E95000019943F091FA024B2360204602B010BDAA
:10E9600020ED080870470000704700000020704745
:10E97000704700000020704770470000704700009B
:10E980000320704708207047064BD3F82C3D3BB15D
:10E990001B7B002B0CBF5020D02040F001007047A3
:10E9A0005020FAE7A04500207047000070470000A3
:10E9B00010B52DED028B174BD3F82C4D3CB3D4ED95
:10E9C000360A94ED380AF0EEE00AB0EEC00A79F0AB
:10E9D00047F9D4ED370AB0EE408A94ED350AF0EEEF
:10E9E000E00AB0EEC00A79F03BF9F0EE400AB0EE72
:10E9F000480A79F035F9DFED087A20EE270ABDEEF6
:10EA0000C00A10EE103A18B2BDEC028B10BD2046C1
:10EA1000FAE700BFA04500200000C8423EF090BBCE
:10EA200010B504463FF098FD054802F00BFB054A7F
:10EA3000034606212046BDE810403FF075BD00BFEB
:10EA4000A02500200CED08083EF040BE08B50846A1
:10EA500007F040FF00280CBF0420002008BD000084
:10EA6000162A01D03EF0A4BB03220A700120704791
:10EA700042F0B8BC08B53EF041FD40F41C6040F0E7
:10EA80000D0008BD10B5044608F066F9204610BD1B
:10EA900008B5094B93F8182DD2060BD403F5805313
:10EAA000D3F868070368DB6A984700280CBF022088
:10EAB000042008BD0120FCE7A0450020044B187885
:10EAC00020B9044B93F8190DC0F38010704700BFB4
:10EAD000685E0020A04500201FB50023019302932B
:10EAE000039304F0D3FA01A904F09CF828B101A81B
:10EAF0001BF05AFA05B05DF804FB10F0EFFD90F83A
:10EB0000C432B02202FB030090ED2F0AF2E70000AE
:10EB10000C4B93F88D228AB9A3F5805393F8292DD5
:10EB200051070BD193F8182DD20609D493F8193D4B
:10EB300013F0020F14BF0420012070470520704716
:10EB400003207047A05500202DE9F04F354F97F86E
:10EB50001C3D012B8DB0044652D9334EDFF8E8A09E
:10EB6000082516F9018BB7F9703308F1FF3B43FA1A
:10EB70000BF3D90740D5207C3CF00AFE8146207C6F
:10EB80003DF0D0FD00F12103994505D2207C0DB068
:10EB9000BDE8F04F3EF02EBABBF1070F2CD8DFE8EE
:10EBA0000BF03E04323436383A3C204B1869596930
:10EBB0005A6AD3F804B0D3F818E0D3F80CC0D3EDF8
:10EBC000007A1B6ACDF82520CDF829306222212356
:10EBD000CDE9003207900891207CCDED037A19230E
:10EBE00003AAC221CDF810B0CDF814E0CDF818C0BA
:10EBF0008DF824803CF036FE013D15F0FF05B0D1C4
:10EC00000DB0BDE8F08F0A4BD0E70A4BCEE70A4BB8
:10EC1000CCE70A4BCAE75346C8E7094BC6E7094B9E
:10EC2000C4E700BFA0450020E4ED0808B05900206B
:10EC3000285A0020A05A0020285B0020545B0020A6
:10EC4000A85C002084590020CC5B0020084BD3F83E
:10EC50009C23920701D43EF09DBA03F5805393EDB7
:10EC6000A90ADFED047AB8EEC00A20EE270A704741
:10EC7000A04500200AD7233C10B594B0044603A851
:10EC800007F03EFD1A4BD3F86807036803A95B6BD6
:10EC9000984750B3247C5AF08DF8059BDDED047A3B
:10ECA0000893069B09930023F8EEE77A9FED117A0B
:10ECB0000B930C930D930E930F9310931193129348
:10ECC0004FF6F853ADF84C300023962267EE877A62
:10ECD0008DF84E303323CDE90032079007AA572133
:10ECE0002046CDED0A7A3CF0BDFD14B010BD00BF4A
:10ECF000A05500200AD7233CF0B5254D0E46074607
:10ED00000FCD95B003AC0FC42B682360731EDBB22C
:10ED1000042B29D814AA02EB830353F8445C2B6814
:10ED200028461B6A98472B6804469B6A28469847E2
:10ED3000002305223D7C089009938DF828208DF84A
:10ED400029608DF82A3094B9232221460DF12B0039
:10ED50007BF0E0FA86222E23CDE9003240F2B31197
:10ED600008AA28463CF07EFD052015B0F0BD2046DF
:10ED70000DF12B0304F1200250F8041B43F8041B8F
:10ED80009042F9D102881A8082789A70E2E700BF37
:10ED900028E50808014802F053B900BFA02500206B
:10EDA000014B93F81C0D7047A0450020024B93F8CF
:10EDB000190DC0F340007047A045002030B52DED7F
:10EDC000028B154B91ED018A0546D3F8680703685D
:10EDD00085B0DB690C46984728B9BDEEC88A18EEA5
:10EDE000103ADB0712D5D4E9040118F023FE68B10C
:10EDF000684607F085FC6A462146284642F018FA24
:10EE000020B10649684607F071FD00B1022005B047
:10EE1000BDEC028B30BD00BFA05500204058002043
:10EE20008B8B162B05D0C02B01D1FFF7C7BF43F04A
:10EE300053BC00207047000030B52DED028B8DB023
:10EE40000023054603930493059304F01FF903A9D7
:10EE500003F0E8FE58B304F019F900F5607393E885
:10EE6000070006AC84E80700DDED060A9DED070A01
:10EE70002D7CF1EE600AB1EE400A79F08DF8204663
:10EE8000B0EE408A1BF090F8DFED0B7A089B0B93F5
:10EE9000012228EE278A0C23CDE90032A82109AAF5
:10EEA00028468DED098A8DED0A0A3CF0DBFC0DB099
:10EEB000BDEC028B30BD00BFE02E6542242938B581
:10EEC000054605D040290DD0BDE8384042F050BD80
:10EED0000C213EF0A1F8044610B12846FFF7ACFF24
:10EEE000204638BD0124FBE708B591ED007AF6EE27
:10EEF000007AB4EEE77AF1EE10FA06DD044801225A
:10EF00000521FEF79FFD002008BD0420FCE700BF9F
:10EF1000A05000202DE9F04188B080461B2200213E
:10EF200001A810EE107A10EE906A11EE105A11EE50
:10EF3000904A7BF0EFF9A3238DF8043095238DF8E8
:10EF400005300B238DF8063059F03CFFCDF8070053
:10EF500008F58150CDF80B101B2201A91830CDF80F
:10EF60000F70CDF81360CDF81750CDF81B4038F076
:10EF700013FD08B0BDE8F08170B58CB00D461446A5
:10EF800006462B22002101A87BF0C4F9A3238DF8AB
:10EF9000043095238DF805300C238DF8063059F098
:10EFA00011FF2B68CDF80F302368CDF813306B6854
:10EFB000CDF817306368CDF81B30AB68CDF81F3043
:10EFC000A368CDF80700CDF8233006F58150EB6833
:10EFD000CDF80B10CDF827302B22E368CDF82B307D
:10EFE00001A9183038F0D8FC0CB070BD70B500F530
:10EFF0008154183400F54E56054606F16402204649
:10F000000E2138F089FB06F1900220460F2138F0DE
:10F0100083FB05F5525220460832102138F07CFB64
:10F0200005F5555605F554522046112138F074FB6C
:10F0300006F1480220466C2138F06EFB06F174029E
:10F0400020466D2138F068FB05F5585220462C32D9
:10F050000D2138F061FB05F55C5220460832BDE811
:10F060007040692138F058BB1FB5002301A900F595
:10F07000965001930293039302F09EF905B05DF858
:10F0800004FB000008B504F001F8BDE8084003F0F7
:10F0900015BD00007FB50E464FF6FF7104461546BC
:10F0A00001F0B6FFE8B11022002168467BF032F98A
:10F0B000A3238DF8003095238DF8013004238DF8BB
:10F0C000023059F07FFECDF8030004F58150CDF8F1
:10F0D00007101022694618308DF80B60039538F040
:10F0E000DBFC04B070BD0000A120704738B50446B9
:10F0F00000F5815501F0A6FF183502460B49284658
:10F1000038F0E6FD04F50053284693F81D2D93F8DA
:10F110001C1D38F019FE04F5965004F06FF904F543
:10F120009070BDE838400FF03DBB00BF0CED080803
:10F1300037B5069D044600B92C7801B9697802B943
:10F14000AA7803B9EB78002064F3070061F30F207D
:10F1500062F3174063F31F6003B030BD2DE9F04F39
:10F160002DED0C8B9DB0E04C0D93D4ED379ADFED77
:10F17000DF5A90ED006A04F50054F7EE006AD4F807
:10F180002C3DD3ED367A93ED387AF0EEE77AB0EE97
:10F19000C77A77EE877A9246F4EEE67AF1EE10FAC5
:10F1A000C8BF86EEA78A06460F46DFEDD17AD8BFE4
:10F1B000B0EE668A28EE277AA6EE257A80ED007AF0
:10F1C000D4F82C3D93ED357A93ED376AB0EEC77ADB
:10F1D000B0EEC66A37EE067AB4EEE67AF1EE10FAD1
:10F1E000CCBFC6EE878AF7EE008A90ED017A68EE12
:10F1F000A77AE7EE257AC0ED017A39F08FFA054655
:10F2000059F0E0FD814618EE900A8846FDF774F942
:10F21000CDE9080118EE100AFDF76EF9CDE90601F7
:10F220007068FDF769F9CDE904013068FDF764F90C
:10F23000B04BB14ACDE90201CDE900982846AF496B
:10F24000AF4D38F0DDFFAF4995ED00AA38461AF012
:10F2500097FA8DED160A9AED000ACDED170A30EEF9
:10F260004A0A8DED181A18F0FFF99DED167AD4EDC3
:10F27000E47AB0EEC77AB4EEE77AA5F59B63F1EED7
:10F2800010FA0C9300F10F82D4F82C3D1B7B002B5D
:10F2900000F00982B4F88E93C9F340099DED177A06
:10F2A000B0EEC77AF4EEC77AF1EE10FA00F3FE8101
:10F2B000D4F82C3D1B7B002B00F0F881B4F88E3382
:10F2C00003F001039DED187A0B93B0EEC77AF4EECC
:10F2D000C77AF1EE10FA00F3EB81D4F82C3D1B7BDA
:10F2E000002B00F0E581B4F88E33C3F38008B0EE54
:10F2F000C00AF4EEC07AF1EE10FA00F3DC81D4F823
:10F300002C3D1B7B002B00F0D681B4F88E33C3F369
:10F31000C00B0DAB00930B999FED7B8A5B46424679
:10F320004846FFF705FFC3B20BEE103AC0F30723C0
:10F330000AEE903AC0F307430CEE903A030E0DEE3E
:10F34000103A9DF834300F90002B40F0B7819DF8B3
:10F350003530002B40F0B281F8EE4B7A694ACDEDA2
:10F36000197AF8EE6A7AB0EE690ACDED1A7AF8EEFB
:10F370006C7A19AB394602F52070CDED1B7A4FF04F
:10F3800001FB8DED140ACDED150AB0EE409AF0EEBA
:10F39000608A9DF836305D4C002B40F094811CEE65
:10F3A000901AD4EDB40A97ED020AB0EE691A04F28D
:10F3B000FC504FF005FCB0EE40CA9DF83730002BF2
:10F3C00040F084819AED000A30EE4A0A18F04CF9B8
:10F3D0001DEE101A4E48F0EE690A4FF007F904F5D9
:10F3E000E163DAF800201A6004F20C73F0EE40BA20
:10F3F00083ED00AA474D95EDDD1A4720F1EE410A55
:10F40000B0EE490A18F044F995EDDD1AB0EE40AAC5
:10F41000F1EE410A4820B0EE680A18F039F995ED8E
:10F42000DE1AB0EE409AF1EE410A4920B0EE4C0AE5
:10F4300018F02EF995EDDF1AF0EE408A4A20B0EE72
:10F440006B0AF1EE410A18F023F996ED007AD6ED39
:10F45000017A9DF834308DED148A6AEE076AF0EE79
:10F4600040BACDED106A69EE276A8DED158ACDEDB3
:10F47000116AD4EDAF6A27EE267AD4EDB06A8DED2D
:10F48000127A67EEA67ACDED137AB3B99DF83530CE
:10F490009BB9B8EE4BBAF8EE6AAAB0EE690A1E48FC
:10F4A0008DED19BA19AB12AA10A9CDED1AAA4FF019
:10F4B00055F98DED140ACDED150A9DF83630002B67
:10F4C00040F0078196ED000AD4EDB10A134860EED2
:10F4D000200A1CEE901A28EE800AB0EE691A4FF04E
:10F4E0006FFBF0EE40AA1BE0A0250020A4707D3F3A
:10F4F00000D7233C51F30808681F0908811F090839
:10F50000783A00206858002000000000A055002034
:10F51000145C0020A045002044590020F859002028
:10F52000844814A9FEF74EFE9DF83730002B40F0BA
:10F53000D38096ED010AD4EDB60A7F4860EE200A2A
:10F54000B0EE691A1DEE101A20EE2B0A4FF038FBB0
:10F55000F0EE409AD5F82C3D1B7B7BBB19A9774870
:10F560008DED198A8DED1A8A4FF022FA9FED740AFB
:10F5700074484FF041FB9FED720A73484FF062F8F8
:10F5800019A972488DED198A8DED1A8A4FF010FA7B
:10F590009FED6B0A6E484FF02FFB67489FED680A9E
:10F5A0004FF02AFB04F5327393E807000C9B87E8C1
:10F5B000070003F59B631B68CAF80030B9F1000F20
:10F5C00000F08D80D5F82C3D83ED368A0B9B002B07
:10F5D00000F09080D5F82C3D83ED358AB8F1000F0E
:10F5E00000F09380D5F82C3D83ED388ABBF1000FF5
:10F5F00000F09580D5F82C3D83ED378A9FED558A34
:10F600009FED4F4AD4EDAF2A94EDB21AD7ED000A20
:10F6100062EE882A2AEE082A21EE081A60EE880A8D
:10F62000F0EE443AB0EE443AF0EE441AB0EE440A3A
:10F6300058F07AFC9FED424AD4EDB02A94EDB31A0B
:10F64000D7ED010A62EE882A29EE082A21EE081A6F
:10F6500060EE880AF0EE443AB0EE443AF0EE441A16
:10F66000B0EE440A58F064FC9FED354AD4EDB12A5F
:10F6700094EDB41AD7ED020A62EEC82A28EEC82A21
:10F6800021EE481A60EEC80AF0EE443AB0EE443A71
:10F69000F0EE441AB0EE440A58F04EFC1DB0BDEC3A
:10F6A0000C8BBDE8F08F4FF00109F7E5012309E667
:10F6B0004FF001081BE64FF0010B2AE6F0EE488AF6
:10F6C000B0EE489A65E69FED1ECA76E6DFED1CBAFD
:10F6D00090E6DFED1BAA23E7DFED199A3AE79DF8E4
:10F6E0003430002B7FF472AFD5F82C3D149AC3F858
:10F6F000D8206BE79DF83530002B7FF46FAFD5F83D
:10F700002C3D159AC3F8D42068E79DF83630002BBD
:10F710007FF46CAFD5F82C3DC3ED38AA66E79DF8B1
:10F720003730002B7FF46AAFD5F82C3DC3ED379A04
:10F7300064E700BFA0250020705A0020E85A00208E
:10F74000000000009C5B0020145C00204459002055
:10F75000F85900200000C8422DE9F04F2DED068B2E
:10F760008FB0B74C0393D4ED37AA04F5005480460C
:10F77000D4F82C3D1B7B0D461746002B00F02E8144
:10F78000B4F88E63C6F3400B06F0010AC6F3800995
:10F7900016F0080600D0012603AB4A4651460093F6
:10F7A00058463346FFF7C4FC94EDDD1A95ED000A88
:10F7B0000590F1EE410A9A2017F06AFF94EDDD1AE8
:10F7C000F0EE409AF1EE410A95ED010A9B2017F008
:10F7D0005FFF94EDDE1AB0EE409AF1EE410A95ED2E
:10F7E000020A984D9C2017F053FF94EDDF1AF0EEBB
:10F7F000408A9D2097ED000AF1EE410A17F048FF7C
:10F8000098ED007AD8ED017A9DF80C3069EE876AA0
:10F810000027CDED066A69EE276AB0EE408ACDED8D
:10F82000076AD5EDAF6A0A9727EE267AD5EDB06A5A
:10F830008DED087A67EEA67A0B97CDED097AFBB9C4
:10F840009DF80D30E3B99DF8143007EE103A9DF89D
:10F85000153007EE903AB8EE477AF8EE677AB0EED8
:10F860006A0A0CAB08AA06A905F569708DED0C7A39
:10F87000CDED0D7A4EF072FF8DED0A0ACDED0B0A3B
:10F880009DF80E30002B40F0AE8098ED000AD5EDCB
:10F89000B10A9DF816106C4860EE200AB0EE6A1AA4
:10F8A00028EE800A4FF08CF9B0EE40AA64480AA90D
:10F8B000FEF788FC9DF80F30002B40F0978098ED04
:10F8C000010AD5EDB60A9DF81710604860EE200ACF
:10F8D000B0EE6A1A20EE080A4FF072F9B0EE408AD4
:10F8E000D4F82C3D1B7B7BB959480C970CA90D977C
:10F8F0004FF05EF89FED570A53484FF07DF99FEDAA
:10F90000550A52484FF078F9BBF1000F71D0D4F886
:10F910002C3DC3F8D870BAF1000F74D0D4F82C3D48
:10F92000C3F8D470B9F1000F77D0D4F82C3DC3F8E8
:10F93000E070002E7AD0D4F82C3DC3F8DC709FED37
:10F94000468A9FED444AD5EDAF2A95EDB21A62EE94
:10F95000882A29EE882A21EE081AF0EE443AB0EE01
:10F96000443AF0EE441AF0EE440AB0EE440A58F07D
:10F97000DBFA9FED384AD5EDB02A95EDB31A62EE69
:10F98000882A29EE082A21EE081AF0EE443AB0EE51
:10F99000443AF0EE441AF0EE440AB0EE440A58F04D
:10F9A000C7FA9FED2C4AD5EDB12A95EDB41A62EE57
:10F9B000C82A28EEC82A21EE481AF0EE443AB0EEE2
:10F9C000443AF0EE441AF0EE440AB0EE440A58F01D
:10F9D000B3FA0FB0BDEC068BBDE8F08F4FF0010914
:10F9E000CA46CB46D7E69FED1BAA5FE79FED198A73
:10F9F00076E79DF80C30002B8DD1D4F82C3D0A9A77
:10FA0000C3F8D82087E79DF80D30002B8AD1D4F8B1
:10FA10002C3D0B9AC3F8D42084E79DF80E30002BC0
:10FA200087D1D4F82C3D83ED38AA82E79DF80F30BA
:10FA3000002B84D1D4F82C3D83ED378A7FE700BFBB
:10FA4000A0250020A0550020F8590020705A002061
:10FA500044590020000000000000C84270B5044670
:10FA6000103043F047FB0B4E0B4B236138256019D8
:10FA700043F05EFD66513035B5F54E7FF7D104F5A4
:10FA80004E7044F0D3FF2046044934F009FC204670
:10FA900070BD00BFBC280908D0280908E821090862
:10FAA00037B500F50D5101220831044636F052FCFD
:10FAB0001C4A1368D90706D41B4904F504531033B4
:10FAC0000B600123136004F50E5017490122183012
:10FAD00033F0B2FF0125002304F58151CDE9005335
:10FAE000124A1831FD2033F039FF114B1A68D20742
:10FAF00005D4104A1D6004F58A54083414600D487A
:10FB0000012133F0B5FF34F0D1FD0B4A0B481388C7
:10FB100043F0400313800421002203B0BDE83040CD
:10FB200033F018BF145E002000220020B8A6090898
:10FB3000185E00200C220020485F0020D82609080B
:10FB40000069C0F3401070470F299DBF302303FBAD
:10FB50000100283000207047014B93F96203704781
:10FB6000A0450020024B93F8290D00F001007047DA
:10FB7000A0450020014BD3F8F40A7047A0450020AF
:10FB8000002910B517DB104C94F8FC2ACBB29A422E
:10FB900011D3D4F8F83A0122595CA4F5005000F0D2
:10FBA00063FD94F8193D38B99A0704D5074A1378CC
:10FBB00043F00403137010BD9B07FCD5034A137870
:10FBC00043F00203F6E700BFA0450020DC5E002002
:10FBD000022A10B50F4C12D13522A4F5005000F0C6
:10FBE00043FD94F8193D9B0705D50B4B1A7818B1C6
:10FBF00042F002021A7010BD42F00402FAE794F8D3
:10FC00001C2D8A42F7D143F057FCBDE8104043F069
:10FC100057BB00BFA0450020DC5E0020064A92F8DA
:10FC2000293D92F8282D03F00103134301D143F03D
:10FC300057BA0020704700BFA0450020332901D0EB
:10FC400044F014BA7047000008B50A68332A07D098
:10FC5000382A08D10A790321FFF7BAFF012008BD2D
:10FC60000A790121F8E7BDE8084043F0A5BF00008C
:10FC700030B589B00446684606F042FD04F5965555
:10FC800004A806F03DFD6946284602F0B3FF70B1B6
:10FC900004A9284602F0DEFF48B104A9684606F030
:10FCA0005DFD236800221B6D69462046984709B018
:10FCB00030BD000000F5805292F85425D2070AD4D6
:10FCC00000F50052D2F82C2D117B09B1FFF7D0BFFF
:10FCD0000368DB6C1847704710B586B0044602A86D
:10FCE000019106F00DFD02A904F5965002F082FF85
:10FCF00028B12368019A1B6D02A92046984706B0D7
:10FD000010BD0000F0B5044685B0684604F596576E
:10FD10000E46154606F0F4FC6946384602F09AFF96
:10FD200010B9002005B0F0BD3146384602F0B2FDF2
:10FD30000028F6D0002DF5D004F58054284694F81C
:10FD4000543543F0020384F85435EBE710B500F561
:10FD50000054D4EDDB7AF5EEC07AF1EE10FA8AB0F9
:10FD60004FF0000343D907930893099306AB01931F
:10FD700007AB03AA04A9009300F5965005AB02F067
:10FD800027FEDDED080A9DED070A77F069FFDDED3E
:10FD9000090A77F065FFD4EDDB7A9DED047A77EE02
:10FDA000A76AB4EEE70AF1EE10FAF4EEC76AACBF48
:10FDB00001200020F1EE10FA0CD802309DED037AFC
:10FDC000F4EEC77AF1EE10FA0CD8003818BF012013
:10FDD0000AB010BDF4EEC77AF1EE10FA9CBF013004
:10FDE000C0B2EBE7012894BF00200120F0E700201B
:10FDF000EEE7000038B500F50055044695F8293DBA
:10FE00005A071AD443F0040385F8293D38F086FCDC
:10FE10000122112138F0DEFB084BD3F86807036894
:10FE20009B68984718B995F96933032B05D120468B
:10FE30000621BDE8384000F015BD38BDA0550020B2
:10FE400008B500F5005090F8293D5A070BD56FF31F
:10FE5000820380F8293D38F061FCBDE808400022AB
:10FE6000112138F0B7BB08BD2DE9F043054685B038
:10FE7000684605F5965806F043FC6946404602F090
:10FE8000E9FEC8B105F50053424CD3F82C2D424F82
:10FE9000127B32B1D3EDDB7AF5EEC07AF1EE10FAD7
:10FEA0000DD8238823F4FF7323F001032380284611
:10FEB0000023FB73FFF7C4FF05B0BDE8F0832846BD
:10FEC00001F066F8064618B9284601F027F80646FC
:10FED0002846FFF73BFF814640B93EB12378002B0F
:10FEE00041D1637803F00103FB73E5E76378DB0737
:10FEF000F7D423780133DBB2082B237006D12846D0
:10FF0000FFF724FF10B1404602F0CEFD2378092B05
:10FF100002D1404602F0C0FD2378092BE1D92388A5
:10FF200023F4FF7323F0010343F48573238038F037
:10FF3000F5FB0222102138F04DFB58F03BFF6368BF
:10FF4000C01A47F23053984209D905F52D50134A8B
:10FF5000022114303CF044FE58F02CFF606028462B
:10FF6000FFF748FFBDE7013B23702388C3F3080375
:10FF7000B3F5807FB5D1637860F30003637038F028
:10FF8000CDFB4A46102138F025FB2846FFF758FFE5
:10FF9000A7E700BF1C5E0020BD5E0020EC2809081A
:10FFA00037B5044601A900F5965004F5005502F056
:10FFB000BBFBD5F8403B834206D0C5F8400B38F078
:10FFC000ADFB3E2138F0E6FA04F5805395F9441B69
:10FFD00093F8E82593F9E835994213D0FF2A11D018
:10FFE00085F8443B38F09AFB95F8442B182138F0FB
:10FFF000F1FA04F52D5095F9443B034A04211430DD
:020000040801F1
:100000003CF0EEFD03B030BDFC2809082DE9F043BB
:1000100095B0064658F0CEFE03AB019306F596590F
:1000200002AB0024009305460EAB0BAA08A9484674
:10003000089409940A940B940C940D940E940F94C4
:10004000109402F0B3FCDFED437A9DED0A7AB4EE32
:10005000E77AF1EE10FA074637DB9DED0D7AB4EE44
:10006000E77AF1EE10FAACBF4FF001084FF000084C
:1000700007AB019311AB009304AA06AB05A9484650
:1000800011941294139402F0A3FC06F50054002876
:1000900094F9DC3A08BF002783B17FB1D4F82C3D36
:1000A0001B7B5BB1B8F1000F08D09DED057AF7EE30
:1000B000007AB4EEE77AF1EE10FA09D594F8483BED
:1000C00073B90023C4F84C3B0FE04FF00008CFE7B2
:1000D000D4F84C0B20BBC4F84C5BC4F8500B04E0C4
:1000E000D4F8500B20B9C4F8505B15B0BDE8F083CC
:1000F000281A43F698239842E3D9002584F8485BF0
:10010000C4F8505B38F00AFB2A461D2138F062FA29
:1001100006F52D50104A022114303CF061FDD0E765
:100120002D1AB5F57A7FE0D994F8483B002BDCD145
:10013000012584F8485B38F0F1FA2A461D2138F091
:1001400049FA06F52D50054A022114303CF048FDCD
:10015000CBE700BF00000034142909082F29090843
:1001600010B5044638F0DAFA0022052138F032FAE8
:1001700004F52D50034ABDE81040042114303CF032
:100180002FBD00BF4C29090800F5005090F8193D1B
:100190009B065ABF90F8180DC0F30010012070475D
:1001A00038B5044602F072FF4FF4804102F0ACF81B
:1001B00004F50052054692F8193DC3F3001181423F
:1001C0001CD060F3041304F52D5482F8193D143447
:1001D00060B138F0A3FA02220B2138F0FBF9084A8B
:1001E00020460221BDE838403CF0FABC38F096FACF
:1001F0002A460B2138F0EEF9024AF1E738BD00BF7C
:10020000642909086F29090870B500F500550446EE
:1002100095F95233ABB3D5F8A46C96B358F0CAFD38
:1002200005F6E42393ED000ADFED167A9FED161A2A
:10023000DFED160A861B20EE270A692017F028FA40
:10024000BCEEC00A10EE103A9E4209D295F8293D44
:100250009A0716D520460021BDE87040FDF79ABCEC
:100260000FD995F8293D9B070BD420460121FDF7B6
:1002700091FC04F52C500122BDE870401221FDF7DD
:10028000E1BB70BD00007A440000804F0000000018
:100290000B46012B10B4114604D0052B06D05DF897
:1002A000044B70475DF8044B00F0DCBA5DF8044B7A
:1002B0000122142100F52C50FDF7C4BB2DE9F041BB
:1002C000044604F5005838F029FA0122052138F0D7
:1002D00081F998F956532046003D18BF0125FFF7D4
:1002E00053FF04F52D56143690B11D4A04213046B3
:1002F0003CF076FC0122102104F52C50FDF7A2FB06
:100300000025294620460322BDE8F041FFF7C0BF83
:1003100004F54057D7F868070368DB6A984768B167
:1003200097F88D3253B197F98C32012B06DC0D4AC8
:10033000042130463CF054FC0125E2E7D7F8680779
:100340000368DB6A984718B1D8F8E03A1B0705D470
:10035000054A042130463CF043FCD2E7034AE7E774
:10036000842909089F290908CD290908DC290908D9
:1003700070B50446154638F0D1F90122062138F04F
:1003800029F92046FFF700FF04F52D56143690B1E9
:100390000122072104F52C50FDF754FB144A0421D7
:1003A00030463CF01DFC0025294620460422BDE8CD
:1003B0007040FFF76DBF04F54053EDB2D3F8680706
:1003C0000368DB6A984768B104F50053D3F8E03A54
:1003D0001B0707D535B1074A042130463CF000FC25
:1003E0000125E1E7044A042130463CF0F9FBDBE754
:1003F000002A0908A72909081D2A0908F8B5044692
:1004000058F0D0FC284BB4F8BE201988274E9142F2
:1004100005460ED01A80264B18603378A3B100240D
:10042000347038F07BF922461321BDE8F84038F0EB
:10043000D1B833781F4FC3B93B782BB11C4B1E4A40
:100440001B68C31A934200D8F8BD0123337004F52A
:100450000053D3F82C0D037B0BB1FEF735FA38F0BF
:100460005DF90122132138F0B5F83B78002BEBD071
:100470003378002BE8D00E4A10491368EB1A8B42F0
:10048000E2D904F500541560D4F82C2D137B002B11
:10049000DAD0002313730A4AD4F82C0D1371BDE887
:1004A000F840FEF7E1B800BF265E0020245E002081
:1004B000285E0020255E002080841E0040420F0040
:1004C000BD5E00207FB500F5005300F54E550835A0
:1004D00093F8481B0446284657F084FC04F59656CA
:1004E000684606F00DF96946304602F083FB04F5D4
:1004F0004053029AC3F8A822039AC3F8AC222021E1
:10050000304601F001FFD0B1284657F0BDFC04F59C
:100510004A55FDEEC07A203504F5805417EE901A46
:100520000222284617EE906A06F0EEF894F8543549
:10053000DB0706D401223146284606F0E5F804B070
:1005400070BD0121284606F087F90028F2D0F6E7B1
:10055000012070470020704700207047002070473E
:10056000002070470020704700207047002070472F
:100570009FED010A704700BF000000009FED010AD7
:10058000704700BF0000000070470000104A026082
:10059000104A426002F15001816002F58251C1604F
:1005A0000D49016102F6E411416102F6E811816131
:1005B00002F5F461C16102F2A471016202F5F56114
:1005C00002F2AC728262054A4162C262704700BFA9
:1005D000A82A0908E848002060380020B826002032
:1005E000042917D8DFE801F003070B0F130000F50B
:1005F0005E501C30704700F55D502C30704700F5A0
:100600005F500C30704700F55F503C30704700F58C
:100610006050FAE70020704700F54050D0F86807B6
:1006200003685B681847000038B500F5405504467C
:10063000D5F8680703685B6998470A4B04F50052D0
:10064000187492F81C2DD5F86807DA7003685B6A95
:100650009847014604F593501030BDE8384030F01B
:1006600055BE00BFBD5E00202DE9F84F00F5005AD1
:1006700006469AF81C3D8B420F46914605D18AF8F2
:100680001D2D01252846BDE8F88FFFF7A9FF044678
:1006900020B9304636F006F82546F3E7DAF82C3D67
:1006A0001B7B06F52D5883F0010B08F11408EBB9FC
:1006B000236859461B6820469847054680B306F5CF
:1006C000405306F58150C3F868474A4639468AF8D0
:1006D0001C7D8AF81D9D183037F036FB40460021FE
:1006E00041F0AAFF3046FFF79FFFCBE703689B6806
:1006F0009847E0B11C4800F037FC0546B8B92368BC
:1007000020461B6A9847194A0346042140463CF09C
:1007100067FA38F003F83A460A2137F05BFFB1E791
:10072000236820461B6A9847114A0346EDE70E48A6
:1007300000F036FC0028BBD106F54053D3F868071B
:100740000368DB6898470028B2D023682046DB683E
:10075000984705460028ABD1236820461B6A984776
:10076000044A0346D1E700BFA0250020302A09082B
:10077000822A0908592A09080148FFF775BF00BFF6
:10078000A025002070B5234B93F8293DDB070546D3
:100790000C46164605D5002363602360A3603360D2
:1007A00070BD42F089FE037F002BF4D0EB699FED12
:1007B0001A7A1B68B3F90A3007EE903AF8EEE77A36
:1007C000C7EE876AC4ED016A2B6A1B68B3F90A3069
:1007D00007EE903AF8EEE77AC7EE876AC4ED006A52
:1007E0006B6A1B68B3F90A305B4207EE903AF8EE89
:1007F000E77AC7EE876AC4ED026AAB6A1B68B3F991
:100800000A3007EE903AF8EEE77AC7EE876AC6ED4F
:10081000006AC5E7A045002000007A440020704728
:100820000120704700207047002070470048704743
:10083000487F090800487047F02A090800207047DF
:1008400043691A680023C2F8D43042691268C2F8BA
:10085000D83042691268C2F8DC3042691268C2F8C6
:10086000E03070470A4608B50021FFF7FDFE034A55
:10087000137843F00803137008BD00BFDC5E00204E
:10088000012070470020704701207047002070470A
:1008900000487047482B090800487047502B09084A
:1008A0000320704730B5084B03F54B52083204461D
:1008B00000F1300507CA85E8070003F5A653183391
:1008C00001201B68E36330BDA025002030B52DED6D
:1008D000028B044687B0574D002301AA03A995ED6A
:1008E000378A039304930593FFF74CFF63689DEDEC
:1008F000037AD3ED0E7A68EE277A27EE277A8DED0C
:10090000037A9DED047A67EE277ACDED047AD3ED74
:100910000F7A28EE277ADDED057A67EE877ACDED3E
:10092000057AD3ED107A93F9443028EE278ADDED6D
:10093000017A27EE888A8DED018A1BB903A9284622
:10094000FDF724FC3C4A94ED0C7AD2EDB27A636850
:1009500094ED0F0AD3ED0E6A77EE677AF0EEE77A40
:10096000F4EEE67AF1EE10FA44BFDDED037A77EEAD
:10097000877A94ED0D7A48BFC4ED0C7AD2EDB37A44
:10098000D3ED0E6A77EE677AF0EEE77AF4EEE67A68
:10099000F1EE10FA44BFDDED047A77EE877A94ED3C
:1009A0000E7A48BFC4ED0D7AD2EDB47AD3ED0F6A5A
:1009B000236977EE677AF0EEE77AF4EEE67AF1EE05
:1009C00010FA42BFDDED057A77EE877AC4ED0E7A34
:1009D000D3ED867A30EE670A16F046FE6368D3EDF3
:1009E000107AB0EEC00AB4EEE70AF1EE10FA09D5BB
:1009F00094ED0F0ADDED017A30EE270A16F034FE91
:100A000084ED0F0A00230D488DF808308DF8093069
:100A10008DF80A308DF80B30029BD0F8300D04F1C0
:100A20003C0204F13001FEF799FB07B0BDEC028BEC
:100A300030BD00BFA0250020A0550020A04500200B
:100A40000020704701207047012070470020704748
:100A500000487047A82B090800487047B02B0908C8
:100A6000012070471FB5044600236A4601A901937F
:100A700002930393FFF786FE6369029A1B68C3F82B
:100A8000D4206369019A1B68C3F8D8206369009A6F
:100A90001B68C3F8DC206369039A1B68C3F8E02075
:100AA00004B010BD0120704700207047012070473E
:100AB00000207047004870472AF80808004870472F
:100AC0002AF8080804207047012070477FB50023EA
:100AD0000393049305930193094800238DF808308C
:100AE0008DF809308DF80A308DF80B30029BD0F864
:100AF000300D01AA03A9FEF731FB07B05DF804FB36
:100B0000A045002001207047002070470120704759
:100B10000020704700487047582C0908004870476B
:100B2000642C09080220704710B5044686B00023E3
:100B300001AA03A9039304930593FFF723FE6368B7
:100B40009DED037AD3ED0B6ADDED047A93F9443021
:100B500027EE267A67EEA67A8DED037ACDED047A3C
:100B60001BB9144803A9FDF711FB6368DDED057A95
:100B700093ED0C7A104867EE877A93ED0D7ACDED00
:100B8000057ADDED017AD0F8300D002367EE877A23
:100B90008DF808308DF809308DF80A308DF80B305B
:100BA000029BCDED017A01AA03A9FEF7D5FD06B09F
:100BB00010BD00BFA0250020A045002038B5044688
:100BC00043F08AFF44F058F804F50054054643F01A
:100BD000EDFF43F0DFFCD4F82C0DFDF745FD284672
:100BE000BDE8384043F0EABF10B500F500541421C9
:100BF000D4F8E80A42F0B0FCD4F8EC0A142142F030
:100C0000ABFCD4F8F00A1E2142F0A6FCD4F8F40A9A
:100C10001421BDE8104042F09FBC000038B50546E5
:100C200042F04AFC42F09CFB05F50054C4F8E80A87
:100C300042F042FC42F09EFBC4F8EC0A42F03CFC5D
:100C400042F0A2FBC4F8F00A42F036FC42F0A6FBE8
:100C50004FF47A71C4F8F40AD4F8E80A42F078FC48
:100C6000D4F8EC0A4FF47A7142F072FCD4F8F40A2A
:100C70004FF47A7142F06CFCD4F8F00A4FF47A71B8
:100C800042F066FC2846FFF7AFFF94F8193D43F0A9
:100C9000080384F8193D38BD08B543F0EDFF43F073
:100CA00011FEBDE8084043F0C3BD000000F5005050
:100CB000D0F82C0DFDF708BE38B500F500540546F8
:100CC00094F956332BB900212846BDE83840FCF78B
:100CD00047BFB4F858338B4219D994F8293DDA0745
:100CE0000FD442F0E9FB037F1BB9D4F82C3D1B7BEA
:100CF0003BB194F8283D01335BB2022B02DC84F84F
:100D0000283D38BD032384F8283D0121DCE794F811
:100D1000283D013B5BB2002BF1DC002384F8283D29
:100D200094F8293DDB07CED4EBE7000038B50D463B
:100D3000044658F03FF8002D0B4B09DD04F5005434
:100D4000186094F8193D6FF3C30384F8193D38BD5A
:100D50001B68C01AB0F5C87FF9D904F5005494F89F
:100D6000193D43F00803F0E72C5E0020F7B5044678
:100D700058F020F8064642F09FFB42F071FB04F564
:100D80000055B0B395F8183D43F0200385F8183DA1
:100D9000D5F8F03A20461989FFF78EFFD5F8F03ADA
:100DA00004F54057B3F90A102046FFF7BFFFD7F804
:100DB00060379FED307AF31A07EE903AD5F8F03AA3
:100DC000F8EE677AB3F90A3067EE877A04F54A508D
:100DD000CDED007A07EE903AF8EEE77A6A4601A97F
:100DE0001430CDED017A38F0F1FDC7F8606703B03B
:100DF000F0BD95F8293DDB07F9D404F54053D3F84D
:100E00006007361A42F00EFA80BB42F055FB9FEDA8
:100E10001A7AD0ED067A67EE877A9FED187AF4EEAB
:100E2000C77AF1EE10FAD8BFF0EE477AFCEEE77A17
:100E300017EE903AB342DAD895F95633002BD6D054
:100E400042F03AFB037F23B9D5F82C3D1B7B002BE6
:100E5000CDD037F063FC0222114637F0BBFB0121F5
:100E6000204603B0BDE8F040FCF77ABE4FF47A7339
:100E7000E0E700BF6F12833A00007A440000C842E6
:100E800038B5044600F58665284604F091FB94F8D1
:100E900041049FED087A242202FB0055D5ED0B7A20
:100EA00067EE877A04F54053FDEEE77AC3EDA47A46
:100EB00038BD00BF0000C842FEF718B90148FFF76F
:100EC0009DBA00BFA025002010B5838F044643B90A
:100ED00035F0FEFE92224FF4801135F0B1FE638FA3
:100EE000A387A08F10BD000038B500F596550446C5
:100EF000284600F0DBFC04F58053022283F8E0244E
:100F000004F16800FFF7E0FF014604F6980015F0D1
:100F10009FF82846BDE8384000F0C2BD38B500F55E
:100F200096550446284600F00DFF08B9002038BD4C
:100F300004F50054D4F82C3D1B7B63B910212846DE
:100F400001F0E2F90028F2D14FF400712846BDE823
:100F5000384001F0D9B98021284601F0D5F90028A0
:100F6000E4D11021F2E7000038B500F50053054642
:100F700093F8293D5B0709D4FFF7D0FF044618B961
:100F800005F5965000F0DEFE204638BD0024FBE754
:100F900008B500F5965000F0D5FE002008BD000011
:100FA00010B500F59654204600F0CCFE50B1042157
:100FB000204601F0A9F928B120462021BDE81040C3
:100FC00001F0A2B9002010BD38B500F50055044667
:100FD00095F8183D590719D5D5F82C3D1B7B2BB931
:100FE00020460021BDE83840FCF7A4BD00F5405381
:100FF000D3F868070368DB68984738B195F8193D5E
:101000001A0703D595F8293DDB07E9D538BD00005F
:1010100037B500F581551835044604F500542846C7
:10102000019136F0D9FD94F8183D019960F3C3039E
:10103000284684F8183D03B0BDE8304037F038BB8F
:101040000720704700487047BC2C090837B5054693
:101050001048FFF739FF0190EC2005F075FE0446BB
:1010600010B10199FDF7A0FA05F50050C0F82C4D1C
:1010700024B990F9A413084805F006FB0749204657
:1010800033F01CFB012032F09DFF03B0BDE830407F
:1010900033F00CBB08260020C42C0908A0EC08087B
:1010A00073B5044600F59350103030F0E3F8204655
:1010B000FFF7BAFA04F5355004F03AFE04F587500C
:1010C000103004F5866644F03FFA304604F00EF91D
:1010D00004F52D5014303EF0BBF92046FFF79EFD7D
:1010E0002046FFF7B3FF5F48FFF7EEFE082005F04C
:1010F0002BFE18B14FF07E530360436004F500559A
:10110000C5F8300D42F0D8F99922292143F082F92F
:1011100042F0D2F942F0F2F82046FFF7BDFD95F813
:10112000193D04F5915043F0400385F8193D1C30FA
:1011300045F016FF4C4B4D491B68986A03684FF405
:101140007A72DB6A98470423C4F8743104F590700E
:101150000CF09EFF06F0B6FB4FF40053036306F05D
:10116000B1FB07F041F88023C4F844340121304634
:1011700004F02EFB3E4B00933E4B019304F581504F
:1011800002AB13E90600183036F0D2FB2046FFF719
:10119000ABFE4FF40023C4F8A83BD5F82C0DFDF7A7
:1011A0000DFA012104F52C50FCF7B6F910B12046D8
:1011B000FFF77CFD04F168063046FFF785FED5F8A1
:1011C0002C3D07EE900A04F54B50D3ED390AB8EEEA
:1011D000670AF2EE0E1AB6EE001A1C3039F07CF8EF
:1011E0003046FFF771FED5F82C3D07EE900A04F566
:1011F0004C50D3ED390AB8EE670AF2EE0E1AB7EE8C
:10120000001A203038F092FE3046FFF75DFED5F828
:101210002C3D07EE900A04F54D501430D3ED390AF9
:10122000B8EE670AF2EE0E1AB1EE041A38F07EFE3E
:1012300095F863131A222046FFF716FA60B92122A7
:1012400001212046FFF710FA95F8193D43F00203FB
:1012500085F8193D02B070BD074A137843F00803C2
:101260001370F1E708260020105E0020BD0E010873
:10127000A0250020B90E0108DC5E0020836833B988
:10128000C36823B94068003818BF012070470120A7
:10129000704700002DE9F0412DED048B92B004461B
:1012A00002AD284605F02CFA94F8D433002B70D008
:1012B00004F580630FCB85E80F0094F81034D4ED6B
:1012C000F28A94EDF38A94EDF49A002B61D094F8AD
:1012D000E833002B5DD02846D4F8D883D4F8DC73EB
:1012E000D4F8E063D4F8E443FFF7C8FF002855D1F1
:1012F0002E4B01932D22002106A879F00BF8A32391
:101300008DF8183095238DF8193046238DF81A3052
:1013100057F058FD9FED260ADFED267ACDF81F1015
:1013200068EE808A28EE008A68EEA78A28EE278A6F
:10133000FDEEE88ABDEEC88A18EE903A29EE000A62
:10134000ADF8233018EE103A20EE270ACDF81B0036
:10135000ADF8253016F05CF9BCEEC00ACDF835804A
:1013600010EE103AADF82730019BCDF82930049BE0
:10137000CDF82D30059BCDF83130CDF83970CDF852
:101380003D60CDF8414037F0C9F92D2206A936F06D
:1013900003FB12B0BDEC048BBDE8F08101AA002173
:1013A000284605F069FA0028A2D0A3E75241C07F81
:1013B000E02E65420000C84230B52DED028B8BB0A7
:1013C000044624220D4601A8002178F0A3FFA323A0
:1013D0008DF8043095238DF8053048239FED1F8A42
:1013E0008DF8063057F0EEFCD4ED847A2B68CDF8FA
:1013F0000F3067EE887A95ED020ACDF80B1017EEE4
:10140000903AD4ED857ACDF8133067EE887A6B6820
:10141000CDF8173017EE903ACDF80700CDF81B3015
:1014200016F0CCF810EE103A94ED860ACDF81F3085
:1014300020EE080A16F0C2F810EE103ACDF823306C
:1014400094F824338DF8273037F068F9242201A965
:1014500036F0A2FA0BB0BDEC028B30BDE02E654237
:1014600030B5104689B00D461446FFF707FF28BB7C
:10147000002301931822002102A878F04BFFA32338
:101480008DF8083095238DF8093049238DF80A30FE
:1014900057F098FCA3680593E3680693019BCDF889
:1014A0000F100793CDF80B008DF8135037F036F975
:1014B000182202A936F070FA09B030BD01AA002145
:1014C000204605F06DF90028D2D0D3E710B590B0D2
:1014D000044604A805F014F904A9204601F08AFB8B
:1014E000002846D001F0D2FD01A901F07DF902A942
:1014F000204600F0C3FC00283DD0DDED027AF1EE7D
:10150000677A03AA002104A8CDED027A05F0B4F9A8
:1015100008B91A4B03931F22002108A878F0FAFE9D
:10152000A3238DF8203095238DF821304A238DF8A0
:10153000223057F047FC069BDDED017ACDF82B30C9
:10154000079BCDF82F30F1EE677A039BCDF833304F
:1015500017EE903ACDF83730029BCDF82710CDF832
:101560002300CDF83B3037F0D9F81F2208A936F018
:1015700013FA10B010BDDFED027AC2E75241C07F0E
:101580005241C07F0023036043608360C3600361F6
:1015900043618361C36103627047000090F8C43205
:1015A000B02202FB030390F8082393F8A13012B194
:1015B000012B28BF01231846704700002DE9F04F8A
:1015C00004468BB04FF0000A0D461CF001F984F878
:1015D00020A204F509704FF07E5756F03DFD4FF400
:1015E0007A73A4F87A3284F8805204F52170C4F832
:1015F0006072C4F86472C4F86872002505F080F85F
:1016000004F531790323C4F8983204F53A76C4F826
:10161000AC52C4F8B052C4F8B452C4F8B852C4F8CA
:10162000BC52C4F8C0524846FFF7ACFF04F54E7BED
:101630003046FFF7A7FFC4F82C53C4F83053C4F862
:1016400034535846FFF79EFFC4F85C53C4F8605308
:10165000C4F86453C4F86853C4F86C53C4F87053A6
:10166000C4F87453C4F87853C4F87C53C4F8805356
:10167000C4F88453C4F88853C4F8A453C4F8A853D6
:10168000C4F8AC53C4F8C053C4F8BC53C4F8B8533E
:10169000C4F8C853C4F8CC53C4F8D053C4F8E453C6
:1016A000C4F8E053C4F8DC5304F57B70C4F8B47399
:1016B000C4F8D87305F024F804F5806005F020F82C
:1016C00004F2144304F586601D605D6004F58463D4
:1016D00004F27C481D605D609D6005F011F804F225
:1016E000444340461D605D609D606D4BC4F85434BA
:1016F00004F51073C4F8583404F51173C4F85C345D
:1017000004F51273C4F8603404F51373C4F8643438
:1017100004F25123C4F8683404F51473C4F86C342B
:1017200004F58E6304F254421D605D609D60FFF716
:1017300029FF04F59460FFF725FF04F59A6304F28E
:10174000BC501D605D609D6004F2DC431D605D6007
:101750009D6004F59D631D605D609D6004F2F4432F
:101760001D605D609D6004F204531D605D609D60BE
:1017700004F214531D605D609D6004F5A763C2F818
:10178000D470C2F8D8701D605D609D6004F244534F
:101790001D605D609D6004F5AC631F605D6004F2D8
:1017A00084531D605D609D6004F5B2631D605D60E3
:1017B0009D6004F5B5631D605D609D6004F0A0FF51
:1017C00004F2CC5324221D605D6004F2D4535146D0
:1017D0001D605D6004F2DC5340461D605D6078F082
:1017E00099FD04F5C060C8F82070C8F81070C8F8FA
:1017F0000070FFF7C7FE04F2246304F27C601F60F0
:101800009D605D60DD6004F234631D605D609D601D
:1018100004F5C8631D605D609D6004F24C631D604B
:101820005D609D6004F5CB631D605D609D6004F2AA
:1018300064631D605D609D6004F062FF194B1A498E
:101840001C60204632F02CFD51462422584678F088
:1018500061FDC4F85873C4F84873C4F8387304F5CC
:101860002B7207CA04F52E7383E80700484694EDEF
:10187000B01AD4EDAF0A94EDAE0A16F0E1FA35468F
:10188000494668466E4616F0FDF90FCE0FC50FCEDD
:101890000FC533682B6020460BB0BDE8F08F00BF4A
:1018A000A42F0908305E0020402E090810B5044618
:1018B00088B001F057FC94F93E32012B02D1274841
:1018C00004F000FF022B0AD1032384F83E3204A95E
:1018D000012304F111008DF8103033F0A9FA94F8C7
:1018E0003E3284F8A83204F2544001F0F7FB94F938
:1018F0003D32642B30D1652304A904F23D208DF8DC
:10190000103033F0D3FA04A9204631F0A9FD18B302
:1019100004238DF818300023CDE9013303930F23FE
:101920000593694604A831F01DFF059B28B108AA5C
:1019300002EB8302009942F8581C0133112B0593E6
:10194000EFD954F0C9FF9DED031ADDED020A9DEDBC
:10195000010A652154F07EFF08B010BDD42C09089F
:1019600070B500F52B7600F52E758CB00446314627
:10197000284617F0A5FEE0B996E8070085E80700BD
:1019800004F5317194EDB01AD4EDAF0A94EDAE0ABE
:101990000191084616F054FA02AD019902A816F01A
:1019A00071F90FCD04F53A740FC40FCD0FC42B6835
:1019B00023600CB070BD000013B540F2751200F545
:1019C0000971044601A811F03FFB04F2544001F0F4
:1019D0006FFD20461CF028F901A811F057FB02B05A
:1019E00010BD0000F8B54B68C0F810328B68C0F825
:1019F0001432CB68C0F8183201F1100607460C46C5
:101A000000F54E750FCE0FC50FCE0FC533682B6096
:101A100004F1440207CA07F54B7383E8070004F199
:101A2000500207CA07F5577383E8070004F15C0208
:101A300007CA07F55A7383E80700683494E807007B
:101A400007F55D7383E80700384601F09FFC3846D0
:101A5000BDE8F84001F082BC13B5044600F25440E2
:101A6000019003F03DF904F5BE610198009102F088
:101A700025FD0099204602B0BDE81040FFF7B2BF37
:101A80004A78064BC2F340121A754A78C2F38012A4
:101A90005A750A78C2F300129A757047BD5E00202D
:101AA00013B540F24D32044600F5097101A811F05A
:101AB000CBFA002104F2544001F028FF94F8783268
:101AC00023B120461CF032FE84F8780201A811F000
:101AD000DDFA02B010BD000038B590F82433054699
:101AE0000C462BB1032B0BD095F88032DB070CD4BE
:101AF00005F27C630FCB84E80F0095F88C0603E0B9
:101B00001CF012F90028EFD038BD0020FCE70000DF
:101B100000F2544090ED350A7047000000F2544046
:101B200090ED360A7047000010B490F824230C465C
:101B30002AB1032A0AD000205DF8044B704700F553
:101B4000B56007C884E807000120F5E75DF8044B9D
:101B50001CF0A8B890F89C03431E584258417047A7
:101B600038B590F824330D468BB900F2544001F09B
:101B700007FD044610B90024204638BD01F05EFC84
:101B8000D5ED007A27EE800A85ED000AF4E7D0ED66
:101B9000E67AC1ED007A90F89443002CEBD090EDFA
:101BA000E47ADFED086AB4EEE67AF1EE10FAF7EEC9
:101BB000006AB8BFB0EE667A67EE877AC1ED007A48
:101BC000DAE700BF0000003490F82433032B01D182
:101BD0001BF0E8BF0020704790F82423032A01D1AE
:101BE0001CF05AB900F2544002F0EAB830B505468C
:101BF00085B00C469AB1032A1BD005F52B7017F05F
:101C000099FD01A920468DED010ACDED020A8DED69
:101C1000031A17F03DFB0123184605B030BD90F8BC
:101C2000F035002BF8D000F224630FCB84E80F00CE
:101C3000E3E790F87832002BEED01CF007F9DCE7F0
:101C400090F82423FFF7D2BF7FB590F8242332B158
:101C5000032A4FF0000309D0039304930CE000F231
:101C6000544007B05DF804EB01F0D4BC03A9039322
:101C7000049305931BF08CFF9DED030ADDED040A30
:101C800007B05DF804FB000037B5044640F2C752C8
:101C90000D4600F5097101A811F0D6F92046294634
:101CA0001CF06CF894F82433032B08BF044601A8F9
:101CB00018BF002411F0EAF9204603B030BD00003F
:101CC00010B52DED028BB0F890361B0782B004469C
:101CD00030D5D0F838349FED198A07EE903AB8EE37
:101CE000E77A01A927EE087A00F515708DED017AE3
:101CF00033F08AF8D4F83C3407EE903AF8EEE77AFD
:101D000001A967EE887A04F51670CDED017A33F0FB
:101D10007BF8D4F834349FED0A7A07EE903AF8EE67
:101D2000E77A01A967EE877A04F51770CDED017A9D
:101D300033F06AF802B0BDEC028B10BD95BFD6330C
:101D40000AD7233C90F82403003818BF01207047BD
:101D500038B590F82423032A0C4604D11BF018FF51
:101D60000125284638BD90F87056002DF9D000F2B4
:101D7000646393E8070084E80700F2E710B590F881
:101D8000242303460C461AB1032A0BD0002010BDB1
:101D900090F878060028FAD003F5BE63D3F88430B3
:101DA0000B60F4E71BF00AFF012084ED000AEEE768
:101DB00030B590F8243385B005460C4623B1032B8B
:101DC00009D0002005B030BD00F2544005B0BDE898
:101DD000304002F075BA002302A9029303931BF06E
:101DE000BFFE0028EDD001A928461BF0C5FE002843
:101DF000E7D0029B2360039B6360019BA360E1E744
:101E00001FB500230C4601A9019302930393FFF72A
:101E1000CFFF28B1019B2360029B6360039BA360FB
:101E200004B010BD90F824231AB1032A05D0002075
:101E3000704700F2544002F077BA1BF091BE0000E8
:101E400013B500230C46694600930193FFF7EAFFA0
:101E500018B1009B2360019B636002B010BD0000BD
:101E600090F824231AB1032A05D00020704700F20D
:101E7000544002F04BBA1BF07FBE000013B50C4675
:101E800001A9FFF7EDFF08B1019B236002B010BD6F
:101E900090F93E323BB990F8803213F0010F14BF35
:101EA000032000207047032070470000F7B5044668
:101EB000FFF7EEFF0546002862D0032839D194F8D9
:101EC00078326BB394F88032D8072BD501A920461D
:101ED0001CF01AF8BDF80430002B18BF002594F848
:101EE000206206F0FD06012E4AD10023032D019346
:101EF00007D101A920461CF013F820461BF0F0FF83
:101F0000064604F2544002F01FFB08B994F821037E
:101F10009DF80430D90703D55A0701D59F0632D45E
:101F200000252DE020461BF081FD002808BF00257C
:101F3000D5E70025D3E713F0020F2EE094F95032D5
:101F400023B99DF80430DB092FD0E9E7002EF8D043
:101F50000DF0C4FBFFF722FB022807D99DF80530DE
:101F60009806DDD59DF80430D906D9D5FB6A93F8DB
:101F70009C30002BE5D118E0DA0601D41B0718D5F8
:101F8000284603B0F0BD0028FAD094F82123B4F914
:101F90009036002ACFD013F0010FF1D1154B1F68F6
:101FA000FB6A93F89C30002BC8D19DF804309C0745
:101FB000E2D405F087FC05F083FB0028B0D10DF0DA
:101FC0008DFBFFF7EBFA0228AAD90DF087FB90F8FA
:101FD000C432B02202FB030090ED2F7AF0EE007ABB
:101FE000B4EEE77AF1EE10FA9AD59DF80530DB09E8
:101FF000C6D195E7105E00202DE9F04790F87832C1
:1020000092B00446002B00F0948020461CF0ECF8BF
:102010002046FFF74BFF03287BD104F54E780027BD
:10202000414620460097019702971BF0E5FE69465E
:1020300020461BF0D7FE009BC4F81032019BC4F869
:102040001432029BC4F81832204601F09FF9204652
:1020500001F084F913F096FF054620461BF072FD4F
:102060000028A8BFC6B203AA4FF0FF312046BCBF6C
:1020700095F80A9395F80B630397A8BFB1460497A8
:1020800005971BF0A9FD03A817F054FB4FF00C0AAD
:102090000AFB095084EDD70AC4EDD80A84EDD91A99
:1020A00004F5577100F5117017F054FB04F55D77D6
:1020B0000AFB065584EDCB0AC4EDCC0A84EDCD1A9B
:1020C0003A464FF0FF31204605F5C4751BF098FDE8
:1020D00095E8070006AE86E807003946304617F057
:1020E0009FFB04F53172414609A815F05BFD3146AE
:1020F00009A815F0D9FC09A9204684EDDA0AC4ED37
:10210000DB0A84EDDC1A1BF00BFF09A92046FFF760
:10211000B7FC94F89236002B3AD109A804F0F0FAF3
:1021200009A920461BF00CFE90B3012384F89236D7
:102130002EE0D0F87C321BB956F03CFEC4F87C028D
:10214000154B1B68D86A03685B68984788B156F0DE
:1021500031FED4F87C32C01AB4F87A32984204D9ED
:1021600020461CF0E3FA84F8780294F878327BB1C8
:102170004BE756F01FFED4F87C32C01A41F2873389
:102180009842E4D836F0CAFA36F0AEFA0028DED12A
:1021900012B0BDE8F08700BF105E002090F8243335
:1021A00023B1032B4FF0000007D0704790F93E2277
:1021B000032A04D10A70012070470870FBE7184613
:1021C0007047000073B50D460DF107010446FFF797
:1021D000E5FF064628B19DF807302BB1032B09D047
:1021E0000026304602B070BD04F27C630FCB85E858
:1021F0000F00F6E7294620461BF096FD94F878621A
:10220000EFE7000037B50D460DF107010446FFF773
:10221000C5FF28B19DF8072029462046FFF7E6FCB8
:1022200003B030BD37B50D460DF107010446FFF789
:10223000B5FF28B19DF8073023B1032B11D0002042
:1022400003B030BD04F2F4531B682B6004F5BF6388
:102250001B686B6004F2FC531B68AB6094F8F005DC
:10226000EEE7204629461BF0BDFD94F87802E7E72B
:1022700010B50446FFF70CFE18B1032807D0002064
:1022800010BD04F25440BDE8104001F04DB994F87F
:102290007832002BF3D020461BF0C8FB0028EED08C
:1022A00094F8203203F0FD03012BE9D194F82403C4
:1022B000C31E58425841E3E710B50446FFF7E8FD56
:1022C00080B1032810D194F8780250B156F072FD15
:1022D000D4F87C32C01A44F62063984294BF0020A0
:1022E000012010BD0120FCE70020FAE708B50246F6
:1022F000FFF7CEFD032804D110461BF011FE01208C
:1023000008BD0020FCE7000013B50C4601A9FFF74B
:10231000EDFF20B1019B1C4214BF0120002002B040
:1023200010BD000030B585B00446019102F0FEFDFD
:102330000199054610B9002005B030BD019102F0A9
:10234000C7FD01990028F6D0284602F0C5FD0028F7
:10235000F1D0B4F890365907EED494F82133002B1D
:10236000EAD00B4A1268D26A92F89C506DB103A968
:102370002046FFF7BBFF30B19DF80E309A07DBD542
:10238000C3F38000D8E72846D6E71846D4E700BF55
:10239000105E002010B50446FFF77AFD032804D133
:1023A0002046BDE810401BF095BC002010BD000089
:1023B0002DE9F04190F824338CB00027032B06461A
:1023C0000C46154600970197029719D11BF0BAFBEE
:1023D0006A4680464FF0FF3130461BF011FCB8F1E1
:1023E000FF3FA760676027600DD113F0CBFD2B4640
:1023F00090F80B13224612F053FE0CB0BDE8F081AA
:102400004FF0FF38EBE713F0BDFD2B4622465FFA95
:1024100088F112F045FE95ED000A684617F0C6F9FE
:1024200003A920468DED051A8DED030ACDED040AB2
:1024300017F0F6F906F5317206F54E7103A815F09E
:10244000B1FB214603A815F02FFB84ED021A84EDA1
:10245000000AC4ED010A95ED007ADFED037AA7EEDC
:10246000271A84ED021AC8E70AE81C411FB5DFED00
:102470000B7A20EE270A0C461946094BCDE900429B
:10248000BDEEC00A18688DED020A064B9DF81820B3
:10249000C06A10F0D3FF04B010BD00BFE02E65424B
:1024A000105E0020E82C09082DE9F0472DED028B85
:1024B00092B0002504460F464FF07E5A00F54E714B
:1024C00006A89046CDF818A009950895079516F02E
:1024D00081FB05F0F7F905F0F3F881462046FFF798
:1024E000D7FC032803D094F82433032B4FD19FED5E
:1024F000558ADFED558A00262379F2B2934247D9F7
:102500000AAA71B22046CDF828A00D950C950B951E
:102510001BF07CFC0AA906A816F02CFFB4EEC80A32
:10252000F1EE10FA0DDD494ACDF800803B464849EE
:102530002046FFF79BFF002012B0BDEC028BBDE8E8
:10254000F0870AA906A803950495059516F0FCFEE8
:1025500003A90EA88DED0E0ACDED0F0A8DED101A10
:10256000CDED111A16F07EFCB9F1000F0DD09DEDE6
:10257000050AB0EEC00AB4EEE80AF1EE10FA04DD86
:10258000344ACDF800803B46D1E70136B4E700235A
:1025900094F8806216F0010001D0012BCCD104F533
:1025A000C0610AA8CDF828A00D950C950B9516F0E2
:1025B00011FB0AA906A816F0DDFEDFED227AB4EEC3
:1025C000E70AF1EE10FA05DD204ACDF800803B461F
:1025D0002149ADE72046FFF75BFC03282DD12046BB
:1025E0001BF066FC94F88032DB0728D438BB0AA9BC
:1025F00006A803950495059516F0A6FE03A90EA856
:102600008DED0E0ACDED0F0A8DED101ACDED111ADC
:1026100016F028FCB9F1000F11D09DED050ADFED91
:102620000A7AB0EEC00AB4EEE70AF1EE10FA06DD5F
:10263000084ACDF800803B46CAE70020D2E70120D7
:102640007AE700BFC2B8323EC2B8B23E142D0908C4
:102650001F2D0908AFE70808242D09082DE9F743C5
:102660001546044688460193FFF702FE019A074685
:1026700038B92848284B00682946C06A10F0DEFEA9
:10268000019A019229462046FFF70EFF064668B3DD
:102690002046FFF7FDFB94F93E12019A43B299429E
:1026A00007D01E4B1B4800682946C06A10F0C6FEC2
:1026B0001CE094F82433834207D0019205F002F91C
:1026C00004F0FEFF019A0028EBD12046FFF7E0FB63
:1026D00018B103280FD0124BE4E7134641462A46AF
:1026E00004F2544000F034FF00B107B90026304630
:1026F00003B0BDE8F08394F87892B9F1000F01D1EE
:10270000084BCFE7134641462A4620461BF09EF968
:10271000EAE700BF105E0020282D0908342D0908C3
:10272000642D0908532D090890F82433032B01D197
:102730001BF00CBC0020704713B540F6783200F552
:102740000971044601A810F07FFC20461BF086FAB0
:1027500001A810F09BFC02B010BD000008B50246B5
:10276000FFF796FB10B1032806D008BDBDE808406E
:1027700002F2544000F0ACBEBDE8084010461BF029
:10278000DBBB00000B4610B411462BB1032B09D064
:1027900000205DF8044B70475DF8044B00F2544094
:1027A00000F0A2BE5DF8044B1BF0CABA13B5044694
:1027B000FFF76EFB0A46014620460192FFF7E2FF53
:1027C00070B9084B019A1B68DB6A93F89C0038B11A
:1027D00094F82413204602B0BDE81040FFF7D2BFA2
:1027E00002B010BD105E002070B590F89432DB0787
:1027F00086B004460D460CD403F040F9437C2422F5
:1028000002FB0300D0ED0B7AF1EE677AC5ED007A9A
:102810003BE002A803F074FF01A92046FFF720FB6C
:10282000E8B90CF05BFF94F95032022B0646E3D175
:10283000FEF7B4FE0228DFD996F8C4029FED147AA1
:10284000B02303FB0066D4F88832D6F8B0209B1A78
:1028500007EE903AF8EEE77A67EE877AD6E702A9B4
:102860002046FFF7A3FF0028DBD0D4F88822039B83
:10287000DFED076A9DED017A9B1A07EE903AF8EEBC
:10288000E77AA7EEE67A85ED007A06B070BD00BF64
:102890000AD7233CF0B50C4687B000F5097106460F
:1028A00040F6DD3201A810F0CFFBA36853B9E3680E
:1028B00043B9636833B9002701A810F0E7FB384635
:1028C00007B0F0BD204604F005F80028F3D094E8E6
:1028D0000F0002AD85E80F000021284603F0BCFF81
:1028E00007460028E7D096F89432DB0704D435F089
:1028F00015FF192135F04EFE95E80F0006F5217CF5
:102900008CE80F0096F8943243F0010386F8943275
:10291000304600F073FD3FF095FA46213FF08CFE03
:102920003FF090FA45213FF087FE084BA2681B68F4
:10293000DB6A1A61E2685A6162689A6119F09CFE6A
:102940000028B9D017F0BEFDB6E700BF105E00202A
:1029500038B5144B1B68DD6A2B6804465B68284653
:102960009847F0B12B690BB96A69D2B1C4F88C32BF
:102970006B69C4F89032A969002204F5217003F054
:10298000C3FE94F8943223F0030343F0030384F866
:1029900094323FF057FABDE83840034A06213AF036
:1029A0001FB938BD105E0020782D090813B5044604
:1029B0000193FFF76DFA0328019B05D1204602B071
:1029C000BDE810401BF04CBA002002B010BD000062
:1029D00010B588B004460593FFF75AFA0328059B03
:1029E0004FF000000AD10690079006A802900B98BD
:1029F00001900A98009020461BF040FA08B010BDE4
:102A000038B5044602F092FA0546D0B194F8243362
:102A1000032B03D095F84641204638BD20461BF0D5
:102A20004DF9FF280446F5D00146284602F054FA35
:102A30000028EFD02146284602F04AFA0028E9D0C3
:102A4000EAE70446E8E7000008B590F82433032BD2
:102A500005D013F097FA90F90A03C0B208BD1BF035
:102A600071F8431CF9D1F4E708B590F8243383B129
:102A7000032B03D1BDE808401BF05CB834F028F903
:102A800040F64C524FF4801134F0DAF84FF0FF303A
:102A900008BD1846FCE7000090F82433032B01D151
:102AA0001BF018BD7047000090F82433032B01D1B0
:102AB0001AF040BF704700001AF0A0BF10B50446DE
:102AC0001DF090FF2046FEF7E5FB2046BDE81040D4
:102AD000FEF7FCBC90F824231AB1032A07D001208A
:102AE000704790F95002003818BF012070471BF062
:102AF000EBB9000030B590F840348BB00446002BA1
:102B000064D1B0F89036DB0660D590ED957ADFEDB4
:102B1000307AB0EEC77AB4EEE77AF1EE10FA11D55A
:102B200090ED967AB0EEC77AB4EEE77AF1EE10FA4D
:102B300008D590ED977AB0EEC77AB4EEE77AF1EE69
:102B400010FA43D42046FFF7C5FF00283ED1D4ED4C
:102B5000976ADFED207A9FED206A94ED967A0090D7
:102B600066EEA76AD4ED957A27EE067A67EE867A46
:102B7000FDEEE66ABDEEC77AFDEEE77A16EE903A14
:102B800017EE901A17EE102A06A803F0D7FD06A933
:102B90002046FFF779F8C8B13FF054F90546D4F85C
:102BA0005C02F9F7A9FCCDE90401D4F85802F9F761
:102BB000A3FCCDE90201D4F85402F9F79DFC074AC1
:102BC000CDE90001062128463AF00AF80BB030BDE5
:102BD000000000340000C8428096184B902D090870
:102BE00090F824330BB1032B01D11BF0DFBC002084
:102BF0007047000030B500F57B7304460D460FCBDF
:102C000085E80F0094F8FC0330BD0000D0F898333D
:102C10000B6090F894037047D0F8A0330B6090F8E5
:102C20009D03704710B500F5697203460C4607CA4C
:102C300084E8070093F8B00310BD000030B500F53C
:102C40006D7304460D460FCB85E80F0094F8C4035E
:102C500030BD000030B500F5866304460D460FCB4D
:102C600085E80F0094F8400430BD000010B500F274
:102C7000444203460C4607CA84E8070093F8500410
:102C800010BD00002DE9F0432DED028B8BB0054601
:102C90000E461746FFF7B4FE014680462846FFF76A
:102CA00041FB0446002848D002F040F9414602F0BA
:102CB00015F986ED000A95F93C32002B3ADD0CF04F
:102CC0000DFDFEF76BFC012834D90CF007FD90F8E0
:102CD000C432D5EDE47ADFED5D8A96ED000AB022CC
:102CE00002FB030095F93C32D0ED2F0A07EE103AB3
:102CF000F4EEE87AB8EEC77AF1EE10FAB7EE008A91
:102D0000B8BFF0EE487A37EE201A20EE270A70EEB0
:102D1000C70A40F20E4014F0BBFCD5EDE47AF4EEA5
:102D2000E87AF1EE10FAB8BFF0EE487A80EE277A32
:102D300086ED007A01233B7003E095F8203333B928
:102D4000387020460BB0BDEC028BBDE8F08395F8DF
:102D500024334FF00009CDF80490CDF80890CDF859
:102D60000C9043B1032B10D0CDF81090CDF81490F7
:102D7000CDF818907CB902233B703246414605F2EB
:102D8000544001F027FB0446DBE701A928461AF06E
:102D900089FF0446E8E795F82433002BEBD004A91B
:102DA0002846FFF763FF04460028E4D001A904A8E1
:102DB00016F0E6FC07A8CDED080A8DED091A8DED99
:102DC000070A17F0F1F804A8B0EE408A17F0ECF803
:102DD00095F93C32002B30DD07EE903AF8EEE77AB9
:102DE00040F2544070EE670A37EE801AF5EEC00AE2
:102DF000F1EE10FA48BFDFED160AF4EE410AF1EEEB
:102E000010FAB0EE480AC8BFB0EE601A14F040FCE9
:102E1000B0EE408AD5EDE47A9FED0C7AF4EEC77AF5
:102E2000F1EE10FAB7EE007AB8BFF0EE477A88EE0E
:102E3000277A032386ED007A7DE7B5EEC08AF1EEAE
:102E400010FA48BF9FED028AE4E700BF000000349B
:102E50000000000038B50446FFF7F6FD94F826336D
:102E60008342054604D013F08DF8294611F078FF0F
:102E70002046FFF7E9FD84F8265384F82503204611
:102E8000FFF7E2FD84F827032046FFF7EDFD04F588
:102E9000607184F828032046FEF746FE84F88C0310
:102EA00000F0CCFA04F5677284EDE40A04F566716B
:102EB0002046FFF7E7FE04F5687184F89403204686
:102EC000FEF74EFE04F5697184F89D032046FEF777
:102ED0007BFE04F56D7184F8B0032046FEF7B0FE6A
:102EE00004F5727184F8C4032046FFF79BF904F5DA
:102EF000767184F8D4032046FFF784F904F57B71DA
:102F000084F8E8032046FEF7E7FD04F5806184F8C5
:102F1000FC032046FFF756F984F810042046FEF71C
:102F200093FE04F2144004F5836380ED000AC3EDC0
:102F3000000A16F03BFB04F21C4304F584612046B2
:102F400083ED000A04F22C42FFF732FA04F58661A1
:102F50002046FFF72BFC80B194F840349BB9012345
:102F600084F84034204600F049FA3EF06BFF4521DA
:102F70003FF062FB2046FEF7A3FE94F8403413B9FD
:102F80002046FFF7B7FD04F244412046FEF7E0FE7D
:102F900084F8500438BD000037B50D46044600F0F3
:102FA000E1F81DB912F0EEFF11F0AAFF4FF4EA723A
:102FB00004F5097101A810F047F894F881322BB993
:102FC0002046FFF7C5FC012384F88132224B1D689F
:102FD000A86A03689B6998472046FEF7C1FC204613
:102FE000FEF73AFD204600F03BFA2046FFF704F8D2
:102FF000286B30B10368D4EDD80ADB6894EDD70AAA
:103000009847D4F81C0208B156F02CFE204600F078
:1030100065F82046FEF74AFF94F8A83284F82403A6
:1030200083420ED084F8A80298B10C4D0C4B0328B3
:1030300008BF1D463EF006FF0A4A2B46062139F01E
:10304000CFFD2046FFF706FF01A810F01FF803B0E0
:1030500030BD054DEEE700BF105E002026FD0808DC
:103060001F2D0908BC2D0908242D0908D0EDE47A8C
:103070009FED057AF4EEC77AF1EE10FAB7EE000A8A
:10308000A8BFB0EE670A704700000034014B186813
:10309000704700BF305E002070470000704700009E
:1030A00070470000002070470020704701207047E3
:1030B00003681B6E1847000000207047002070470F
:1030C00000207047002070477047000000207047C4
:1030D00000207047002070477047000070470000D4
:1030E00008B512F04FFF90F80A0308BD30B52DED7A
:1030F000028B9FED1A1ADFED1A0A91ED000A87B0D4
:1031000005462D200C468DED011ACDED000A14F078
:10311000BFFA9DED011ADDED000AF0EE408A2E2087
:1031200094ED010A14F0B4FA9DED011ADDED000AE8
:10313000B0EE408A2F2094ED020A14F0A9FA03A9F8
:1031400005F52B70CDED038A8DED048A8DED050A12
:1031500031F090FF07B0BDEC028B30BDC2B8323EFB
:10316000C2B832BE10B5044655F024FED4F80C3374
:103170001BB1C21AB2F57A7F12D30A4A1268D26A18
:1031800092F89C2002B15BB9C4F80C0394F83D425C
:1031900012F0F8FE80F8054304F094FB80F8254017
:1031A00010BD00BF105E00202DE9F0432DED028B15
:1031B00091ED007AD1ED037A87B08DED047AB0EE0F
:1031C000C77AB5EEC07AF1EE10FADDE91087DDF8C6
:1031D0004C90CDED057A0C4615461E4606DCF0EE09
:1031E000E77AF5EEC07AF1EE10FA02DD04A816F0E7
:1031F00051FA6B20B7EE001AFFEE000A9DED050AAA
:1032000014F046FA6C2089ED000AB7EE001AFFEEC2
:10321000000A9DED040A14F03BFA04A888ED000AA8
:1032200016F09EF9B7EE008A002852D00023C9F8A4
:10323000003088ED008AD4ED067A67EEA77AF4EEC6
:10324000C87AF1EE10FA4ADB0023336085ED008A7C
:10325000DFED3F0A96ED000A7C20B7EE001A14F06D
:1032600017FA86ED000A95ED000A7D20B7EE001AE8
:10327000FFEE000A14F00CFA85ED000AD4ED067A90
:10328000129BDFED346AF1EE677AC3ED007A96EDBA
:10329000007AF0EEC77AF4EEE67AF1EE10FA2BD56A
:1032A00003AB02AA01A9204614F02AFE9DED018A73
:1032B000B0EE480A74F04EFC85ED000AB0EE480A04
:1032C00074F09EFD87ED000A07B0BDEC028BBDE8EF
:1032D000F08304A816F030F90028A7D1ABE738EE48
:1032E000670A14F033F986ED000A94ED087AC7EE08
:1032F000007AC5ED007AABE794ED076AC6EE077A6F
:10330000C7ED007A96ED007AB0EEC77AB4EEE67AB1
:10331000F1EE10FAC4D495ED007ADFED0F6AB0EE4D
:10332000C76AB4EE666AF1EE10FAB9DCB4EE477A19
:10333000F1EE10FAB4D6B0EEE77AB4EE667AF1EEBA
:1033400010FAADDCF4EE677AF1EE10FABCD7A7E71D
:103350000000000000000034FFFF7F7F1FB500F574
:103360001D73039300F51C73029300F51B73019307
:1033700000F51A73009300F5187200F5197300F543
:103380004E71FFF711FF05B05DF804FB9FED196A60
:10339000D0ED846ADFED187A90ED860A66EE866AD3
:1033A00020EE060A26EEA77A10B5BDEEC77AC0ED6C
:1033B0007E6A80ED817A90ED857A27EE067A044662
:1033C00067EE275A60EE277AFDEEE55AFDEEE77AC2
:1033D000C0ED825A17EE903A002BBCBF03F50C43A8
:1033E000A033C0F80C3280ED7F7A14F0E7F884ED5A
:1033F000800A10BDE02E65420000C8421FB50E4B8A
:103400001B680446B3B1684603F07AF96946204662
:10341000FFF720FC20B16A4600212046FEF720F885
:1034200094F89432DB0705D504F52172012120467A
:10343000FEF716F804B010BDD860002008B502F001
:103440001DFBBDE8084001F0E3BD000010B580F8A9
:103450001013044655F0AEFCC4F8140310BD000070
:1034600010B590F81033044653B155F0A3FCD4F8CE
:103470001433C01AB0F57A7F84BF002384F8103368
:1034800094F8183353B155F095FCD4F81C33C01A96
:10349000B0F57A7F84BF002384F8183310BD000094
:1034A00000F5AA700B4607C883E8070001207047A3
:1034B0000023C0F89C30C0F89830C0F89430C0F8B1
:1034C000A830C0F8A430C0F8A030C0F8AC307047C5
:1034D00070470000024B0B604FF07C531360704745
:1034E000000048427047000010B500F5B4700C466B
:1034F0000FC884E80F00204603F0F6F830B1FFF75C
:10350000C5FD00F521700FC884E80F00204603F0C8
:10351000EBF880F00100C0B210BD000010B5044609
:1035200003F01AFC204610BD10B5D0F860310446F7
:103530005BB155F03FFCD4F86031C01A41F28833DA
:10354000984294BF0020012010BD0120FCE700003C
:1035500013B5009303680192DB6D9847DDE9002104
:10356000044628B90448054B0068C06A0FF066FF9E
:10357000204602B010BD00BF105E0020282D0908B3
:1035800013B50446019101F0D1FC2368019ADB6B6D
:10359000014608B190F84611204602B0BDE810403F
:1035A0001847000090ED007ADFED0F7AB0EEC77A91
:1035B000B4EEE77AF1EE10FA14D590ED017AB0EEA0
:1035C000C77AB4EEE77AF1EE10FA0BD590ED027AF5
:1035D000B0EEC77AB4EEE77AF1EE10FA4CBF0120F4
:1035E00000207047002070470000003410B501F043
:1035F0009DFC044658B190F8461101F069FC30B1C9
:1036000094F846112046BDE8104001F065BC00204A
:1036100010BD00002DE9F0432DED028B8FB0036843
:1036200000259B6B0395049505950695029502A9C7
:1036300004469847064638B1FFF700FFDDED027AF1
:1036400027EE800A8DED020A0CF048F8FDF7A6FF80
:103650000746002E50D0DDED027AD4ED646A94ED79
:10366000657A23680B9527EE877A67EEA67A8DED4B
:10367000097ACDED0A7A0C950D955B6B0BA9204666
:1036800009AD98470BA9284615F0D4FE012F8DED02
:10369000030ACDED040A40F2B3800CF01FF890F855
:1036A000C432DFED5B7AB02505FB030090ED308A74
:1036B00028EE278AB0EE480A74F04CFAF0EE408A01
:1036C000B0EE480A74F09CFBCDED0B8A8DED0C0A30
:1036D0000CF004F890F8C43205FB030090ED2F0ABB
:1036E0000BA815F0C7FE09AD8DED050ACDED060A54
:1036F00005A896BB03C885E00128CED89DED020A37
:10370000B5EEC00AF1EE10FA7FDD07AED4F89421D1
:10371000D4F8903107923046089315F0D5FE23680F
:103720000B950C950D955B6B0BA920469847DDED2D
:10373000077A9DED0B7A77EE877A9DED0C7ACDEDC9
:10374000077ADDED087A77EE877A09ABCDED087A56
:1037500096E8030083E8030049E0236993ED000A3B
:10376000B7EE008A38EE408A15F084FE04F5BC7985
:103770008DED090A4846B0EE480ACDED0A0A15F06B
:1037800079FE0BA92846CDED0C0A8DED0B0A15F03C
:1037900051FE04F5C47603AFC4ED5F0A314684EDF3
:1037A0005E0A384615F056FE04F5C0788DED090A1C
:1037B0004046B0EE480ACDED0A0A15F05BFE0BA9B3
:1037C00028468DED0B0ACDED0C0A15F033FE97E877
:1037D000030084ED600AC4ED610A86E803004946EF
:1037E000404615F027FE8DED090ACDED0A0A9DED44
:1037F000090ADDED0A0A0FB0BDEC028BBDE8F083CB
:10380000DDE9030185E80300F1E709950A95EEE794
:1038100035FA8E3C10B590F84213044603F078FC5C
:103820007C23C0B203FB0044D4F8A00010BD00000C
:10383000044B026F1B68DB6A5A60426F9A60826FAA
:10384000DA607047105E0020F0B58FB0044612F0C9
:1038500099FB002302930393049390F80A1301AB9E
:1038600002AA054611F0C2FB04F19407D8B39DEDFE
:10387000010AB5EEC00AF1EE10FA34DD02A815F027
:10388000A5FF04F1B00684ED2C0AC4ED2D0A84EDE9
:103890002E1A3946304615F0A9FF04F17C01304656
:1038A00015F058FF04F1880105A88DED050ACDED4E
:1038B000060A8DED071A15F04DFF08A88DED080AD0
:1038C0009DED010ACDED090A8DED0A1A15F06EFF86
:1038D0000BA904F128008DED0B0ACDED0C0A8DED3E
:1038E0000D1A14F0B9FB95F80A030C2303FB0050E2
:1038F000394600F5117015F02DFF84ED2C0AC4ED4A
:103900002D0A84ED2E1A0FB0F0BD00002DE9F0470E
:103910007E4B00251F682DED028BC0F89C50C0F82F
:103920009850C0F89450C0F88450C0F88050C567D3
:10393000C0F89050C0F88C50C0F88850C0F8B8500B
:10394000C0F8B450C0F8B0500446F86A03688AB0B2
:103950005B680E46984704F12809002854D055F0BA
:1039600029FA42F20F7398424ED8FB6A9FED688A9B
:1039700093ED010A84ED1C0AD3ED020AC4ED1D0A81
:1039800093ED031A484684ED1E1A14F059FA3EF0DE
:1039900059FAD4ED1E7A67EE887A054617EE900A3A
:1039A000F8F7AAFDD4ED1D7A67EE887ACDE9040117
:1039B00017EE900AF8F7A0FDD4ED1C7A67EE887A2E
:1039C000CDE9020117EE900AF8F796FD514ACDE9CC
:1039D00000010621284639F003F994ED1E8AB0EE65
:1039E000480A74F0B7F884ED650AB0EE480A74F03E
:1039F00007FA84ED640A55F0DDF9C4F864010AB0F1
:103A0000BDEC028BBDE8F087A6B194ED1C0AB4EEC4
:103A1000400AF1EE10FA0DD6D4ED1D0AF4EE600A5C
:103A2000F1EE10FA06D694ED1E1AB4EE411AF1EE3C
:103A300010FA67D712F0A6FA90F80B334FF00C0A81
:103A40000AFB030303F5C473074693E8070007AEB8
:103A500086E807004FF01508B2EE028AF2EE068AF9
:103A6000304616F0A1FAB4EEC80AF1EE10FA11D5FC
:103A700008F1FF3818F0FF0815D1304616F094FA17
:103A8000F1EE047AB4EEE70AF1EE10FA1CDC2567D9
:103A9000656731E0304616F087FAB4EEE80AF1EED9
:103AA00010FAE5DCE9E7384611F05EF9384611F026
:103AB00027FA97F80B330AFB037303F5C47393E8F3
:103AC000070086E80700CBE7DDED098A9DED088A4F
:103AD0009DED070A68EEA80AE8EE080AF1EEE00A92
:103AE00074F05AFAF1EE680A84ED1D0AB1EE480A44
:103AF00074F052FA84ED1C0A9FED071AD4ED1D0AEA
:103B000094ED1C0A484614F09BF966E7105E00200D
:103B1000E02E6542302F0908000000000021FFF769
:103B2000F5BE000037B5044608461546019116F06B
:103B30003BFAB7EE007AC7EE007AB4F8D0300198BD
:103B40000133A4F8D03094ED337A37EE277A84ED40
:103B5000337AB0EE007AF4EEC77AF1EE10FA06D5B9
:103B6000B6EE007AF4EEC77AF1EE10FA0DDC9FEDB6
:103B70000E7AF4EEC77AF1EE10FA13D59FED0B7AB8
:103B8000F4EEC77AF1EE10FA0CDDB0EE670A15F02C
:103B90000DFE012085ED000AC5ED010A85ED021A32
:103BA00003B030BD0020FBE700247449BD378635E3
:103BB00070B52DED028B00F1280600F134058AB0B6
:103BC00029460446304615F06DFEB6EE008A20EE1A
:103BD000088A2846B0EE480A15F0E8FD07A93046E5
:103BE000CDED080A8DED091A8DED070A15F0C8FD17
:103BF00030468DED010AB0EE480ACDED020A8DED9A
:103C0000031A15F0D3FD07A928468DED070ACDED5F
:103C1000080A8DED091A15F0B3FD04A901A88DED70
:103C2000040ACDED050A8DED061A15F04FFE324659
:103C300001A920468DED070ACDED080A8DED091A80
:103C4000FFF770FF58B955F0B5F80121C4F86001CD
:103C50002046FFF75BFE0AB0BDEC028B70BD2A4622
:103C600004A92046FFF75EFF0028ECD004F14002D3
:103C700007A92046FFF756FF0028E4D0EBE7000035
:103C800030B52DED028B0D4683B091F842130446FA
:103C9000284603F03DFAC1B27C2000FB015190316F
:103CA00004F1280013F05CFF68468DED000ACDEDAD
:103CB000010A15F07BFCDFED1C7AB4EEE70AF1EEA9
:103CC00010FA05D59FED190A03B0BDEC028B30BD8B
:103CD000684615F0DFFC684615F042FC0028F1D17B
:103CE000284694ED428A03F07BFBF0EE400AB0EEEA
:103CF000480A13F0F7FB80B9284603F071FB84ED06
:103D0000420AB0EE408A73F025FF84ED430AB0EE1C
:103D1000480A74F075F884ED440A04F58671684623
:103D200015F0FCFBD0E700BF0000003400000000ED
:103D30009FED0C7AB4EEC70AF1EE10FA0BD4DFED6A
:103D40000A7AB4EEE70AF1EE10FA07DCC0EE077A61
:103D5000B0EE670A7047F7EE007AF9E7F2EE047A00
:103D6000F6E700BFF3665F3F58A00B4108B51C3073
:103D700015F01CFCF1EE007AB4EEE70AF1EE10FA51
:103D80009DBFF1EE027A37EEC00ADFED047A9FEDB7
:103D9000040A98BF20EE270A08BD00BFCDCC4C3ED8
:103DA000CDCCCC3D08B5836993F9000038B10BF058
:103DB00095FCFDF7F3FB012894BF0020012008BD0E
:103DC000F8B52DED028B054603F07CFD03F078FC81
:103DD0000446B8B3FFF75AF990F8213393B3284655
:103DE000FFF7E0FF064668B30BF078FC90F8C432AA
:103DF000B02707FB030090ED2F7AF0EE087AB4EEBF
:103E0000E77AF1EE10FA1DD495ED1E8A0BF066FCF0
:103E100090F8C432DFED1E7A07FB030090ED300A04
:103E200098EE270A13F0E0FBDFED1A7AB0EEC00A35
:103E3000B4EEE70AF1EE10FA08DC54F0BBFF3446AA
:103E4000C5F85001BDEC028B2046F8BD05F5AA70FF
:103E500016F0AAF8B0EE408A0BF040FC90F8C4329D
:103E60009FED0D7A07FB0303D3ED2F7A67EE877A78
:103E7000B4EEE78AF1EE10FADFD554F09BFFD5F8E7
:103E80005041001BB0F5FA6F8CBF00240124D9E724
:103E9000E02E654200003442CDCC4C3F10B50A4BB9
:103EA0001B68DB6A93F89C3004465BB954F082FFD0
:103EB000D4F86431C01A44F61F6398428CBF0020C6
:103EC000012010BD0020FCE7105E0020F8B52DEDAC
:103ED000068B04460BF002FC054603F0F3FC064695
:103EE00005F0B8FD002840F0AA802046FFF768FFE3
:103EF000002800F0A7803046FFF78CFCD4F8DC30B7
:103F0000984200F018813046FFF784FCD4F8DC308A
:103F1000DFED8E7AC31A08EE903AF8EE688A3046E2
:103F200068EEA78AFFF776FC94F8BC30C4F8DC0092
:103F3000F3B9304603F0D6FBD0B104F1280796F868
:103F400042233946304603F04FFAD4ED1D0AB0EE55
:103F5000401A384694ED1C0A13F072FF0023C4F88F
:103F60009030C4F88C30C4F88830012384F8BC3019
:103F700020463146FFF784FE95F8C40205EB001594
:103F8000B0EE408A2B6FC4F8E03004F1B000D4EDFD
:103F9000129A16F009F86368DFED6D7A93ED007AF6
:103FA000B4EEE77AF1EE10FA68EE299AB0EE40AA84
:103FB00001D5C3ED007A2046B0EE4A0AFFF7B8FEFD
:103FC000636820EE299A93ED000A29EE009AFFF724
:103FD000CDFE29EE009A204684ED249AFFF75EFF7D
:103FE00038B1D4ED247AB2EE007A67EE877AC4ED68
:103FF000247AF0EE007AF4EEE78AF1EE10FA10D5AA
:10400000DFED547AB4EEE7AAF1EE10FA09D5DFED50
:10401000527A69EEA79AD4ED2A7AE9EEA87AC4ED2D
:104020002A7A9FED4E0A94ED367ADFED4D7AB0EEA6
:10403000C88A28EE008AA7EE278A84ED368ABDEC6E
:10404000068BF8BDFFF722F890F82133002B72D0D1
:104050002046FFF7A7FE00286DD095F8C42205EB97
:104060000213196FD4F8E0308B4264D0B02606FBFF
:10407000025292ED2F7AF0EE087AB4EEE77AF1EE82
:1040800010FA58DBCB1AC4F8E01008EE903A95F815
:10409000C4329FED341A94ED1E0ADFED337A06FB2D
:1040A0000353D3ED309A69EE819AF8EE688A39EEBF
:1040B000C00A68EEA78A13F0D7FAB0EE409A73F000
:1040C0009FFE94F8BC30B0EE408AF3B1F3EE047A70
:1040D000F4EEE78AF1EE10FA17DC95F8C40206FB5D
:1040E000005595ED2F7AF2EE027AB4EEE77AF1EE12
:1040F00010FAFFF64AAFDFED1D7AB0EEC99AB4EEC2
:10410000E79AF1EE10FAFFF640AF9FED198AD4ED71
:104110001D0A94ED1C0AB0EE691A04F1280013F090
:104120008FFE012384ED248A84ED238A84ED228A84
:1041300084F8BC3029E7BDEC068B04F188009FEDC4
:104140000D0ABDE8F84015F085BB00BFBD378635C8
:10415000CDCC4C3DC2B8B23E0AD7233CCDCC4C3E70
:10416000CDCC4C3F35FA8E3C6F12833A1904863F12
:1041700000000000EC51783F30B50C2303FB010137
:1041800001F1C003144693E807008BB004AD85E845
:10419000070094E8070083E807002846FFF702FAC3
:1041A00007AB58B194E8070083E807009DED070AC4
:1041B000DDED080A9DED091A0BB030BD95E807004A
:1041C000F2E70000F0B52DED028BD0F818318B60CE
:1041D000D0F81C31CB6085B004460D4601F04EFC92
:1041E00006460BF07BFAA36993F90030022B0746D1
:1041F0004BD1FDF7D3F9022847D997F8C432B02242
:1042000002FB0373D3F8B0100022284602F07CFAB8
:10421000D4ED4A0A94ED490A284602F089FD94F843
:104220002C3163B354F0C6FD9FED228A97F8C41277
:104230008DED018A01AA064638460AF0CDFAD4F877
:1042400020019FED1D0A361A07EE906AF8EE677A94
:1042500040F23C4027EE800AB6EE001AF0EE480A23
:1042600013F016FADDED017A30EE270A04F1F000C2
:104270008DED010A15F0FEF8284602F059FD94F87C
:104280002C0105B0BDEC028BF0BD707C242303FB38
:10429000006696ED0B8AFEF7F9FED0EDA27A9FED4F
:1042A000077AF8EEE77AE8EE077AFDEEE77A17EE9E
:1042B000901AA9E7000000006F12833A0000C8427C
:1042C00030B589B0044668460D4602F019FA6946D1
:1042D0002046FFF709F918B90024204609B030BD7F
:1042E00004A802F00DFA204604A9FFF76BFF04466C
:1042F0000028F1D004A9684602F022FC85ED000AEE
:10430000C5ED010A85ED021AE7E700001FB500239D
:104310000C4601A9019302930393FFF7D1FF08B163
:10432000039B236004B010BD30B585B001AD002300
:104330000C462946019302930393FFF7C1FF0346FE
:1043400018B195E8030084E80300184605B030BDB5
:10435000F8B52DED028B06460F46154600F0E6FD3A
:104360000446A0B1394600F0B3FD80B1204639467D
:1043700000F0B2FD044650B100F0D8FD394600F01F
:10438000ADFD85ED000ABDEC028B2046F8BDFEF7C1
:104390007DFE90F82033B7EE008A7BB13046FFF700
:1043A00001FD044650B1D6ED538AFFF747F8C8EE39
:1043B000007A67EEA87AC5ED007AE4E7D6ED538A75
:1043C000FFF73CF8C8EE007A002467EEA87AC5ED46
:1043D000007AD8E770B52DED048B1646FFF7B8FFCD
:1043E000054670B3FEF752FE90F93C424CB30BF019
:1043F00075F9FDF7D3F8012823D9E4B207EE904A06
:10440000B8EE678A0BF06AF990F8C43296ED009A1C
:10441000B02202FB0300D0ED2F8AFFF70FF838EE31
:10442000281A78EEC80A40F2654029EE000A13F017
:104430002FF9B0EE408AFFF701F8C8EE007AC6ED1A
:10444000007ABDEC048B284670BD000038B50D46DF
:104450000BF044F90446FDF7A1F8022881BF94F857
:10446000C402B02303FB0040D43089BF07C800203A
:1044700085E80700012038BD30B585B000230D4622
:1044800001A9019302930393FFF7E0FF044620B1D3
:10449000039B2B60204605B030BD01F0EFFA417C54
:1044A00000F0A6FF04460028F4D001F0E7FA00F07F
:1044B00051FEB1EE400A85ED000AEBE7F8B5036F57
:1044C0004B60436F8B60836FCB6000F14C070C46F1
:1044D000054601F110060FCF0FC60FCF0FC63B6880
:1044E000336005F1280104F1340014F073FB234616
:1044F000012203F8442B05F1B00207CA83E8070044
:1045000005F1940207CA04F1500383E8070005F19E
:104510001C0207CA04F15C0383E8070004F174017C
:104520002846FFF793FF04F1840184F880002846B1
:10453000FFF7A2FF04F18C0184F888002846FFF7FA
:1045400041FE84F89C00F8BD08B503F0BBF9BDE856
:10455000084003F0B5B8000010B5044615F0D2F9D4
:1045600050B904F10C0015F0CDF928B904F1180088
:10457000BDE8104015F0C6B9012010BD38B500F1F6
:10458000280504462846FFF7E7FF28B12046012109
:10459000BDE83840FFF7BAB9D4ED107AB7EE007A2B
:1045A000F4EEC77AF1EE10FA06D5BFEE007AF4EE1B
:1045B000C77AF1EE10FA12DC2046FFF7F9FA284626
:1045C000FFF7CAFF0028E1D1D4ED107AB2EE047AE9
:1045D000F0EEE77AF4EEC77AF1EE10FAD6DC38BDE9
:1045E00010B5044615F0E0FC2046BDE8104015F07B
:1045F00045B900002DE9F04F2DED048B9FEDCA8ADF
:1046000095B00446F0EE408A8DED028A8DED038A66
:104610008DED048AFFF75AFC11F0B4FC0023054627
:1046200095F87921012AA8BF012293423FD20021A7
:10463000284610F001FB01230028F1D008AB0BAA9B
:10464000002128468DED0B8A8DED0C8A8DED0D8AAB
:1046500010F026FD9DED080AB5EEC00AF1EE10FA45
:1046600023DD0BA815F0B2F811A904F128008DED97
:10467000110ACDED120A8DED131A13F015FA0EA8DA
:104680008DED0E0AB0EE680ACDED0F0A8DED101A11
:1046900015F08CF811A904F1E4008DED110ACDEDAF
:1046A000120A8DED131A15F0A1F80123B8E795F859
:1046B0000B130C2303FB015104F1280B01F5C4710A
:1046C000584613F0F1F984ED070A94ED3F0AC4ED62
:1046D000080A70EE288A84ED091AC4ED3F8A0AF0B0
:1046E000FDFF0646FEF7D2FC90F8213301932046E9
:1046F000FFF758FB80B13046FCF750FF02280BD97A
:1047000096F8C4226169B02303FB026391F900109B
:1047100093F8D200884263DA94ED3F7ADFED837A32
:10472000B4EEE77AF1EE10FA61D4D4ED538AFEF7D5
:104730005DFF58B100F0FAFB90F8461100F0CEFB97
:10474000F0EE408AFEF77AFE60EE288A236C626BF8
:10475000A16A1393B0EE680A11A81292119115F094
:1047600025F804F5AA7102A88DED020ACDED030A21
:104770008DED041A15F03AF854F01CFB002307469F
:1047800084F814312046FFF70DFB002865D096F819
:10479000C422B02302FB033232445268C4F8182109
:1047A00096F8C42202FB033333449B68C4F81C31DF
:1047B00054F000FB0123C4F8200184ED498A84ED04
:1047C0004A8A84F82C31D4F80031002B58D102AB3E
:1047D00093E80700C4F80071F03484E8070006E0AD
:1047E00006EB0212176FD4F80021BA4204D115B0BB
:1047F000BDEC048BBDE8F08FD43393E8070094F848
:1048000014310DF1080C8CE807001BB904F1F0031A
:1048100083E807000123604684F8143104F5AA7187
:1048200014F0AEFF11A904F14C008DED110ACDED8D
:10483000120A8DED131A13F065F9B5EEC00AF1EE08
:1048400010FA8DED110AD8BF9FED370ACDED120A8F
:104850008DED131A84ED530A94E794ED3F7AD4ED6D
:10486000497ADDED026AE6EE877ADDED036AC4ED92
:10487000497AD4ED4A7AE7EE267AC4ED4A7AA2E77D
:10488000D4ED3F7A254B8DED058AF5EEC07AF1EE39
:1048900010FA8DED068A0793A9D9214B9FED217A55
:1048A0001B68DB6A67EE877A93F89CA0B7EE007A04
:1048B000C7EE279ABAF1000F4AD094F8143113B911
:1048C000019B002B42D0E36804F1F001D3ED008A94
:1048D00002A814F055FF69EEA88A8DED110A11A8FF
:1048E000B0EE680ACDED120A8DED131A14F05EFFDA
:1048F0000EA905A88DED0E0ACDED0F0A8DED101A4B
:1049000014F074FF05A8FFF76BFE05A815F014F866
:10491000F0B154F04FFAC4F8600168E7000080BFBE
:10492000105E00200AE81C4100000000CDCC4C3E87
:10493000CDCC4C3FCDCC4C3D920A06BF920A063FEF
:10494000C2B8B23E728A0E3C5B821839DDF804A010
:104950005FED0B8A0023CDE90833CDE90A33CDE9B9
:104960000C334FF0FF32009204F1E40895F87921FE
:10497000012A1046A8BF0120834255D20123002AF4
:10498000FAD095F82D130029F6D0B0EE690A40460A
:1049900014F060FF0DF12C09BAF1000F3FD0424630
:1049A00000212046FFF7E8FB8DED0B0ACDED0C0A48
:1049B0008DED0D1A4846FEF7F5FD70BB4846FFF732
:1049C0000FFE484614F0B8FF38BB05A9484614F05E
:1049D0007DFF05A94846CDED090A8DED0A1A8DED3A
:1049E000080A14F05FFF08A8B0EE409A15F0DCFA50
:1049F000009B33B9F4EEC08AF1EE10FAD8BFB0EEE6
:104A0000680AB5EEC09AF1EE10FAF7EE008A4FF0A0
:104A1000000358BFF0EE408A00930123A6E798E810
:104A2000070089E80700C5E7009B002B7FF471AF02
:104A3000002384F804312046FFF7C2F938B120463C
:104A4000FFF7B0F9002840F025818DED0A8A95F82E
:104A50000A3395F878219A4240F233812B4493F837
:104A60002C33002B00F02D8195F80B3395F879212C
:104A70009A4240F226812B4493F82D33002B00F00C
:104A8000208108A9584613F03DF88DED080ACDEDB8
:104A9000090A8DED0A1A08A814F034FF002840F026
:104AA000178108A814F048FF002840F011815FED3D
:104AB000617A94ED357A68EEA78A5FED637AE7EE66
:104AC000278A04F1B000C4ED358A15F06DFAA368A9
:104AD0005FED687A93ED007AB4EEE77AF1EE10FAC2
:104AE000F0EE408A00F1F8802046B0EE680AFFF749
:104AF0001FF908A814F05AFEA3688DED110ACDED38
:104B0000120A8DED131A93ED000A11A814F04EFE4F
:104B1000204684ED1F0AC4ED200A84ED211AFFF718
:104B2000BDF928B1B2EE000A04F17C0014F092FE47
:104B3000019BB3B33046FCF731FD012831D996F81B
:104B4000C402B02303FB006696ED2F7AF0EE087ADC
:104B5000B4EEE77AF1EE10FA23D595F80B030C23A7
:104B600003FB005595ED627AF1EE0C7AB4EEE77A2C
:104B7000F1EE10FA15DBD4ED1D7A1FED917AF4EE0B
:104B8000C77AF1EE10FA0CDD1FED947AF4EEC77AD5
:104B9000F1EE10FA05D5B6EE000A04F17C0014F02F
:104BA00059FE5FED997AF4EEE78AF1EE10FA22D51C
:104BB0001FED9C0A08A814F0F9FD0EA88DED0E0A51
:104BC00094ED3F0ACDED0F0A8DED101A14F0EEFDB5
:104BD00011A904F1A0008DED110ACDED120A8DEDA1
:104BE000131A14F003FED4ED2B7A94ED3F7A77EE8E
:104BF000877AC4ED2B7A94ED2B7AF1EE047AB4EE39
:104C0000E77AF1EE10FA3BDB11F0BCF95FEDB27A16
:104C100094ED2B1A94ED280A21EE271A40F2C930A0
:104C2000F1EE410A8DED011ACDED000A12F030FDD2
:104C30009DED011ADDED000A84ED280A40F2CA302C
:104C400094ED290A12F024FD9DED011ADDED000A14
:104C500084ED290A40F2CB3094ED2A0A12F018FDB7
:104C600004F1A00184ED2A0A04F1940014F0BEFDC1
:104C700084ED2A8A84ED298A84ED288A84ED2B8AA2
:104C80000023C4F8E430C4F8E830C4F8EC3084ED14
:104C90003F8A9CE5E368F7EE000A93ED000A12F004
:104CA00021FC00283FF4D1AE94ED1C0AB0EEC00AFE
:104CB00073F0A6F8DDED0A7A27EE800A8DED0A0A78
:104CC000C5E68DED0A8A8DED098A8DED088AE2E64A
:104CD0002046FFF753FC1CE6C3ED007A04E700BF53
:104CE0002DE9F04D2DED0E8BA0B0044611F04AF9E0
:104CF000D0EDC67A90ED618AF4EE487AF1EE10FAC2
:104D000048BFB0EE678ADFED677AB4EEE78AF1EE6E
:104D100010FA0EDD0023C4F8E430C4F8E830C4F81B
:104D2000EC300023C4F8FC3020B0BDEC0E8BBDE8A5
:104D3000F08D2046FEF788FD2046FEF739FFB0EEE5
:104D4000480A2046FFF756FC2046FFF717FCFEF7FF
:104D50009DF916AD00F53A7204F1280116A812F07B
:104D600021FF0FCD04F14C060FC60FCD0FC62B68E7
:104D7000336004F1740204F1780304F1700104F16A
:104D80004C0013F0BDF894ED1E8AB0EE480A72F0A4
:104D9000E1FE84ED650AB0EE480A73F031F8204672
:104DA00084ED640AFEF744FDFEF770F904F5B47172
:104DB000FDF750FF53F0FEFFD4F89831C31A632B70
:104DC000B2D9C4F8980133F0A9FC9FED378A0546A3
:104DD00053F0F8FFD4ED1C7A67EE887A074617EE99
:104DE000900A0E46F7F788FBD4ED1D7A67EE887AB5
:104DF00041EC1D0B17EE900AF7F77EFB94ED1E0AAF
:104E000020EE080A41EC1C0B12F0D8FBD4F8D400B9
:104E100010EE108AF7F770FB8246D4F8D8008B4664
:104E2000F7F76AFB41EC180BD4F85401F7F764FB71
:104E300041EC190BD4F85801F7F75EFB41EC1A0B63
:104E4000D4F85C01F7F758FB94ED53EA41EC1B0BE7
:104E5000FEF7F4FACEEE007A17EE900AF7F74CFB65
:104E6000CDE9140140468DED12BB8DED10AB8DEDFB
:104E70000E9B8DED0C8BCDE90AABF7F73DFB0B4B91
:104E800001930B4B0093CDE908018DED06CB8DED21
:104E900004DBCDE90276074B074A0849284633F080
:104EA000C5F941E7CDCC4C3EE02E654235080908F6
:104EB0008B0809085C2F0908672F0908242D0908A9
:104EC00070470000002070477047000000207047C6
:104ED0000020704700207047002070479FED010AB6
:104EE000704700BF000000009FED010A704700BF3F
:104EF00000000000002070477047000010B5044615
:104F0000143000F019F804F12C0000F015F804F149
:104F1000700054F037FF04F1F00054F033FF4FF00D
:104F2000FF33C4F84C31204610BD0000014B186817
:104F3000704700BF345E00207047000008B52DEDBB
:104F4000048BB0EE609AF0EE408A00F00FF9B0EEFC
:104F5000408A89EE280A73F089F8DFED0B7A20EE9B
:104F6000270A73F01BF8DFED097A38EE278ADFEDA8
:104F7000087A28EE278AF7EE007A37EEC00A28EE84
:104F8000000ABDEC048B08BD41D3423E33938843F5
:104F9000A1D81943FFF7D2BF08B52DED048B9FEDC3
:104FA000179AF0EEE07AF4EEC97AF1EE10FAF0EE2C
:104FB000408AB0EE608A04D5B7EE000ABDEC048BDF
:104FC00008BD00F0D3F8DFED0E7A9FED0E7ADFED2D
:104FD0000E6A70EE277A9FED0D0AE8EEC77A27EE8B
:104FE000800A88EE007AC6EE877AF4EEC97AF1EE8E
:104FF00010FAE1DBB1EEE70AE0E700BF00000034A1
:1050000033938843F4FDD43BCDCC9C3F48A18F43E0
:10501000427CD0ED257A242101FB020292ED0B0A9D
:10502000D2ED090A30EE270AFFF7B6BF38B52DEDED
:10503000088BDFED21AA9FED21AA9FED21BA05463D
:10504000B0EE409AF0EE609AB0EE408A1524013C32
:10505000A4B25CB3F0EE490A2846B0EE480AFFF766
:105060006DFFF0EE490A70EE698A284638EE2A0A8A
:10507000FFF764FFB0EEE87A70EE697AB4EECA7AB0
:10508000F1EE10FA77EEE87A10D468EEAA8A40F2D0
:10509000631088EEA70AB0EE4B1A38EE400AF0EE25
:1050A0004A0A12F0F5FAB0EE408AD0E7B0EE480AAC
:1050B000BDEC088B38BD00BFCDCCCC3D0AD7233C1E
:1050C00000247449002343608360C360036143612B
:1050D0008361C361002380F82030704790F820205E
:1050E000531CDBB2062B80F8203000EB820288BF15
:1050F000002382ED010A88BF80F82030704700004D
:105100004FF0FF3310B543610E4BC0F8A8300023B9
:10511000044680F8C830A830FFF7D4FF0A4BC4F823
:10512000A83004F5867052F097FF084B08491C60C0
:1051300020462FF0B5F8D4F89030C4F894302046CB
:1051400010BD00BF8031090890310908385E002089
:105150002832090808B5A83034F010FBDFED027AD8
:1051600020EE270A08BD00BF00007A4490ED3C0AFB
:10517000DFED057AB0EEC07AB4EEE77AF1EE10FA20
:1051800048BF90ED3D0A70470000003473B5D0F879
:10519000A43004460E4663B153F00CFED4F8A4309C
:1051A000C01A42F20F73984203D894ED280A02B055
:1051B00070BD114B1D687DB195F846112846FFF76B
:1051C0008BFE48B195F8461101AA2846FFF77AFEF2
:1051D00010B19DED010AEAE7242101FB064494ED9C
:1051E0000A0ADFED067AB4EEE70AF1EE10FA58BFCC
:1051F000B0EE670ADBE700BF345E002000000C421F
:1052000008B561B10378022B02D9064853F0A4FD1A
:105210005A1C027000EB83004160012008BD084663
:10522000FCE700BF483009082DE9F84305460E4663
:105230009146002400F13C082B7CA34211DD0023A1
:105240004A46314601200DF07BFD24236343074687
:10525000002158F803000DF083FD874204D001348B
:10526000EAE70020BDE8F8830120FBE770B50B46B4
:10527000064614469AB111469847054628B9236850
:1052800020465B68BDE87040184701463046FFF78E
:10529000B7FF20B92B6828465B689847EFE770BDD9
:1052A000F0B50D4685B011461A46CDE90213044605
:1052B000FFF7BAFF034698B90A4800684068042718
:1052C0000668CDE90037DDE902123668064BB047C3
:1052D00002462946204605B0BDE8F040FFF7C6BFAC
:1052E0000022F6E7105E0020801A06007FB5D0EDA0
:1052F000247A9FED347AF0EEE77AF4EEC77A012350
:10530000F1EE10FA0446037609D49030002303A985
:10531000019003932FF060FD01982FF099F900227E
:1053200076232949E2632266C4F884202046FFF7E9
:10533000B7FF2378032B28D0237C032B25D094F9A7
:105340009D20002A15DAD4F80031DA041FD4002594
:10535000637EEB40DB07EAB21FD40135082DF7D19D
:1053600023781BB1237C0BB1636873B9174801F034
:10537000A9F977231649D2B22046FFF791FF237887
:10538000032B02D0237C032BDDD104B070BD637EE0
:10539000002BDCD101236376D9E73820019201F09C
:1053A000D3FC064618B1019A214655F0DDFB314683
:1053B0002046FFF725FF2378032BE6D0237C032B21
:1053C000CBD1E2E700000034F9A0060864300908F8
:1053D000C9A80608054B1B682BB141694A1C02D0BD
:1053E000184633F065B90020704700BFD860002030
:1053F00002290BD8242303FB010191F8390030B1B5
:1054000091F83A0018B191F83B00704700207047BE
:105410002DE9F047044653F0CDFCD4F8F86042F291
:105420001073861B9E4288BFC4F8F80000274FF017
:10543000240942F2107A237CFDB2AB421CD92946E2
:105440002046FFF7D5FF70B109FB054898ED0D0A1E
:10545000D8ED097AD4ED250A30EE270A2046FFF769
:10546000E5FD88ED0C0A564504D909FB05403030AE
:105470002FF0EEF80137DEE7617C2046FFF786FE6D
:1054800084ED3D0ABDE8F08770B52DED028B044632
:1054900086B053F08FFCD4F89830C31AB3F57A7FF6
:1054A00005463FD33C4B94ED257A1B689FED3B8A24
:1054B000DB6AD4ED247A93F89C60F0EEC76AF4EED0
:1054C000C86AF1EE10FA22D5F0EEE76AF4EEC86A87
:1054D000F1EE10FA1BD502A801F012F916BBFDF788
:1054E000D5FD02A9FDF7B6FBE0B1DDED037A9FED36
:1054F0002C7AF8EEE77A67EE877AB0EEE77AB4EEC8
:10550000C87AF1EE10FA11D4C4ED257A11E077EEE5
:10551000676AB7EE006AF0EEE66AF4EEC66AF1EE8C
:1055200010FA1EDC06B0BDEC028B70BD1D4BC4F83A
:105530009430C4F89850FDF7A9FDFDF7FDF820461A
:10554000FFF766FF3CF07EFC0546D4F89400F6F7C2
:10555000D3FF154ACDE900010621284637F040FB6C
:10556000E0E7F0EEE76AF4EEC86AF1EE10FAD9D49B
:10557000002EC9D02046903080ED007A2FF068F8D8
:105580003CF060FC094A012106B0BDEC028BBDE88D
:10559000704037F025BB00BF105E002000000034D3
:1055A0000AD7233C6F12833AAD30090888300908C6
:1055B000F0B52DED048B85B0044640F2723200F553
:1055C000867103A80DF040FDD4ED227AD4ED236A54
:1055D0009FED796A637C37EEE67A2422B0EEC77AD3
:1055E000B4EEC67AF1EE10FAC1BF9FED747A67EEA1
:1055F000877A9FED737AE6EE877A02FB03430025F4
:10560000C4ED237A93F839602378E9B28B4206D946
:1056100004EB81030135586800F09EFAF4E7DFEDF2
:10562000698A9FED698A9FED699A0027237CFDB204
:10563000AB4264D9242303FB054393F83920002AA5
:105640005BD0D3ED0C7AF4EEE87AF1EE10FA0BDBD6
:10565000F4EE677AF1EE10FA06D6F0EEE77AF4EEA1
:10566000487AF1EE10FA04DD242303FB05435A6A5D
:105670001A63242303FB0543D3ED090AD3ED0D7A06
:1056800093F8382070EEA70AA2B993ED0C0A2046D1
:10569000FFF780FCD4ED257A30EE670AB4EE400ABD
:1056A000F1EE10FA16D7242303FB0545002385F8F5
:1056B0003A3022E0012A09BFD3ED0C7A93ED0B0AB0
:1056C00077EEE00AD4ED3B7A04BF80EE897A87EE6C
:1056D000270AE3E7F0EEC07AF4EE487A2423F1EEED
:1056E00010FA03FB0545E1DC012385F83A30D4EDDF
:1056F000237A37EE800A85ED0B0A013796E7627C44
:1057000020461146FFF774FE48B1242101FB0242F6
:1057100092ED0B0AD16904F1A80034F00FF894F966
:105720009C10277C002907DBB94205DACAB2114672
:105730002046FFF75DFE68B900226274D5B2AF4221
:1057400009D929462046FFF753FE01320028F5D03B
:10575000657400E062742046FFF796FE2046FFF76E
:1057600039FE10B1204654F04BFE637C242505FB26
:10577000034393F83930B34216D032F0CFFF4FF6DF
:10578000FF7132F095FF78B1607C05FB004494F81E
:105790003930002B14BF00220422019232F0BEFFE8
:1057A000019A122132F016FF03A80DF06FFC05B02C
:1057B000BDEC048BF0BD00BF0AD7233C0AD7A33C45
:1057C00048E17A3F00000034FFFF7F7F0020194648
:1057D0002DE9F04F0446007C0F4687B004F13A03F0
:1057E00000220121D5B2A84203F1240305D903F810
:1057F000231C03F8241C0132F4E76F4B1E68F06A87
:1058000003685B68984740B13CF01CFB6B4A06217B
:1058100007B0BDE8F04F37F0E3B93CF013FB684A3E
:10582000062137F0DDF9002303A904F18800039372
:105830002FF0D2FA0A2553F0BDFA80462046FFF732
:10584000B7FE53F0B7FAA0EB0800B0F5FA7F02D923
:105850005C4800F037FFB06A03680A215B6898472C
:10586000617C2046FFF7C4FD0028E7D0B06A0368DA
:1058700064215B68013D984715F0FF05DBD1524B71
:1058800005951B888DF80650CDE90355ADF8043019
:10589000052553F08FFA80462046FFF789FE53F026
:1058A00089FAA0EB0800B0F5FA7FD1D8617C2046D8
:1058B000FFF79EFD0028EFD094F810B00DF10C0812
:1058C000A14601AA4FF0000A5FFA8AF18B4516D96A
:1058D0002046FFF78DFD50B1D8ED007A99ED097A99
:1058E000137877EE877A0133C8ED007A13700AF1E6
:1058F000010A08F1040809F124090132E4E7B06A59
:10590000036864215B68013D984715F0FF05C0D12D
:10591000A9464FF02408237C5FFA89F6B34226D9C2
:1059200006AB334413F8143C33B908FB064686F83B
:105930003B3009F10109EEE7002FFAD007EE903A6B
:1059400006AA02EB8602F8EEE77A12ED030AD4ED1E
:10595000250A204680EE270AFFF768FB08FB064071
:1059600002A930308DED020A2FF036FAE1E7617CB2
:10597000DFF85C902046FFF709FC002684ED3D0A25
:105980004FF02408237CF7B2BB420FD908FB074332
:1059900093F83B3043B13CF055FA7B1C4A46062154
:1059A00037F01EF90135EDB20136EBE70DB90748C6
:1059B0004FE707B0BDE8F08F105E0020C83009083F
:1059C000F3300908093109083CE5080845310908A0
:1059D0002331090808B5037C022B02D9034853F090
:1059E000BBF95A1C0274184608BD00BF643109088F
:1059F00038B5057C02460024E1B28D4206D9104636
:105A0000FFF7F6FC01340028F6D138BD281E18BF78
:105A10000120FAE770B50D4609780729044606D833
:105A2000027E437E22B901228A401343437670BD31
:105A3000002BFCD000262278F3B29A42F7D904EB6F
:105A40008303294658680368DB6898470136F2E704
:105A500037B50D460192FFF7CBFF0199044630B9E7
:105A60000448054B00682A46C06A0DF0E7FC204652
:105A700003B030BD105E00200B5D0A08014B1868B2
:105A8000704700BF385E00207047000073B5436860
:105A90001B7C8B4205460C4642D900F108012122AD
:105AA00001A80DF0D1FA53F085F96A68242303FBAD
:105AB0000423D969411AB1F5FA7F33D2196A401A21
:105AC000B0F5FA6F2ED2D3ED097A9FED177AF0EE8A
:105AD000E77AF4EEC77AF1EE10FA54BF0120002005
:105AE000242606FB04F31A449FED107A82F839004D
:105AF00069680B44D3ED0A7AF4EEC77AF1EE10FA36
:105B000006D49FED0B7AF4EEC77AF1EE10FA04DDBD
:105B100006FB0411002381F8393001A80DF0B6FA14
:105B200002B070BD0020DBE700000034000048C375
:105B30000000484310B5044B0446C0E9003108306A
:105B400052F08AFA204610BD203309084368242009
:105B500000FB0131CA63704713B503680191044625
:105B60009B689847236801991B69204602B0BDE8ED
:105B700010401847F8B52DED028B43681B7C8B4213
:105B800005460C46F0EE408AB0EE608A1FD953F00D
:105B900011F924276B6867433B4493ED090AF0EE43
:105BA000680A064611F09EFCA0B96B68242202FB2D
:105BB00004331E626B6824214C432344C3ED098ADD
:105BC0006B68234483ED0A8A69680C44E661BDEC86
:105BD000028BF8BD6B683B4493ED0A0AF0EE480A6D
:105BE00011F080FC0028E0D0E4E70000DFED2A7A25
:105BF000B0EEC07AB4EE677AF1EE10FA49DCB4EE9A
:105C0000400AF1EE10FA44D6436893F9FC3063B1D0
:105C100090ED087ADFED217AF0EEC76AF4EEE76ADC
:105C2000F1EE10FA03D580ED080A01232BE077EEA0
:105C3000407A37EE006AF0EEE77AC7EE866ADBB2AA
:105C40009FED176A07EE903A26EE866AF8EE677ABD
:105C5000B4EEE76AF1EE10FA9FED126A15DDF2EE8E
:105C6000047A66EEA76A436AC6EE267A0133436277
:105C70000023F7EE006A76EEE76A27EE800AA7EEC9
:105C8000260A80ED080A18467047F0EE467A01238E
:105C9000EFE70023F7E700BFFFFF7F7F000000343E
:105CA00000004843CDCCCC3D90F83C35934207D919
:105CB00000EB8200D0F8140510B103689B6A184706
:105CC000002070472DE9F34105466E4686E80C003A
:105CD000134B45F8043B04460F4600F5C8782846A8
:105CE0002C3500F017FCA845F9D196E8030004F51F
:105CF000A863C4F8387583E80300089BC4F84835E6
:105D0000084920462EF0CCFA074B1A6812B1074812
:105D100053F022F820461C6002B0BDE8F08100BFBD
:105D200008350908D03309083C5E002034330908DF
:105D30002DE9F04F90F83C6585B00446002E55D112
:105D40007F2380F84C350DF10F01042328308DF8A6
:105D50000F302FF07DF804F5C87504F21458271D94
:105D60005FFA86F91822FF21284674F0D3FA85F8E5
:105D7000589097F924A0BAF10A0F4DD039DCBAF146
:105D8000040F0FDCBAF1020F0FDD442000F0DCFF3E
:105D9000834620B13B462A46214654F083FFC8F88B
:105DA00000B002E0BAF1090F2AD0D8F8000050B1D3
:105DB000296EC5F85CA031B1244B43F826102EF0B3
:105DC0007DFC2EF073FC58F8040B09F101095FFA11
:105DD00089F920B103689B68984784F83C9501369F
:105DE000092E05F1640507F12C07B9D105B0BDE80E
:105DF000F08FBAF1190F1DD0BAF11F0FC5D0D4E73B
:105E0000382000F0A1FF83460028C8D03B462A4630
:105E1000214655F0BFFBC2E7302000F095FF8346D6
:105E20000028BCD0CDF800903B462A46214655F0CC
:105E30004BFDB4E7482000F087FF83460028AED032
:105E40003B462A46214655F0B1FDA8E7405E0020BA
:105E500090F83C358B4283BF642303FB010090F82C
:105E6000D50100207047000090F83C358B4283BF7D
:105E7000642303FB010090ED6A0A9FED010A70475D
:105E80000000000090F83C358B4206D900EB810001
:105E9000D0F8140508B155F0B7B89FED010A704766
:105EA0000000000010B490F83C458C420A4614D91A
:105EB00000EB8104D4F814457CB1E468246A6406DC
:105EC00003D55DF8044BFFF7DDBF642101FB02033E
:105ED00093ED6A0A5DF8044B70479FED010AF9E7FC
:105EE0000000000090F83C358B420BD900EB81009C
:105EF000D0F8140538B1C3681B6A1A4214BF0120D8
:105F0000002070470020704770B590F83C359342F0
:105F100004460E46154601D8002070BD00EB8203F2
:105F2000D3F814050028F7D003689B699847002828
:105F3000F2D0642202FB0544D4F8AC313360ECE7C4
:105F400070B590F83C35934204460E46154601D88C
:105F5000002070BD00EB8203D3F814050028F7D0B1
:105F600003689B6998470028F2D0642202FB05442D
:105F7000D4ED6C7AF4EE677AF1EE10FAE8D6C6ED5D
:105F8000007AE6E770B590F83C35934204460E4639
:105F9000154601D8002070BD00EB8203D3F814052C
:105FA0000028F7D003685B6998470028F2D0642284
:105FB00002FB0544D4F8B4313360ECE790F83C358B
:105FC00093420ED900EB8203D3F814355BB16423FE
:105FD00003FB020292F8E40130B1D2F8E0310B6029
:105FE00070470020704718467047000008299DBF81
:105FF0002C2303FB01004068002070472DE9F04F7F
:106000004B4B2DED028B1B68DB6A93F89C3089B0FB
:106010000446002B00F08680DFF82CB19FED458A06
:106020004FF0000994F83C355FFA89F5AB4279D915
:1060300004EB8503D3F8140500285DD003685B6B7F
:106040009847642303FB0543074693F8D431834202
:1060500052D2032861D8DFE800F04F025259364E81
:106060004FF000083BF0EEFE94F83C25AA4284BFB6
:10607000642202FB05424FF0640105F1010301FBBC
:1060800005458CBFD2F8A82118EE102A8246D5F813
:10609000B001CDE90632F6F72FFA079ACDE90401EF
:1060A0001046F6F729FA069B0096CDE902015A46FA
:1060B0000421504636F094FD0123204A84F84D35E2
:1060C00085F8D471D372D4F848354BB3002255B259
:1060D0005957481C03D0414502F10102F7D194F908
:1060E0004C35AB4208DBD4F84435D4F84005424681
:1060F0003146984784F84C5509F1010992E72C2361
:1061000003FB05430E4E93F92B80ABE72C2303FBD7
:1061100005430C4E93F92C80A4E70026B046A1E776
:106120001D46DCE709B0BDEC028BBDE8F08F00BF77
:10613000105E00200000000061330908BD5E0020F1
:1061400092690A08583309087033090890F83C35F9
:106150008B4207D900EB8100D0F8140510B1036819
:10616000DB6918470020704708299CBF642303FBA4
:10617000010000F5C870704790F83C35934207D98C
:1061800000EB8200D0F8140510B103685B6A184771
:10619000002070472DE9F04F002493B005460E46CD
:1061A000174621462F2206A8059405F2145974F0CB
:1061B000B1F805F1280A4FF02C0B05F5F6730BFB2F
:1061C00004F259F8040B1AF90210E5B230B951B9CA
:1061D0000134092CF3D14FF0010813E0642262432B
:1061E0009A58914212D01548154B00680193013519
:1061F000EDB20095134BC06A324639460DF01EF9D8
:106200004FF00008404613B0BDE8F08F05A93322D7
:10621000039354F0DBFF039B804605A90028D7D1E8
:10622000064801910135EDB200680095054BC06A42
:10623000324639460DF002F9E4E700BF105E002057
:10624000F53E0908983309082DE9F04FDFF88090F2
:10625000DFF880A0DFF880B08DB00646002796F802
:106260003C35FCB2A3422ED9642505FB046595F8A4
:10627000DC3133B395F8DD1119BB4FF00108202252
:10628000444404A889F8198074F044F807EE904A51
:106290004AF21043F8EEE77A03AA4C21ADF8283011
:1062A00050462423CDED037A36F0ACFA3BF0CAFD1C
:1062B0009BF80030054A0094042136F091FC85F8E3
:1062C000DD810137CBE70DB0BDE8F08FA8330908B9
:1062D000BD5E002059610020CD2200202DE9F04F45
:1062E0002F4B1E6885B0044646B1D0F838153046AD
:1062F00032F0DEF910B1304631F086F852F05AFD36
:106300004FF0000801904FF02C0A4FF0640B94F806
:106310003C355FFA88F5AB4239D904EB8507D7F8ED
:10632000140588B30AFB05430BFB054993F92820A4
:10633000D9F8EC118A4227D132B30268D26890476B
:10634000D7F814050268126B904799F8D52112B15D
:10635000019BC9F8D831BEB1D4F83815304632F0B7
:10636000A7F988B152F02EFDCDE9021002460B4686
:10637000D7F81405294655F021F9DDE90232D7F89E
:106380001405294655F090F908F10108BFE72046A9
:10639000FFF734FE204605B0BDE8F04FFFF754BFCD
:1063A000D86000202DE9F0474FF000082DED028B5A
:1063B00004468946B0EE408A474601264FF0640AFB
:1063C00094F83C355FFA88F5AB421AD929FA05F3FF
:1063D000DB070AD504EB8503D3F8140578B103680D
:1063E000B0EE480A9B6B984706400AFB054508F14A
:1063F000010895F8D4319F4238BF1F46E0E70646B2
:10640000F3E727B97F23A4F84C35034BDF72BDECCB
:10641000028B3046BDE8F087BD5E002090F83C3529
:106420008B4207D900EB8100D0F8140510B1036846
:10643000DB6B1847002070470B46114690F83C254F
:106440009A4207D900EB8300D0F8140510B1036815
:106450001B6C18477047000070B504460E460025B7
:1064600094F83C35E9B28B4205D932462046FFF715
:10647000E3FF0135F4E770BD2DE9F84390F83C5592
:106480000246002400F128062C2700F5F6784FF08C
:106490006409E1B28D420FD907FB04F309FB04F054
:1064A000F35658F80000834209D11BB11046FFF79C
:1064B000CFFC10B10134ECE70120BDE8F8830020E7
:1064C000FBE7000010B590F83C258A42044617D936
:1064D000642202FB010393F8D431022B03D004D9C8
:1064E000032B18BF0023184610BDFFF797FF48B9CC
:1064F0002046FFF7C1FF00280CBF06230123F2E767
:106500000023F0E70623EEE7014B1868704700BF51
:106510003C5E002010B5034904462DF0C1FE204624
:1065200010BD00BF8835090810B50446203045F07D
:10653000C7FA044B04491C6020462DF0B1FE2046EA
:1065400010BD00BF645E002000370908F7B5B7EE44
:10655000000A0022022104462DF0A4FA204655F03C
:1065600075FA45F09BFB144B1D680646E86A036804
:106570005B6A98470B46022102460091304645F07F
:10658000B5FAB4F94A60002E14DDEF6A3B6838466C
:106590005B68B4B2984728B197F84D3013B1C92E53
:1065A000A8BFC824A86A03685B68214603B0BDE899
:1065B000F040184703B0F0BD105E002010B504464F
:1065C00055F012FA2046BDE8104055F03DBA0000E3
:1065D0002DE98048284BDFF8A490DFF8A4A0DFF86D
:1065E000A4B01446012293B005460E461A704FF02F
:1065F000000852F0DFFBD9F800300393A0EB08024B
:1066000041F287339A4207461FD9CDE900560398D5
:106610005346342205A9C06A0CF010FF214605A894
:10662000049451F097FDCDE9005603985B4634225F
:1066300005A9C06A0CF002FF04943BF003FC049B24
:1066400005AA022136F0B4FAB8463BF0FBFB3AF05B
:10665000F7FC3BF0F7FB3CF039FB0A2105A80CF0F6
:10666000D9FC039B986A036805215B68984705A8D5
:106670000CF0DCFCBDE700BF685E0020105E00206F
:1066800078360908F97C0A080FB400B595B016AA47
:10669000002152F8043B039205A83C220193049187
:1066A00073F038FE054A019B402104A851F0FAFC22
:1066B000039A034804A9FFF78BFF00BF803609083F
:1066C000963609080FB407B504AA034852F8041B0C
:1066D0000192FFF77DFF00BFA8360908014B18683B
:1066E000704700BF645E002008B50449102273F0B3
:1066F000B7FDB0FA80F0400908BD00BF6C5E002015
:106700001022002173F006BE0378416023F00D03D0
:10671000022A037008D0032A0AD0012A03D1DBB26F
:1067200043F0010303707047037843F00803F9E76F
:10673000037823F0050343F00503F3E773B504463C
:106740000E4615460193FFF7DBFF2046C4E90265BC
:10675000069A0199FFF7D8FF02B070BD4B684360FD
:106760000A78037862F3000303700B780278C3F3AE
:10677000800363F3820202700B78D2B2C3F3C003CA
:1067800063F3C302027070470078420704D4030722
:1067900004D400F0010070470320704702207047C6
:1067A000F0B585B005461646FFF7EEFF88420F4666
:1067B00005D16B6833600124204605B0F0BD032885
:1067C00001D10024F8E70329FBD001280BD00228CF
:1067D00016D018BB6D68012F22D0022F2ED0002FAB
:1067E000EFD13560E7E7FCF751FC90F89432DB0716
:1067F000E7D56D68FCF74AFCD0F888321D44EAE71B
:106800006846FFF77DFFFCF741FC6946FCF722FA7A
:1068100004460028D0D06D68019BEFE70025DAE739
:10682000FCF734FC90F8944214F00104C9D0FCF752
:106830002DFCD0F88832ED1A3560BDE76846FFF7C9
:106840005FFFFCF723FC6946FCF704FA04460028C6
:10685000B2D0019BEFE7000073B501AA05460E46D2
:10686000FFF79EFF044620B1019932462846FFF704
:106870004BFF204602B070BD13B5144601AAFFF7C6
:106880008FFF48B1DDED017A9FED047AF8EEE77AEB
:1068900067EE877AC4ED007A02B010BD0AD7233CB8
:1068A00007EE900A9FED090AF8EEE77A08B527EEA1
:1068B000800A71F04FF9DFED067AB4EEE70AF1EEE7
:1068C00010FAD8BFB0EE670A08BD00BF50E0EF3045
:1068D0000AD7233C10B50446806811F083F820B134
:1068E000E068BDE8104011F091B810BD73B585683F
:1068F00004460E461DBBC36823B98B688360CB6812
:10690000C3600125636873B92378DB070BD5204684
:10691000FFF73AFF01AA01463046FFF741FF10B1E9
:10692000019B636005462046FFF7D4FF20B9B3689A
:10693000A360F368E3600125284602B070BD00251E
:10694000E0E700000D4B83424FF000038B4106DA75
:1069500000F1255000F5311000F5E0507047084B6C
:1069600098424FF0FF3371EB0303BEBF00F1564076
:1069700000F5130000F52440704700BF00D2496BBA
:10698000002EB69490EA010F01D4401A7047C31745
:10699000401A63EBE1710D4B83424FF000038B41D2
:1069A00006DA00F1255000F5311000F5E05070478F
:1069B000074B98424FF0FF3371EB0303BEBF00F16A
:1069C000564000F5130000F52440704700D2496B93
:1069D000002EB69470B52DED028B84B00446684647
:1069E0000D46FFF78DFEFCF751FB6946FCF732F9C7
:1069F000064608B3A368029ADFED128A03999B1A30
:106A000007EE903AF8EEE77A67EEA87AC5ED007ADD
:106A1000E068FFF7B7FF08EE100AA068024402EB37
:106A2000D272B8EEC88A5010FFF73AFF28EE288AD3
:106A300028EE000A85ED010A304604B0BDEC028B59
:106A400070BD00BFF67C8E3F37B500230C4601AA0F
:106A5000022105460193FFF7A3FE10B9002003B001
:106A600030BD21462846FFF7B5FF0028F6D0DDED02
:106A7000017AF8EEE77AC4ED027AF0E710B52DED71
:106A8000028B84688A680B46111B08EE901AC16855
:106A9000D868FFF777FF224402EBD27208EE100AA3
:106AA0005010FFF7FDFEB8EEC88AF8EEE88A28EE2F
:106AB000000A20EE000AA8EEA80ABDEC028BB1EE97
:106AC000C07A9FED020A27EE000A10BD8262363CB2
:106AD000F0B52DED028B0D4689B08C680646D0E9E5
:106AE0000271E868FFF74EFF08EE100AE01900EBAC
:106AF000D0704010FFF7D4FE73686A689FED0E1ADD
:106B00009B1A07EE903AE41BB8EEE77AF0EE400AE3
:106B100007EE904A9FED090AB8EEC88AF8EEE77AC8
:106B200028EE008A27EE011A27EE800A68EE200A76
:106B300009B0BDEC028BF0BD0AD7233C8262363C23
:106B400084B004B0FFF7C4BF38B52DED028B0C46FE
:106B50000246C168E068FFF715FF9568A46808EE73
:106B6000100A601900EBD0704010641BFFF798FE0C
:106B700007EE904AF8EEE77AF8EEC80A87EE807AD8
:106B8000BDEEC70A10EE103A5B4200EE103AB8EEC6
:106B9000C00A71F001FADFED087A30EE270ABDEC89
:106BA000028BB5EEC00AF1EE10FA44BFDFED037AB6
:106BB00030EE270A38BD00BFDB0FC93FDB0FC940ED
:106BC00030B52DED028B0B4685B08C68D0E90251B3
:106BD000D868FFF7D7FE08EE100A601900EBD070F6
:106BE0004010FFF75DFE641B07EE904AF0EE400A8E
:106BF000B8EEC88A9FED060AF8EEE77A28EE008A1A
:106C000027EE800A68EE200A05B0BDEC028B30BD8D
:106C10008262363C82B002B0FFF7D2BFF0B52DEDF4
:106C2000028B0B468F68D0E9025185B0D868FFF718
:106C3000A9FE7B1903EBD37304465810FFF730FE0F
:106C4000781B10EE106AF5F745FC14A3D3E9002376
:106C5000F5F7AAFCF5F7A0FF08EE100A2046F5F7B5
:106C600039FC0EA3D3E90023F5F79EFC0446304619
:106C70000D46F5F741FC02460B4620462946F5F73E
:106C800093FCF5F789FF00EE900AB0EE480A05B0D4
:106C9000BDEC028BF0BD00BFAFF3008000000040F0
:106CA00050CC863F094B984206DDC0F1D64000F536
:106CB000930000F5A4407047054B9842BEBFC0F159
:106CC000144000F5360000F53850704700E9A4354F
:106CD00000175BCAF8B52DED028BDFED148A07684B
:106CE00020EE280A0646FDEEC07A0D4617EE904AC1
:106CF00004EBD47007EB6000B0EE608AFFF7D0FDC4
:106D000028EE288A3819C8EE007AFFF7CBFF3060EA
:106D100017EE900AF6F71AF92B68C01841EBE371E9
:106D2000FFF710FEBDEC028B2860F8BD02AAB3424B
:106D300000F10C010830FFF7CDBF00000148FFF75C
:106D4000DFBC00BF6C5E00200121884238BF0846CE
:106D50006EF034BFFFF7F8BF08B16EF033BF704775
:106D6000FFF7FABFF8B506460F46144622B96EF093
:106D700029FF25462846F8BD10461EB9BDE8F84053
:106D80006EF0ECBE6EF0EAFE05460028F2D0BC4282
:106D90002246314628BF3A4673F072FA30466EF00A
:106DA00011FFE7E737B504460846089D11461A4625
:106DB000036801959DF81C5000951D68069BA84727
:106DC0002060204603B030BD00214FF0FF3310B5E6
:106DD00000220363044601600171C0F8051041728E
:106DE00080F8251000F13C0300F50B70D9709A6013
:106DF000DA601A615A619A61DA611A625A629A62B9
:106E0000DA631A645A649A64DA641A655A659A6590
:106E1000DA65DA661A675A677C339842E6D121460A
:106E200004F5167006F0FCFD044B1A6822B90449FB
:106E30001C6020462DF034FA204610BD7C5E0020F8
:106E40006839090873B5D0F83C320191994204467B
:106E500013D0D0F84032994218D0D0F844328B4247
:106E600016D102200AE0D4F8343253B3D4F83832C1
:106E70004BB34FF0030002B070BD002094F82230F5
:106E80008342F8D8431C84F82230F4E70120F5E768
:106E9000D0F83062002EE6D194F841233546B60092
:106EA0009AB1A319C3F83012A319019AC3F83C226E
:106EB00094F82230AB429CBF6B1C84F822302846E9
:106EC000D9E70126E8E70226E6E704F50C7001A9F8
:106ED00030442EF08FF8E7E738B504460D462DF024
:106EE000FFFF291D201D2DF0FBFF05F1080104F116
:106EF00008002EF0CFF805F1140104F114002EF073
:106F0000C9F805F1200104F120002EF0C3F805F1C5
:106F10002C0104F12C002DF077FF05F1300104F174
:106F200030002EF07FF805F13C0104F13C002EF01A
:106F3000B1F8AB6BA3636B6B636338BD2DE9F043B2
:106F4000A1B00023002500F13C0706468DF807504C
:106F500003930493059306930793089309930A9365
:106F60000B931093119312931393149315931693F9
:106F7000179318931C931D931E9300F50F78B94631
:106F800058F8043BF3B1F26E934223D0D6F8E820D0
:106F9000934221D0D6F86421934213D10221EBB25F
:106FA00099420FD0C1EB411109EB8104214601A8A0
:106FB000FFF792FF39462046FFF78EFF01A93846BA
:106FC000FFF78AFF0135032D07F17C07D8D121B0E7
:106FD000BDE8F0830021E2E70121E0E72DE9F04779
:106FE00004460E461546804607464FF0000A3146D5
:106FF0002046FFF727FF7A6FB2425FFA8AF90ED177
:10700000C3B2022B0BD87C2202FB0A44012084F875
:107010003E0084F83F3085F80090BDE8F0870AF123
:10702000010ABAF1030F07F17C07E0D100273146CE
:107030002046FFF707FFD8F86C205FFA87F912B9EE
:10704000C3B2022B19D90137032F08F17C08EED106
:1070500031462046FFF7F6FEC2B2C2EB421304EB04
:10706000830393F83E7067B9022A0BD8012083F896
:107070003E0083F83F202A70CFE77C2000FB0744C6
:10708000C4E700274FF07C0904F13E0A3146204650
:10709000FFF7D8FE034609FB07F05FFA87F81AF8F6
:1070A000002012B9DBB2022B09D90137032FEDD131
:1070B00094F8230004280BD9144851F04DFE0444E1
:1070C000012084F83E0084F83F3085F80080A4E772
:1070D00004F54377002157F8043BB342CAB208D104
:1070E000904202D8531C84F8233003322A700020C7
:1070F00093E73BB9411C04EB800084F82310C0F8EF
:107100000C63F2E701310529E5D1F0E7A037090862
:10711000C9B200EB8101D1F83C3253B1026F934206
:107120000AD0D0F8EC20934208D0D0F868219342DE
:1071300006D04FF0030070470020704701207047D1
:10714000022070472DE9F8430F469146044600F5AA
:10715000BA7894F83E5035B97C344445F9D10025CD
:107160002846BDE8F88300234A46394601200BF043
:10717000E7FD00210646E06E0BF0F2FD8642EBD102
:10718000EEE70000012303FA01F1D0F808331942B9
:107190000AD14AB190F82030032B1FBF591C80F848
:1071A000201000EB83004261704700002DE9F0439E
:1071B000DFF87C8085B0044600F50F7600257C273B
:1071C000B14656F80C3CD9F800209342E9B206F1DA
:1071D000040619D1C3B12046FFF79AFFC0B207FBDE
:1071E000004090F83E307BB903A9A9F10C0003934D
:1071F0002DF000FF3AF026FE56F8043C009342467C
:107200002B46012135F0ECFC0135032DD8D104F1DA
:107210006C0504F5F074296821B9AB6813B12846F0
:107220002CF03AF97C35A542F5D105B0BDE8F083E4
:10723000BC37090838B504461546FFF769FFC0B2E8
:10724000022808D87C2303FB004029465030BDE8C3
:1072500038402DF00FBF38BD38B504461546FFF74E
:1072600057FFC0B2022808D87C2303FB0040294600
:107270005C30BDE838402DF0FDBE38BD37B50D4659
:1072800004468DED010AFFF743FF022D07D8C0B277
:107290007C2303FB004001A968302DF09DFD03B065
:1072A00030BD000038B50546FFF732FFC4B2022CEE
:1072B00013D8C4EB4414A4003C3504F1080028445E
:1072C00000212CF0E9F804F1340104F130002944E4
:1072D0002844BDE838402DF08DBE38BD70B5054658
:1072E0000E461446FFF714FFC3B2022B0DD87C20C4
:1072F00000FB035394E80700443383E8070031465A
:107300002846BDE87040FFF7CDBF70BD37B50446D5
:107310001546FFF7FDFEC0B2022809D87C2303FB07
:1073200000400DF1070140308DF807502DF0D8FDD9
:1073300003B030BD1FB590F92C30044623B390F94B
:1073400021300BB36846FFF7DBF9FBF79FFE694678
:10735000FBF750FCC0B1DDED037A9FED0C0AF8EEAF
:10736000E70ADDED027AF8EEE77A0123C0EE800A43
:1073700084F83D3387EE800A06F0A4FDDFED047A41
:1073800020EE270A84ED0A0A04B010BD8096184B3F
:1073900035FA8E3C024690F9210058B192F840032C
:1073A00040B1114491F92C0220B192F92400033824
:1073B00018BF01207047000038B590F8223005460C
:1073C0005BB100242346E1B22846FFF7E3FF08B192
:1073D0000133DBB20134032CF5D1184638BD00006F
:1073E00090ED0A0A7047000038B50C46D1ED066AE8
:1073F00011460546FFF78CFEC3B27C2000FB035309
:10740000D4ED087AD3ED260A94ED076AD3ED255A18
:1074100093ED245A26EE600A67EEA00AA5EEA70AAD
:10742000F0EE607AE5EE867AB7EE007AA6EEE67ABE
:1074300067EEE60AB1EE400AE5EE070A70F0ACFD31
:107440009FED071ADFED070A40F6580010F020F90B
:10745000D5ED0A7ABDE8384030EE270A10F004B9BD
:10746000DB0F4940DB0F49C02DE9F04190F8223095
:107470008B4204460D4602D20020BDE8F081FFF7A2
:1074800047FEC0B204F13C06C0EB401006EB8000A2
:10749000083012F089FDDFED157AB0EEC00AB4EEC7
:1074A000E70AF1EE10FAE7D429462046FFF730FE4E
:1074B000C5B27C2000FB05473B6F002BDCD0032DC1
:1074C000DAD000FB05603030D7F86C802CF0BEFFBE
:1074D000D7E91B32934201D1984505D07C2000FBAF
:1074E0000544C4F86C80C7E70120C6E700000034FB
:1074F0002DE9F74F04460E46174600F50F7A4FF078
:10750000000B5AF8049B5FFA8BF8B9F1000F26D0F4
:1075100041462046FFF73EFF08B341462046FFF7AD
:10752000F7FD7C23C0B203FB004090F83E505DB9EC
:1075300008F101031B4ADBB23946304650F0B2FD78
:10754000284603B0BDE8F08F5AF8102C914506D0BC
:10755000154A3946304650F0A5FD0025F0E70BF1FD
:10756000010BBBF1030FCCD14FF0000894F822308F
:107570005FFA88F18B420DD920460191FFF774FF25
:10758000054620B901992046FFF704FF20B908F10C
:107590000108EBE70125D3E7044A3946304650F0AD
:1075A00081FDCDE7E4370908F93709081E380908D5
:1075B0002DE9F0412DED048B90F842139FED348AB4
:1075C000DFED348A9FED349A82B00646FFF7A0FDC6
:1075D00006F13C07C5B27C2000FB057554354FF021
:1075E000000896F822205FFA88F39A424ED919468D
:1075F0003046FFF7CFFE10B908F10108F1E7194650
:107600003046FFF785FDC4B27C2000FB0474D4ED46
:10761000157AF0EEE77AF4EEC87AF1EE10FA04F19A
:1076200054040ED5D4ED017AF0EEE77AF4EEC87A80
:10763000F1EE10FA05D5002002B0BDEC048BBDE8D8
:10764000F0812946204612F0BFFCB4EEE80AF1EEC4
:1076500010FAF0DC2946204611F0B4FFB4EEC90A56
:10766000F1EE10FAE7DC2146284611F0F3FE6846F9
:107670008DED000ACDED010A11F098FFDFED077ADC
:10768000B4EEE70AF1EE10FAB6DDD4E70120D3E755
:1076900000000034DB0FC93F920A863F00004843D8
:1076A000022910B5044608D8FFF732FD7C23C0B28A
:1076B00003FB004494F83D0010BD0020FCE70000EF
:1076C00013B590F8421301910446FFF7E9FF30B17A
:1076D0000199204602B0BDE81040FFF75BBE02B042
:1076E00010BD0000F7B590F921500446002D73D06D
:1076F00090F84053002D6FD090F84213FFF7D0FF61
:1077000094F83D33064613B92046FFF713FE0025D3
:1077100094F82020EBB29A4207D904EB8303013599
:10772000586903689B689847F2E751F043FB0027CC
:10773000224604F5BA7140F2F315D2F89C30C31A10
:10774000AB428CBF0023012382F83D307C32914252
:1077500047EA0307F1D194F92430032B07D194F8B9
:107760003C33002B3BD0D4F83803002849D167B113
:10777000236B013309D030F0D1FF216B30F098FF3B
:1077800018B130F0CBFF2FF053FF94F92C32002BBF
:107790003AD194F92D32CBBB94F92E3213B1022396
:1077A00084F8423394F842132046FFF779FF86426B
:1077B000054611D030F0B2FF4FF6FF7130F078FF80
:1077C00050B1002D14BF00220422019230F0A6FF18
:1077D000019A032130F0FEFE284603B0F0BD0123DC
:1077E00084F83C330420FFF7AFFA054610B1214678
:1077F00006F0B6F994F92430C4F83853032BB2D00C
:10780000B5E706F0C7F9B2E70023C9E70123C7E7E8
:1078100038B590F921300446D3B190F84053BDB14A
:10782000FFF776FCC0B2022812D87C2303FB004489
:10783000D4ED1A7A9FED087AF4EEC77AF1EE10FAD9
:1078400006D4B7EE087AF4EEC77AF1EE10FA00DD4E
:107850000025284638BD00BFABAA2A3F70B5D0F836
:10786000085315F4003504460E460DD190F8403308
:107870005BB90A78072A07D8012303FA02F290F8C5
:107880003F33134380F83F3370BD94F82020EBB2B0
:107890009A42F9D904EB8303314658690368DB68DF
:1078A00098470135F1E7000038B505466C242B599F
:1078B0001BB1002128192BF0EFFD7C34B4F5F07FCB
:1078C000F5D138BD014B1868704700BF7C5E0020C1
:1078D00010B50446006810B103685B6898472046FD
:1078E00010BD000010B50446006810B103685B6865
:1078F0009847204610BD00002DE9F04FD0F80853FE
:107900008DB015F4807B9DF858909DF85CA00446DE
:107910000F461646984660D1FFF714FC054600282E
:107920003FD0CDE906BB069B04934FF0000B4246C7
:1079300039462046CDE905BBFFF704FC0646002882
:107940003DD0CDE90ABB0A9A089200234A4608A90D
:10795000CDE9093304A8534600F042FF074608A8C2
:10796000FFF7C0FF09A8FFF7BDFF0AA8FFF7B0FFA8
:1079700016B10BA8FFF7ACFF04A8FFF7B3FF05A8EB
:10798000FFF7B0FF06A8FFF7A3FF15B107A8FFF7A1
:107990009FFF3A46082120460DB0BDE8F04FFFF7A3
:1079A000F1BB04230E49CDE9010309680D4B009397
:1079B000496833463A4606A8FFF7F4F9B3E70423CB
:1079C0000749CDE901030968064B0093496843461E
:1079D0003A460AA8FFF7E6F9B5E70DB0BDE8F08F23
:1079E000105E0020801A06002DE9F04F9146012418
:1079F000D0F808238BB08C40144098469DF854A0D2
:107A00009DF850309DF858B006460F4635D11A46BD
:107A100041460593FFF796FB059B054600B3CDE96C
:107A20000844089A069200235A46514606A8CDE912
:107A30000733C847044606A8FFF754FF07A8FFF717
:107A400051FF08A8FFF744FF15B109A8FFF740FF51
:107A50002246394630460BB0BDE8F04FFFF792BBE7
:107A600004220749CDE901020968064A00924968E3
:107A7000424608A8FFF796F9D3E70BB0BDE8F08FB0
:107A8000105E0020801A06002DE9F04FB04BDFF8A1
:107A9000CC921D6804466868036889B09B68984763
:107AA000002607464FF001084FF0080A08FA06F3CF
:107AB0003B4240F02D820136202EF7D16868DFF876
:107AC0009CA20368DB689847002607464FF001092F
:107AD0004FF0060809FA06F33B4240F02B820136CC
:107AE000202EF7D16868DFF8789203689B68984782
:107AF000002607464FF001084FF0080A08FA06F37F
:107B00003B4240F028820136202EF7D16868036896
:107B10009B6898470026804601274FF01A0907FA0C
:107B200006F313EA080F40F026820136202EF6D124
:107B300068680368DB689847002607464FF0010A2B
:107B40004FF01A09B0460AFA06F33B4240F02E8283
:107B50000136202EF7D16868DFF808920368DB68E9
:107B60009847002607464FF0010AB0460AFA06F386
:107B70003B4240F036820136202EF7D16868DFF8AC
:107B8000E4910368DB689847002607464FF0010A36
:107B9000B0460AFA06F33B4240F033820136202E0B
:107BA000F7D16868DFF8BC9103689B6898470026A6
:107BB00007464FF001084FF0020A08FA06F33B426D
:107BC00040F02F820136202EF7D16868DFF89491BB
:107BD00003689B689847002607464FF001084FF05E
:107BE000020A08FA06F33B4240F02B820136202EAF
:107BF000F7D16868DFF8709103689B6898470026A2
:107C000007464FF001084FF0060A08FA06F33B4218
:107C100040F02E820136202EF7D16868DFF84891B7
:107C20000368DB689847002607464FF0010AB04614
:107C30000AFA06F33B4240F02B820136202EF7D1A0
:107C4000444BDFF82891079307AF04264FF00C0A46
:107C5000686803689B6898474FF0000805904FF0EC
:107C6000010B059A0BFA08F3134240F0218208F148
:107C70000108B8F1200FF4D168680368DB68984701
:107C80004FF0000805904FF0010B059A0BFA08F32E
:107C9000134240F01E8208F10108B8F1200FF4D120
:107CA000013E16F0FF0607F10107D1D16868DFF841
:107CB000C0A003689B6898474FF001080746B1468B
:107CC00008FA06F33B4240F017820136202EF7D126
:107CD0006868DFF89CA00368DB68984700260746C1
:107CE0004FF00109B04609FA06F33B4240F0148216
:107CF0000136202EF7D16868DFF878A003689B680A
:107D00009847002607464FF00108B14608FA06F3E7
:107D10003B4240F011820136202EF7D16868DFF82F
:107D200054A00368DB689847002607464FF0010916
:107D3000B04609FA06F33B4240F00E820136202E8F
:107D4000F7D16868044B079303689B68984713E072
:107D5000105E00200C0D0E0F20212223D1AA010855
:107D6000F1BA010851B201086D8701081DB0010880
:107D700035AD0108C5B70108BA4A804600264FF064
:107D8000010909FA06F313EA080F1AD00DF11C0ACB
:107D90000427F3B24FF0000B1AF8011B0091CDE954
:107DA000019B102120460593FFF71EFE94F8231037
:107DB000052900F0BC80013F17F0FF07A94A059B89
:107DC000EAD10136202EDCD168680368DB68984769
:107DD000A44A804600264FF0010B0BFA06F313EA83
:107DE000080F1AD00DF11C090427F3B24FF0000A56
:107DF00019F8011B0091CDE901AA10212046059335
:107E0000FFF7F2FD94F82310052900F09080013F60
:107E100017F0FF07934A059BEAD10136202EDCD1EB
:107E20006868DFF848A203689B6898470027804687
:107E30004FF0010909FA07F313EA080F15D01026CD
:107E4000FBB24FF0000B5246CDE9019B0096032197
:107E500020460593FFF7C8FD94F82320052A66D035
:107E60000136F6B2142E059BEDD10137202FE1D15A
:107E70006868DFF8F4A103689B689847002780468C
:107E80004FF0010909FA07F313EA080F15D0142679
:107E9000FBB24FF0000B5246CDE9019B0096152135
:107EA00020460593FFF7A0FD94F82320052A3ED035
:107EB0000136F6B2182E059BEDD10137202FE1D106
:107EC0006868694E0368DB689847002780464FF072
:107ED000010A0AFA07F313EA080F15D014255FFA0E
:107EE00087FB4FF000095B46CDE9019900953246CA
:107EF00015212046FFF778FD94F82330052B16D086
:107F00000135EDB2182DEED10137202FE1D10EE071
:107F10001E230093CDE9018AF3B24A460021204690
:107F2000FFF762FD94F82330052B7FF4C4AD09B050
:107F3000BDE8F08F1E230021CDE90031CDF8088087
:107F4000F3B252462046FFF74FFD94F82330052B3D
:107F50007FF4C5ADEBE70D230093CDE9018AF3B2C1
:107F60004A460C212046FFF73FFD94F82330052BAD
:107F70007FF4C9ADDBE7F1B26923CDE900790C22CA
:107F800020460591FFF7B8FC94F82330052BCED09E
:107F90006823CDE9007905990C222046FFF7ACFC57
:107FA00094F82330052B7FF4C0ADC0E7F1B269230C
:107FB000CDE900890C2220460591FFF79DFC94F83D
:107FC0002330052BB3D06823CDE9008905990C2215
:107FD0002046FFF791FC94F82330052B7FF4B8ADD1
:107FE000A5E71C230093CDE90188F3B24A46052199
:107FF0002046FFF7F9FC94F82330052B7FF4BBAD46
:1080000095E71E230093CDE90188F3B24A46052186
:108010002046FFF7E9FC94F82330052B7FF4BEAD32
:1080200085E71C230093CDE9018AF3B24A46052176
:108030002046FFF7D9FC94F82330052B7FF4C2AD1E
:1080400075E71E230093CDE9018AF3B24A46052164
:108050002046FFF7C9FC94F82330052B7FF4C6AD0A
:1080600065E700BF45BE01088D940108B18C010889
:108070000C230093CDE9018AF3B24A46062120463B
:10808000FFF7B2FC94F82330052B7FF4C3AD4EE725
:108090000C230093CDE90188F3B24A46062120461D
:1080A000FFF7A2FC94F82330052B7FF4C6AD3EE722
:1080B000CDE901BA3B7800934A465FFA88F307217D
:1080C0002046FFF791FC94F82330052B7FF4CFADC9
:1080D0002DE70023CDF808A001933B7800934A4692
:1080E0005FFA88F307212046FFF77EFC94F82330DF
:1080F000052B7FF4D0AD1AE70C230093CDE901895D
:10810000F3B252460F212046FFF76EFC94F823305D
:10811000052B7FF4DAAD0AE70C230093CDE9018843
:10812000F3B252460F212046FFF75EFC94F823304D
:10813000052B7FF4DDADFAE630230093CDE901890C
:10814000F3B2524609212046FFF74EFC94F8233043
:10815000052B7FF4E0ADEAE630230093CDE90188FA
:10816000F3B2524609212046FFF73EFC94F8233033
:10817000052B7FF4E3ADDAE670B50446FFF784FC27
:1081800094F82330052B29D0002594F83F33EB4099
:10819000DB07E8B215D40135082DF6D194F8233069
:1081A000052B1BD094F8203013B194F82230ABB9D2
:1081B0000B4B0C491B6898690368BDE870401B684D
:1081C000184703F087FB02460028E4D0112120461F
:1081D000FEF7D8FF94F82330052BDCD170BD00BF2B
:1081E000105E0020383809082DE9F04F90F9213051
:1081F00089B00446002B00F00481012300F50C75C2
:1082000080F84133024600F50F712B462E46D06EA2
:10821000002859D0002384F8413394F94030642B6E
:108220005BD094F9BC30642B00F08D8094F9383128
:10823000642B00F08A80D4F830722FBB01A920464D
:108240002BF00EF900B30C230593012306978DF84C
:108250001830714B07936946BDF80430049704A8A1
:10826000ADF810308DF800702BF07CFA9DF90010FD
:1082700051B1022908DC38B1C9B27C2303FB0141AA
:108280006C3128462CF0CEFE94F841B3BBF1000FC0
:108290005DD0E36E6367D4F8E830C4F8F030D4F80A
:1082A0006431C4F86C3194F8233003F1C30204EB59
:1082B00082020021042B7CD852F8040B1061013398
:1082C00042F8041CDBB2F5E753F8040B0028A1D1F7
:1082D0008B4202F17C029AD19FE7002066238DF841
:1082E00010307C2303FB004004A940302CF0DEFD5D
:1082F00004A920462BF0B4F800289CD004238DF864
:1083000018300023CDE901330393312305936946E7
:1083100004A82BF027FA059B28B108AA02EB8302D8
:10832000009942F8E01C0133332B0593EFD94EF04E
:10833000D3FA9DED031ADDED020A9DED010A6621D7
:108340004EF088FA77E70120C8E70220C6E7012748
:10835000A94655F8043B23B1AB600137042FF7D190
:1083600097E7AA46B8465FFA88F3022BF5D8DAF801
:10837000002055F8043C9A4205D104A95046CDF896
:1083800010B02CF04FFE5AF8043B08F101020BB973
:108390009046E8E704A906EB88000193CDF810B0F9
:1083A0002CF040FE019BAB6001A948462CF03AFE40
:1083B000D3E794F8413313B92046FEF7BFFD94F894
:1083C00022300BB3154B1B68986A036864215B6805
:1083D00098472046FFF786F994F83E3003B9E366E4
:1083E00094F8BA300BB9C4F8E83094F836310BB9C8
:1083F000C4F86431FAF74AFEFAF7B4FE0123A4F890
:10840000403309B0BDE8F08F2046FFF7B5FE94F881
:108410002230002BE0D0D5E710D50908105E0020EF
:10842000704700000120704701207047436898683A
:108430007047000010B5054B03600446C06A10B1D8
:1084400003685B689847204610BD00BFFC3C0908E4
:10845000406803689B6A184733B46C46406884E8F8
:108460000C000368DD6A94E80C00AC4602B030BC36
:108470006047000010B50446FFF7DCFF2046FEF71A
:108480006BFC204610BD000040680AF08BBB00006A
:10849000406801230AF086BB40680AF05FBB000019
:1084A00040680A220AF004BB40680AF019BB0000C9
:1084B00090F8313013B1002101F028B97047000065
:1084C00040680AF093BB000073B5044605250026FA
:1084D000E06A8DF8076003680DF10702DB6801218F
:1084E000984778B19DF807300C2B09D0102B05D098
:1084F000092B07D184F8333002B070BD1523F9E79A
:108500001423F7E7013DE3D12846F5E710B4C06A2C
:1085100003681C690822A44601235DF8044B31213D
:108520006047000010B4C06A03681C690122A446B9
:1085300000235DF8044B322160470000F7B5044684
:10854000C06A03685B6998470546002871D0E06AF5
:1085500003685B69984703689B689847E06A03680B
:108560009B69984760B9344B34491B689869036824
:108570001B6898472B682846DB689847002655E01B
:108580002046FFF7CFFF0028F4D02046FFF79CFFDE
:108590000028EFD0E06A03680121DB6A9847204693
:1085A000FFF7B4FF30B9244B25491B68986903686D
:1085B0001B68DEE7E06A0368DB69984730B91E4B49
:1085C00020491B68986903681B68D2E7E06A94F841
:1085D0003310012784F8317003685B6A9847E06ABA
:1085E00003689B6A98470146204601F0F1F8064669
:1085F0000028BFD094F830301BB13946204601F036
:10860000F7F894F83210204601F018F92B68284644
:10861000DB689847E06A009403681D6A0A4B01937F
:1086200002AB13E90C0042F21071A847304603B0C8
:10863000F0BD0646FAE700BF105E0020683C09085E
:108640008E3C0908AD3C09083D87010870B500253E
:1086500086B0CDE9005500230446C06A8DF8085065
:1086600005930393049303686A469E6810210923C7
:10867000B047A0B19DF8003013F0010615D194F871
:1086800034300133DBB2052B84F8343007D1204677
:10869000FFF748FF2046FFF739FF84F83460E06AAF
:1086A00003681B6B984706B070BD9DF8083084F8CE
:1086B00034501B07F3D4BDF901309FED1E6A06EE5E
:1086C000903ABDF9033007EE103ABDF90530F8EEE7
:1086D000E66A07EE903ACDED036AF0EEE66AB8EE90
:1086E000C77AF8EEE77AF4EEC66AF1EE10FA8DED8D
:1086F000047ACDED057A0DD5B0EEC77AB4EEC67A20
:10870000F1EE10FA06D5F0EEE77AF4EEC67AF1EE65
:1087100010FAC4D49FED080A03A811F09BF8B2EE3A
:10872000040A03A811F096F80A2203A9204601F0D2
:10873000EBF8B4E7000000349A99193EFFF786BFC2
:1087400010B5044B044640F8043BFFF7CBF8204635
:1087500010BD00BF143D090810B50446FFF7F0FF37
:108760002046FEF7F9FA204610BD0000F7B5036871
:108770000F4616461BB90024204603B0F0BD002466
:10878000046008200193FEF7DFFA054620B1124B82
:108790000360019B4360019401A8FFF7A3F8002D3B
:1087A000E9D03820FEF7D0FA04460028E3D000F0E4
:1087B000ADFE0A4BE562236084F8307084F83260C5
:1087C0002046FFF7BBFE05460028D5D1236820468A
:1087D0005B6898472C46CFE7143D0908FC3C090824
:1087E0002DE9F74F046806460D4690469946002C41
:1087F0006CD00B68002B49D0236820469B6A9847B1
:1088000003689B689847012328680DEB0302002149
:108810000AF0C8F998B39DF80130EA2B2FD1DFF8A0
:10882000F0B04FF0060A28680023802206210AF0E3
:1088300095F920B3DBF80070B86A03680A215B6819
:108840009847002328681A4606210AF087F9B0B134
:10885000B86A03680A215B689847012328680DEB12
:10886000030206210AF09EF948B19DF8014014F078
:1088700040042FD00AF1FF3A1AF0FF0AD3D1306832
:1088800003689B6A98470368DB68984700241DE0EB
:10889000022223460F2128680AF060F9B86A0368AB
:1088A00001215B689847306803689B6A98470368B2
:1088B000DB689847336834604A46414601A8019313
:1088C000FFF754FF044601A8FFF70CF8204603B059
:1088D000BDE8F08F224623460F2128680AF03EF9B2
:1088E000B86A036801215B68984702232146306813
:1088F0000DEB03020AF056F904460028C8D0B86907
:10890000024903681B689847B9E700BFD43C0908CF
:10891000105E0020002100F0F9BE000070B5044692
:108920008CB00426013E76B2731C4AD0E06A15234F
:108930006A465D210AF036F90028F3D0E06A152373
:1089400006AA5D210AF02EF905460028EAD0152274
:1089500006A9684671F084FC0028E3D19DF8003038
:1089600084F830309DF8073084F832309DF81430A8
:1089700084F83C309DF813309DF8102084F83D3089
:108980009DF80F3043EA0223E3879DF8013084F815
:1089900031309DF8083084F83330039B9DF80C206B
:1089A000C3F30F23A3869DF80B3043EA0223E3862B
:1089B000049BC3F30F232387019BC3F30F23638718
:1089C00007E0054B05491B68986903681B689847D1
:1089D000002528460CB070BD105E0020483D0908F7
:1089E0002DE9FF4104460023C06A8DF80730036873
:1089F000DFF850819B6A984703689B689847E06A54
:108A000003680A21DB6C9847E06A0A2204210AF015
:108A10004FF80425013D6DB26B1C32D000234B2171
:108A2000E06A82220AF09AF8D8F800600746B06A35
:108A3000036802215B689847002FEBD001231A4698
:108A40004B21E06A0AF08AF80746B06A03680221FF
:108A50005B689847002FDDD0E06A01230DF1070223
:108A600040210AF09FF80028D4D09DF80720322A30
:108A700010D0002DCED1B069304903681D68322373
:108A8000A847E06A03689B6A98470368DB689847D1
:108A900000254EE02046FFF741FF0028F1D0E06AB4
:108AA0000123172251210AF059F80028E9D0522257
:108AB000E06A012311460AF051F80028E1D0E06A8B
:108AC000012338224C210AF049F80028D9D0E06A65
:108AD00003689B6A98470368DB689847E06A05214A
:108AE00009F0FEFFE36A2046996800F071FE054632
:108AF000F8B194F84410204600F0A0FE94F84530F8
:108B00001BB10121204600F073FEE06A03680221D8
:108B1000DB6C9847E06A02940368DE6A084B0393B3
:108B200004AB13E90C0044F21B11B04750F042F9BA
:108B30002064284604B0BDE8F08100BF703D0908FC
:108B4000AD8C0108105E002070B5C58F90F93D60B6
:108B5000AD03B5FBF2F2A2F5804404FB04F2D5119B
:108B600090F83C200498D201624306FB0522521281
:108B7000A03002F58012424312134A43DB0003EB9C
:108B8000623000B270BD000010B5848E53005C43AB
:108B9000B0F93A30C91AC38FD31AB0F93820B0F9F6
:108BA0003600534304F500449B10C3EBC13300EB84
:108BB0002440044993FBF0F04FF400420EF096FD80
:108BC00000B210BD0080FFFF10B52DED028B8AB002
:108BD00004460823C06A05AA422109F0E3FF18B140
:108BE000BDF81A20D30719D4E06A09F0FFFF50F04E
:108BF000E1F8236CC31AFA2B0CD9206400238222DB
:108C00004B21E06A09F0AAFF0123E06A1A464B21D2
:108C100009F0A4FF0AB0BDEC028B10BDBDF9141021
:108C200094F932300093920894F930300392C910CD
:108C30002046FFF789FFBDF9161094F93330039AE7
:108C4000009308EE900A94F93130C9102046FFF7DE
:108C50007BFFBDF91810039A491008EE100A204650
:108C6000FFF792FF07EE900AF8EEE88AF8EEE77A4F
:108C7000B8EEC88AB3EE000A07A8CDED097ACDEDAB
:108C8000078A8DED088A10F0F9FDB2EE040A07A8F4
:108C900010F0E0FD50F08EF80A22206407A920466B
:108CA00000F032FEE06A09F0A1FFB3E7FFF78CBFE6
:108CB000F7B503680D4616461BB90024204603B0DD
:108CC000F0BD0027076048200193FEF73DF80446F9
:108CD00050B100F01BFC0D4B2360019BE362019738
:108CE00084F8446084F8455001A8FEF7FBFD002C91
:108CF000E3D02046FFF774FE05460028DED1236846
:108D000020465B6898472C46D8E700BFA83D090875
:108D100010B5044B044640F82C3BFEF7E3FD20461B
:108D200010BD00BFA83D090810B50446FFF7F0FFCD
:108D30002046FEF711F8204610BD0000002100F08B
:108D4000E5BC0000F8B504460D4617461E4600F087
:108D5000DDFB094B23602B68E362002200232A60BD
:108D600084F8307084F831606365A365E365236639
:108D70006366A3662046F8BDC03D0908F8B51C46E9
:108D800009331646DB086A46A2EBC30300AF9D46D3
:108D9000C06AA31C6A4609F005FF054628B12246B1
:108DA0000DF10201304671F06BFA2846BD46F8BD60
:108DB0002DE9F34106460F4614464FF0FBFF114BD9
:108DC000D3F800800546D8F82800036801215B68C5
:108DD000984701230DF1070207213046FFF7CEFF28
:108DE00060B19DF80730DA0702D4B7EB531F05D006
:108DF0004FF0E0FF431BA342E5D3002002B0BDE8E3
:108E0000F08100BF105E00202DE9F041DFF86082A4
:108E100092B0044602AF002646F02002E06A00232A
:108E2000D2B2502109F09AFE002800F00C810325EF
:108E3000013D6DB26A1C00F00681D8F80030986AD6
:108E400003684FF496719B68984701230DF1060261
:108E500055212046FFF792FF002800F0F4809DF88E
:108E6000063013F0E00F40F0EE80DB07E0D5022380
:108E70000DF1060252212046FFF780FF002800F086
:108E8000E280BDF8063001365BBA202E27F8023B9F
:108E9000C2D1BDF824309DF826109FED6D7ADFED2C
:108EA0006D6A9FED6D6A43F30B0207EE902A1B0972
:108EB00003F47063BDF82620F8EEE77A0B4343F322
:108EC0000B03C4ED0D7A07EE903A02F470639DF83F
:108ED0002820F8EEE77A134343F30B03C4ED0E7A30
:108EE00007EE903A9DF92230F8EEE77AC4ED0F7A5A
:108EF00007EE903A9DF92930F8EEE77A67EE877A27
:108F000007EE103AB8EEC77A9DF92A30C4ED107A10
:108F100027EE267ADFED517A84ED117A07EE103ACA
:108F2000B8EEC77A9DF92B30E7EE267AC4ED127AB7
:108F300007EE903AF8EEE77A9DF9233067EEA67ACD
:108F4000DFED476AC4ED137A07EE903A9DF92C30B5
:108F500007EE103AB8EEC77A9DF92E3027EE267A42
:108F6000F8EEE77A84ED157A67EE867A07EE103A26
:108F70009DF93030C4ED147A07EE903AF8EEE77AB6
:108F80009DF92D3067EEA67AB8EEC77AC4ED177A50
:108F900027EE267A07EE903A84ED167AF8EEE77A15
:108FA0009FED307A9DF92F3067EE877AC4ED187AFD
:108FB00007EE903A9DF93130F8EEE77A06EE903AF6
:108FC00067EE877AF8EEE66AC4ED197ADFED267A65
:108FD000BDF93830E6EE877A07EE103A9DF9323067
:108FE000C4ED1A7AB8EEC77AF3EE077AE7EE067A9E
:108FF00007EE103ADFED1D6AC4ED1B7AB8EEC77AB2
:1090000027EE267A84ED1C7A9DF9333007EE103A6C
:10901000B8EEC77A9DF9343027EE267A84ED1D7AB2
:1090200007EE103A9DF9353007EE903AB8EEC77A60
:10903000F8EEE77A27EE267A67EEA67A84ED1E7AB6
:10904000C4ED1F7A00E0002012B0BDE8F08100BF3F
:10905000CDCC4C3E0000803B0000003B0AD7233CB7
:109060000000003D0000803817B7D1B80AD7A33AF6
:10907000105E002073B501230E460DF10702062194
:109080000446FFF77BFE18B90025284602B070BDE4
:109090009DF80730013B012B0CD80023E06A1A46EB
:1090A000062109F05BFD0028EED0062200212046B3
:1090B000FFF77EFEE06A00233246062109F04EFDEE
:1090C00005460028E0D0262231462046FFF770FEF4
:1090D000DBE7000013B501230DF107020721044669
:1090E000FFF74CFE10B9002002B010BD9DF807300C
:1090F0001B070CD50023E06A1A46062109F02EFD55
:109100000028F0D0062200212046FFF751FEE06A39
:1091100000230722062109F021FD0028E3D01322B5
:1091200007212046FFF744FE0028DCD0E06A002338
:109130000522062109F012FD0028D4D017220521AE
:109140002046FFF735FE0028CDD001212046FFF74D
:1091500091FFC9E7F7B50446C06A544F03689B6A9C
:10916000984703689B689847E06A03680A21DB6CAC
:109170009847E06A0A22042109F09AFC0525013D7E
:109180006DB26B1C00F08980E06A0023B6227E215C
:1091900009F0E4FC0028F2D03B68986A03681821C3
:1091A0005B686E4698470123324600212046FFF750
:1091B000E5FD0028E3D09DF80030332BDFD12046B9
:1091C000FFF722FE002868D0E06A002380225021A9
:1091D00009F0C4FC002860D02046FFF77BFF002880
:1091E0005BD0E06A002386222E2109F0B7FC00281C
:1091F00053D0E06A00232422042109F0AFFC0028A8
:109200004BD0E06A00230222062109F0A7FC0028C7
:1092100043D0142202212046FFF7CAFDE06A002352
:109220000722052109F09AFC002836D001212046AA
:10923000FFF720FF002830D0E06A03680321DB6CD1
:109240009847E06A03689B6A98470368DB68984719
:10925000E06A172109F044FCE36A2046996800F0AF
:10926000B7FA0546B0B194F83110204600F0E6FA9E
:1092700094F830301BB10121204600F0B9FAE06AC1
:109280000368DF6A0A4B0094019396E80C0042F2EF
:109290001071B847284603B0F0BDE06A03689B6AC6
:1092A00098470368DB6898470025F3E7105E0020C5
:1092B0008994010810B586B00C236A463121044612
:1092C000FFF75CFD002800F0D5809DF80A309DF87E
:1092D00009209FED697A9FED696ADFED694A94ED97
:1092E000115A94ED1D4A94ED1E3A1B0403EB022320
:1092F0009DF80B2003EB02631B1207EE903AF8EE89
:10930000E77AF7EE006AA7EE876A9DF801309DF8CC
:109310000020D4ED147A94ED107A77EEA67A1B042F
:10932000A7EE867A03EB02239DF8022094ED0D6AE6
:10933000D4ED157A03EB02631B12F0EE475A07EEE9
:10934000103AB8EEC77A35EE265A27EE247A9DF801
:1093500004309DF80320A5EE076A1B0403EB0223EB
:1093600094ED1B7A9DF8052094ED135A35EEC77ADB
:10937000D4ED185AA7EE876A03EB02631B12F0EED6
:10938000667AE7EE257A9DF80620D4ED125AC6EEED
:10939000273A03A9204607EE903AF8EEE77A75EEF1
:1093A000A65A67EEA47A94ED0E6A9DF80730D4EDC4
:1093B0001C4AA5EEA76A1B0403EB0223D4ED165A40
:1093C0009DF80820F0EE467A94ED196AE7EE257ACA
:1093D00003EB02631B12F0EE665AE7EE065A0A220E
:1093E00035EE265A87EEA56A07EE903ADFED255A4C
:1093F000F8EEE77A67EEA57AD4ED0F5AE5EE275A34
:10940000D4ED177A94ED1A5AE7EE275AF0EE667A01
:10941000E7EE057AE4EEC46AC5EEA72AF0EE637AB9
:10942000E4EEC67A94ED1F7A87EEA65AF0EE467AFD
:10943000E4EE637AC7EEA65AF0EE437AD4EE077AEA
:10944000A4EEC37A26EE476AB2EE047AA7EEA36AC8
:1094500025EE075AC6EE267A65EE875A77EEA27A8F
:109460008DED035A67EE877ACDED045ACDED057A7E
:1094700000F04AFA06B010BD5B9E803A85EBCBC186
:1094800047ABE73BF61BEB3BFFF714BF30B513468A
:10949000026885B00D461AB90024204605B030BDDB
:1094A00000210160802001930392FDF74DFC0446EA
:1094B00020B1019B2A4603A9FFF744FC03A8FEF74D
:1094C00011FA002CE8D02046FFF744FE054600289C
:1094D000E3D1236820465B6898472C46DDE700000F
:1094E00010B5044B044640F82C3BFEF7FBF9204630
:1094F00010BD00BFC03D090810B50446FFF7F0FFDE
:109500002046FDF729FC204610BD0000064B10B593
:1095100003600446FEF7D6F9A06004F10C004EF09B
:109520009BFD204610BD00BFD83D090873B5054618
:109530007C23AC682E7903FB0643C6EB461604EB8E
:109540008604084693F8A410019010F019FA94F9D3
:109550003C3001983BB9AB6893F8251002B0BDE8E8
:10956000704010F00DBA94F84010F7E737B58468F2
:10957000057901917C2303FB054595F83F3004EB09
:109580008304D4F84C325BB14FF014FCC5F89C0056
:109590000199D4F84C0203B0BDE8304003F0F8BDA7
:1095A00003B030BD2DE9F04F90F804A08768CAEBF6
:1095B0004A144FEA840806460D4607F13C0B08F1B1
:1095C00008018BB05944284610F010F93179B06881
:1095D0000BEB8404FEF71CF938B17C2303FB0A7300
:1095E00093ED1A0A284610F035F97C2303FB0A7321
:1095F00093ED146ADFED3A7AD3ED156AB0EEC67AD0
:10960000B4EEE77AF1EE10FA0FD5B0EEE67AB4EEEA
:10961000E77AF1EE10FA08D594ED077AB0EEC77A42
:10962000B4EEE77AF1EE10FA1BD47C2303FB0A7345
:10963000D86D196E5A6E9B6D02900391049007913C
:1096400001A829468DED016ACDED056A06920892C2
:1096500009930EF029FA85ED000AC5ED010A85EDA2
:10966000021A7C2303FB0A770023C7F88C30C7F863
:109670008830C7F88430B06890F95C3208F13C0952
:1096800008F14808D944D8446BB133795BB94146F5
:1096900000F5167004F034FA414628460BB0BDE8D8
:1096A000F04F10F0A3B890F93430012B0BD190EDAE
:1096B0000E0A484610F07AF884ED120AC4ED130A37
:1096C00084ED141AE8E7022BE6D1FCF71DFF002217
:1096D00001A9FCF719FC0028DED09DED010AE8E79E
:1096E0000000003410B5037984687C2202FB034437
:1096F00007C904F1900383E807004FF05BFBC4F84F
:109700009C004FF04FFBC4F8A00010BDF0B505461B
:1097100085B0A6220E4600F10C0103A809F094FCC6
:10972000AC682F797C2303FB0743D3F8B42022B91C
:1097300003A809F0ABFC05B0F0BDBEB196ED007A10
:10974000D3ED2A7A67EE877AC3ED2A7A96ED017A0D
:10975000D3ED2B7A67EE877AC3ED2B7A96ED027AFA
:10976000D3ED2C7A67EE877AC3ED2C7A7C2607EE50
:10977000902A06FB0741A831B8EE670A0846019116
:1097800010F07CF801992846FFF7ACFF06FB074371
:109790000022C3F8B020C3F8AC20C3F8A8200022F0
:1097A000C3F8B420C4E7000073B504468068237989
:1097B00001917C2606FB03000D466C3001A92BF0BD
:1097C00011FCA368227906FB02331D6702B070BD4D
:1097D00070B5021D044680680E46FDF7FFFB054686
:1097E00018B131462046FFF7DFFF284670BD000064
:1097F00007B5826803797C2000FB032090F93C00C8
:1098000002280BD002F13C00C3EB43138DF8071084
:1098100000EB83000DF107012BF03EFB03B05DF878
:1098200004FB0000836802797C2101FB023393F979
:109830003C00003818BF012070470000836802799F
:109840007C2000FB023383F8A4107047F8B505466E
:1098500008460F4610F070F810B100242046F8BDFD
:10986000384610F04FF804460028F6D1AB6893F95B
:1098700034637EB1384610F097FB95ED097ADFED41
:109880001F7AF0EEC76AF4EEE76AF1EE10FA03D53C
:1098900085ED090A0124E1E777EE407A30EE076AA8
:1098A000F0EEE77AC7EE866AF6B207EE906A9FEDB1
:1098B000146AF8EE677A26EE866AF4EEC67AF1EE5E
:1098C00010FA48BFB2EE046ADFED0E7A45BFAB6A0C
:1098D00066EE866AB0EE676A87EEA66A46BF013317
:1098E000AB620124F7EE007A77EEC67A20EE060A24
:1098F000A7EE270A85ED090AB0E700BF0000003493
:1099000000004843CDCCCC3D2DE9F74304460E463C
:109910001746FFF70BFE31462046FFF727FE31467C
:109920002046FFF73FFE31462046FFF78FFF30B35A
:1099300004F10C01992201A809F086FBA56894F8AE
:1099400004804FF07C0909FB0854A83431462046B6
:109950000FF04CFF09FB0851D1F8B4300133C1F8C6
:10996000B4304FB1BB4207D35B08C1F8B430B0EE9E
:10997000000A20460FF082FF01A809F087FB03B020
:10998000BDE8F08310B50446FDF7C2FBC0B23C341D
:10999000C0EB401004EB800010BD0000F8B50A4E8B
:1099A000044600F5167704F5137555F8040B08B155
:1099B00003F022FFBD42F8D13368986A03680121A1
:1099C0005B689847EFE700BF105E002008B5FFF71F
:1099D000E5FF0000F0B5144E00EB810773780446F4
:1099E000D7F84C026FF3410387B00D467370C8B1CE
:1099F00002F0F0FA68B1737843F0100373702C44EE
:109A00000023A372D7F84C0207B0BDE8F04002F083
:109A100065BAD7F84C12684602F00CFB009B012B8C
:109A2000EDD1E8E707B0F0BDDC5E002070B506467A
:109A30000D46002445FA04F3DB07E1B202D53046B7
:109A4000FFF7C8FF0134032CF4D170BDFF21FFF7ED
:109A5000EDBF000030B500F5137587B000F5167442
:109A600055F8041B21B9A542FAD1002007B030BD3A
:109A7000684602F0DFFA009B013B022BF3D801207D
:109A8000F4E700002DE9F0472DED028B88B0044685
:109A90000D469046B0EE408AFDF702FE30B9002632
:109AA000304608B0BDEC028BBDE8F0872946204661
:109AB000FDF770FC06460028F1D004EB8507D7F8C7
:109AC0003C22D7F830329A4206D038F0BBF95C4AD3
:109AD000032133F085F8E2E7D7F84C3283B94FF42D
:109AE0009870FDF731F9814608B102F089FFC7F897
:109AF0004C92B9F1000F03D138F0A4F9514AE7E7CD
:109B0000B4F84A32D90711D505F0E8FD90F80823DA
:109B100090F8C43232B9B02202FB030090F8A130B1
:109B2000012B03D838F08EF9474AD1E72046FFF7DA
:109B300091FF20B9454A537843F00203537094F9DA
:109B4000353053B329462046FFF71CFF90F900300B
:109B5000002B53D029462046FFF714FF90F80490BD
:109B6000B9F12B0F19D829462046D7F84CA2FFF798
:109B700009FF94F9353090F90020022BD4BF002161
:109B80000121012BD4BF00230123003A009118BF0B
:109B900001224946504602F0B5F9631900229A7233
:109BA00075B3D4EDC10AB4F84822D7F84C0270EE70
:109BB000A00A2B46B0EE480A414602F0C3F994F8D9
:109BC0003E33002B31D1224A069412680127E773F5
:109BD000906A0268156D1F4A0792029309224FF49A
:109BE0000063CDE9003208AA12E906001A4BA84723
:109BF000C8B938F027F9194A02216AE79946B2E74D
:109C000029462046FFF7BEFE90F90030002BC8D051
:109C1000D4EDC10AB4F84822D4F84C022B46B0EE79
:109C2000480A4146C9E784F83E7300230DF1170145
:109C300004F124008DF817302BF038F930E700BF1D
:109C4000E83D09081A3E09083D3E0908DC5E00208F
:109C5000105E0020CD9901085B3E0908663E0908A8
:109C60002DE9F0412DED028B002443739DF8203047
:109C7000837305460F469046B0EE408A264647FA63
:109C800004F3DB07E1B210D5B0EE480A424628469D
:109C9000FFF7F8FE064640B939462846FFF7C6FEEC
:109CA000BDEC028B3046BDE8F0810134032CE6D1D7
:109CB000F6E70000F8B500242DED028B05460F46AF
:109CC000B0EE408A427383732646E1B2B0EE480A92
:109CD0003A462846FFF7D6FE0134002818BF06464C
:109CE000032CF2D1BDEC028B3046F8BDF0B500EB91
:109CF00081030D46D3F84C129BB0044611B90020E5
:109D00001BB0F0BD0BA802F079F96319987A00280E
:109D1000F6D10B9A002A48D0042AF0D101229A7277
:109D20000DAA07CA02AB83E8070010AA07CA05AF4D
:109D300087E8070013AA07CA9DED180A08AE86E84F
:109D400007001A46294620468DED010AFDF7C6FA9E
:109D50003A4629462046FDF76DFA32462946204606
:109D6000FDF77AFA9DED010A29462046FDF786FAAD
:109D70009DF8643083B129462046FFF703FE90F931
:109D800000304BB194F93530012B05DD9DF85D2095
:109D900029462046FDF7BAFA2046FFF75BFE20B9B8
:109DA000034A537843F0040353700120A8E700BF2F
:109DB000DC5E00202DE9F0410546884600F513776A
:109DC0000024012657F8043BE1B26BB148FA04F3D2
:109DD000DB0709D52846FFF789FF002857F8040C50
:109DE00008BF002602F07AF80134032CEAD130468D
:109DF000BDE8F0812E4B2DE9F04F1F68FB6A93F808
:109E00009C8087B00446B8F1000F38D1DFF8A8A0D5
:109E100000F5137600F1030B054656F8040BA5EB8D
:109E200004095FFA89F9E8B102F0C0F828B19AF89C
:109E3000013043F008038AF8013056F8040C02F0B0
:109E4000C9F8F8B9637B6BB1AB7A5BB956F8041CFF
:109E5000684602F0EFF8009B042B03D149462046E8
:109E6000FFF744FF01355D45D7D1124B204683F8FB
:109E70001280FFF7EFFD054630B10123237407B0D0
:109E8000BDE8F08F8046EDE7237C002BF7D0A37B65
:109E9000002BF4D0B86A03684FF47A715B68984776
:109EA000B86A03689B6B294607B0BDE8F04F1847B6
:109EB000105E0020BD5E0020DC5E0020F0B50025B5
:109EC00087B000F513762C46012756F8041B41B1E4
:109ED000684602F0AFF8009B1BB107FA05F31C437C
:109EE000E4B20135032DF0D1204607B0F0BD0000EB
:109EF0002DE9F04F2DED028B03270E7C9FED348A68
:109F000091B005468846B946AC5D0134E4B2B4FB75
:109F1000F9F303EB4303E41AE4B205EB8403D3F84B
:109F20004C1209B9AC554CE003A802F083F8DDF8F7
:109F30000CB00BF1FF33022BF4D8304631F028FC83
:109F40008246304632F0EEFB00F11B039A4508D200
:109F5000304633F04FF8002011B0BDEC028BBDE865
:109F6000F08FAC55284698F810A0FFF7A7FFDDED5D
:109F7000057A8DF83100FCEEE77A9DF810208DF817
:109F8000332017EE903A8DF8343006AB03CB1B88A4
:109F9000ADF83D305C221B23CDE90032CDF8350011
:109FA000CDF8391009AABF2150468DED098A8DEDF3
:109FB0000A8A8DED0B8A8DF830408DF832B031F081
:109FC00051FC013F17F0FF079ED10120C4E700BFFD
:109FD000000000002DE9F04F0F7CA1B00646884636
:109FE000032500EB070999F805400134E4B2032387
:109FF000B4FBF3F303EB4303E41AE4B206EB84038C
:10A00000D3F84C1211B989F805400AE011A801F003
:10A01000F5FFDDF844A0BAF1030F08DCBAF1000F38
:10A02000F1DA013D15F0FF05DDD1012012E0AAF1C2
:10A030000402032AF5D8384631F0AAFB8346384695
:10A0400032F070FB00F13602934506D2384632F00A
:10A05000D1FF002021B0BDE8F08F89F805403046DF
:10A0600098F810B0FFF72AFFDDF848E0CDF80CE0D3
:10A07000DDF84CE0CDF810E0DDF850E0CDF814E06C
:10A08000DDF854E0CDF818E0DDF858E0CDF81CE03C
:10A09000DDF85CE0CDF820E0DDF860E0CDF824E00C
:10A0A0003219DDF864E01C9BCDF828E0DDF868E0AB
:10A0B00092F80AC09DF874109DF87520CDF82CE038
:10A0C0000E93DDF86CE01E9B8DF835008DF83C108A
:10A0D0008DF83D20CDF830E08DF834408DF836A075
:10A0E0008DF837C02422CDF83E303623CDE900323A
:10A0F000C0212C2303AA584631F0B4FB91E700009D
:10A100007FB58A8B0B464AF2B9518A4205465FD029
:10A110004AF2BA518A4274D04AF2B8518A420BD1FB
:10A12000474A1268D26A92F89C203AB137F08AFE08
:10A13000444A052132F054FD042479E0D3ED007A3D
:10A14000F5EEC07AF1EE10FAF6D49FED3F7AF4EE18
:10A15000C77AF1EE10FAEFDC93ED017ADFED3B6A9E
:10A160001C6993ED030AB0EEC77AB4EEE67A93ED7C
:10A17000027AFCEEE77AB0EEC77AF1EE10FAB4EEAE
:10A18000E67A17EE903A54BF01260026F1EE10FA57
:10A1900054BF01220022003C18BF012413F0FF012C
:10A1A00010D18DED030A0292FDF700F89DED030A30
:10A1B000029A234631462846FFF77CFD0028BBD093
:10A1C000002435E0134600943246FFF749FDF5E7D9
:10A1D000D3ED007AF5EEC07AF1EE10FAACD49FED33
:10A1E0001A7AF4EEC77AF1EE10FAA5DCFCEEE77A03
:10A1F00017EE903A13F0FF0108BFFF21FFF7DAFDD9
:10A20000DCE7D3ED007AF5EEC07AF1EE10FA93D4E4
:10A210009FED0D7AF4EEC77AF1EE10FA8CDCFCEECD
:10A22000E77A17EE904A14F0FF0404D1FFF70EFC12
:10A23000204604B070BD2146FFF7F8FBC0E700BF21
:10A24000105E0020983E090800007F4300000034A3
:10A25000F0B58BB00E4614460746FFF793FB54301B
:10A2600007C884E8070031463846FFF78BFB90EDBE
:10A27000057ADFED267AB0EEC77AB4EEE77AF1EE32
:10A2800010FA054611D590ED067AB0EEC77AB4EE15
:10A29000E77AF1EE10FA08D590ED077AB0EEC77ABA
:10A2A000B4EEE77AF1EE10FA24D431463846FFF7DF
:10A2B00069FB016A426A836AE869D5F814E0D5F857
:10A2C00018C0099001A8CDF804E00291039204910E
:10A2D000CDF814C00693079208930DF091FD98B144
:10A2E000214601A80DF0E0FB84ED000AC4ED010A4F
:10A2F00084ED021A31463846FFF744FB00F10801AD
:10A3000020460FF08DFA01200BB0F0BD00000034A4
:10A310002DE9F0472DED048BACB0B0EE608A054618
:10A32000B0EE409A0F46F0EE418A9046FCF73EFFB1
:10A33000DFED8B7AB0EEC87AB4EEE77AF1EE10FA80
:10A340004BD5B0EEE87AB4EEE77AF1EE10FA44D5E8
:10A3500023AC2046FCF7D4F9F8F798FE2146F8F72D
:10A3600049FC064658BB05F0B9F990F8083390F857
:10A37000C42233B1B02303FB020393F8A130012BB5
:10A3800007D84FF0B00909FB020090F8A130022B6A
:10A390000BD837F057FD734A032132F021FC3046C9
:10A3A0002CB0BDEC048BBDE8F08705F097F990F870
:10A3B000C43209FB0300AC300FC884E80F00DDEDA8
:10A3C000257A9FED691AB8EEE78ADDED267AF8EE78
